:100000000C948D0B0C94BE0B0C94BE0B0C94BE0B7D
:100010000C94BE0B0C94BE0B0C94BE0B0C94BE0B3C
:100020000C94BE0B0C94BE0B0C94BE0B0C94BE0B2C
:100030000C94BE0B0C94B5130C94BE0B0C94BE0B1D
:100040000C94BE0B0C94BE0B0C94BE0B0C94BE0B0C
:100050000C94BE0B0C94BE0B0C94BE0B0C940410B1
:100060000C94BE0B0C94FF9E0C94D59E0C94BE0B6E
:100070000C94BE0B0C94BE0B0C94BE0B0C94BE0BDC
:100080000C94BE0B0C94BE0B0C94BE0B0C94BE0BCC
:100090000C94AB9E0C94819E0C94BE0B0C9440155A
:1000A0000C94BE0B0C94BE0B0C94BE0B0C94BE0BAC
:1000B0000C94BE0B0C94BE0B0C94BE0B0C94BE0B9C
:1000C0000C94BE0B0C94BE0B0C94BE0B0C94579E60
:1000D0000C942D9E0C94BE0B0C94039E0C94D99DF5
:1000E0000C94BE0B084AD73B3BCE016E84BCBFFDCF
:1000F000C12F3D6C74319ABD56833DDA3D00C77FF8
:1001000011BED9E4BB4C3E916BAAAABE0000008090
:100110003F07634236B79BD8A71A39685618AEBA5C
:10012000AB558C1D3CB7CC5763BD6DEDFD753EF6F0
:10013000177231BF000000803F08000000BE92240B
:1001400049123EABAAAA2ABECDCCCC4C3E00000040
:1001500080BEABAAAAAA3E00000000BF000000803B
:100160003F0000000000084178D3BB4387D1133D16
:10017000190E3CC3BD4282AD2B3E68EC8276BED9DF
:100180008FE1A93E4C80EFFFBE01C4FF7F3F00001E
:10019000000000000C94080C0C94D9770C94598C36
:1001A0000C94EB810C94308C0C94458C0C94C38B88
:1001B0000C9472890C949E130C94E9780C94580C4E
:1001C0000C945D8C0C9475750C94C00B0C94618C24
:1001D0000C94678C0C94EA750C948C0C0C949B8595
:1001E0000C94AD7E0C9472780C942F820C946978E8
:1001F0000C944E100C94A88A0C94C9740C94D27C64
:100200000C9468890C9466780C9481810C94418CD0
:100210000C94FE8A0C946F790C94128B0C94AA7532
:100220000C94668C0C946C780C94A9760C94EE81EA
:100230000C9490750C94268C0C94B7850C94A17535
:100240000C94A98A0C94538C0C947B780C94060C17
:100250000C94348C0C94DE830C9488890C942C8C34
:100260000C946B8C0C94180C0C94D90C0C9478781E
:100270000C94A0760C94EF8A0C944F8C0C946F78AD
:100280000C943B8C0C94B5890C9432820C94B2760D
:100290000C94768B0C9427890C94D6810C9441870E
:1002A0000C940D880C944EAD0C94090C0C94D586CE
:1002B0000C94F3750C944B8C0C9460750C942B0C73
:1002C0000C9475780C94588A0C94FC750C94FE7AF6
:1002D0000C9450780C94BD890C94F77A0C94C70B4D
:1002E0000C948A0C0C94AB0D0C946D890C94B20D8B
:1002F0000C947E750C9425880C94070C0C94D9757D
:100300000C94AE0D0C94208B0C942D880C940576D7
:100310000C94388C0C9487750C9484800C94857D97
:100320000C94870C0C947E780C9493AC4E414E49FF
:100330004E495459494E46CDCCCC3D0AD7233C17A3
:10034000B7D13877CC2B329595E6241FB14F0A00F0
:100350000020410000C84200401C4620BCBE4CCAE0
:100360001B0E5AAEC59D7400407A10F35A00A0725D
:100370004E18090010A5D4E80000E87648170000E0
:10038000E40B54020000CA9A3B000000E1F50500AE
:100390000080969800000040420F000000A08601F7
:1003A000000000102700000000E8030000000064C7
:1003B00000000000000A0000000000010000000032
:1003C000002C76D888DC674F0823DFC1DFAE59E107
:1003D000B1B796E5E3E453C63AE651997696E8E676
:1003E000C28426EB898C9B62ED407C6FFCEFBC9C49
:1003F0009F40F2BAA56FA5F490055A2AF75C936B5B
:100400006CF9676DC11BFCE0E40D47FEF520E6B515
:1004100000D0ED902E0300943577050080841E08EF
:100420000000204E0A000000C80C333333330F980D
:100430006E12831141EF8D2114893BE65516CFFED4
:10044000E6DB18D1844B381BF77C1D901DA4BBE460
:1004500024203284725E228100C9F124ECA1E53DA2
:10046000274E6F2053656E736F7221004E6F2044CC
:100470005320546865726D6F6D6574657221004418
:100480005320546865726D2E004D6F74696F6E0055
:1004900046696E64696E6720576946692049500055
:1004A0007365703D006976616C3D006E69746572BC
:1004B0003D00230043616C2E204661696C65640039
:1004C00043616C2E20446F6E65004E6F206E656533
:1004D000642100496E76616C69642050285061295E
:1004E000005365614C6576656C2050285061293A4F
:1004F0000043616C696272617465205000416972E9
:100500002054656D70286F43293A0043616C2E209A
:100510004D6F74696F6E004453542054656D7020A4
:1005200073656E736F720043757272656E742073BB
:10053000656E736F72004F322073656E736F720059
:1005400055562073656E736F720043616C696272F9
:10055000617465004661696C6564005442206361A2
:100560006C2E20646F6E65005570706572204C694A
:100570006D69743A3E004C6F776572204C696D6905
:10058000743A3E0054757262696469747900466118
:10059000696C65640070482063616C2E20646F6E26
:1005A00065007048313020507265737320420070CE
:1005B000483420507265737320410043616C696256
:1005C00072617465004E45543D426C7565746F6F81
:1005D0007468204C45004E45543D426C7565746FFF
:1005E0006F7468004E45543D576946690053657401
:1005F00074696E67204661696C6564005365747444
:10060000696E6720446F6E65004368616E676520A0
:100610004E6574776F726B3E00547970653A004294
:10062000542F57694669204E6574776F726B00438B
:1006300068616E67652053656E736F723E00437527
:100640007272656E742053656E736F72004F7468BA
:10065000657200496E642E20342D32306D410041A8
:100660004353373132203C3330410041435337311B
:1006700032203C32304100414353373132203C3547
:1006800041003E4D617820566F6C743A3E004368DD
:10069000616E676520766F6C746167653E005479A2
:1006A00070652000566F6C746167652053656E73CA
:1006B0006F72004368616E6765207479706520749D
:1006C0006F0053656E736F723D4448540054656DFE
:1006D000702048756D6964697479002028303D6127
:1006E00075746F3B313D616363656C3B323D696E90
:1006F000636C20616E676C65290023416363656CE0
:1007000065726174696F6E20413D00556E6B6E6F4E
:10071000776E00496E647573747269616C20342D54
:1007200032306D4100414353373132204D61783DC5
:100730003541002343757272656E742073656E7364
:100740006F723A00696E7075742044535463616C23
:100750006962726174653A0020766F6C74616765D6
:100760003D00235475726269646974792055707014
:100770006572204C696D69743A200020766F6C7444
:100780006167653D002354757262696469747920FC
:100790004C6F776572204C696D69743A2000235460
:1007A0007572626964697479204C6F776572204C48
:1007B000696D69742056696E663A20004D61782033
:1007C00072616E67653D0023566F6C7461676520CA
:1007D00073656E736F723A00342D32306D41004193
:1007E0004353373132204D61783D00414353373117
:1007F00032204D61783D3541002343757272656E3C
:10080000742073656E736F723A00234453205468EA
:1008100065726D6F6D657465722063616C6962727B
:100820006174656420666F72202300445354002372
:100830004E6F206E65656420746F2063616C696221
:10084000726174652063757272656E742073656E73
:10085000736F722100234143533731322063757225
:1008600072656E742073656E736F72206F66667347
:10087000657420563D00235556207A65726F2076A8
:100880006F6C74616765203D0055565A00234F32E6
:1008900020766F6C253D00234F322063616C6962C6
:1008A000726174696F6E3A200023566F6C746167D1
:1008B000652870483D3130293A0023566F6C7461C9
:1008C00067652870483D34293A0050483400555433
:1008D000454D503D004448543D00413D002354697E
:1008E0006D65206475726174696F6E3D0023546993
:1008F0006D6520696E74657276616C3D005769465E
:10090000692049503A00234D5320456E61626C6561
:100910006400234D532044697361626C6564002355
:100920005265737420706172616D657465727320B5
:10093000746F2064656661756C742076616C756592
:1009400073004C6F67676572204E616D653A2000D9
:10095000697465726174696F6E3D0073656E736F63
:1009600072233D0043757272656E742073746174F6
:1009700075733A206379636C653D006E6379636CCF
:10098000653D006E73656E736F72733D006D6178C7
:100990006E73656E736F72733D00656E61626C6538
:1009A000643D00234D756C746973656E736F72736B
:1009B000206D6561737572656D656E742073657405
:1009C00074696E67733A002353657474696E677354
:1009D000206F6620616C6C2073656E736F72733A62
:1009E000002353697A65206F6620686561646572CB
:1009F000202B20616C6C2073656E736F72733A20CC
:100A0000002353697A65206F6620686561646572AA
:100A10003A20004F6666206169722D636F6E642113
:100A2000004974277320746F6F20636F6F6C21000F
:100A300054656D702069732066696E652100497385
:100A4000206169722D636F6E64206F6E3F00497480
:100A5000277320717569746520686F74210049746B
:100A60002773207665727920686F742120004F66A5
:100A700066206169722D636F6E642100497427736B
:100A800020746F6F20636F6F6C210054656D702050
:100A900069732066696E6521004973206169722D52
:100AA000636F6E64206F6E3F004974277320717509
:100AB00069746520686F7421004974277320766516
:100AC000727920686F74210054656D702048756DCF
:100AD0006964697479002320616E642072656164C1
:100AE0007920746F207573652100206D6F62696CC9
:100AF00065206C6F676765722073746172746564DA
:100B0000200043616C6962726174696F6E2050727B
:100B10006573737572653D00536561206C6576651C
:100B20006C20502863616C63293D00234572726F0D
:100B3000723A707265737375726520424D50303829
:100B4000352C20636865636B20776972696E672155
:100B50000049522054656D702073656E736F72206A
:100B6000666F756E6400206D6F62696C65206C6FD6
:100B7000676765722073746172746564202E2E2E0F
:100B80002000576946692049503A00235769466951
:100B900020495020616464726573733A2000456493
:100BA00055484B205345534C6F676765720053653A
:100BB0006E736F7220736C6F7420616E6420747931
:100BC00070653A0057656C636F6D6520746F2045E2
:100BD0006455484B00005EBCE2613FDD83C29C7EF1
:100BE00020A3FD1F41009D23BE46DB65F88C11AF9D
:100BF00032CA57E974232D2D2D2D2D2D2D2D2D2D60
:100C00002D2D2D2D2D2D2D2D2D2D2D2D2D2D2D2D14
:100C10002D2D2D2D2D2D2D2D2D2D00235265736F56
:100C20006C7574696F6E3A20202000234D696E2028
:100C300056616C75653A2020202000234D61782094
:100C400056616C75653A202020200023556E69712D
:100C500075652049443A202020200023447269769B
:100C60006572205665723A202020002353656E730A
:100C70006F723A2020202020202000232D2D2D2DA2
:100C8000204D61676E657469632053656E736F7282
:100C9000202D2D2D2D2D2D2D2D2D2D2D2D2D2D2D91
:100CA0002D2D2D2D2D00482D6669656C643A202868
:100CB0000020202020202020202020202020202054
:100CC0002000202020202020202020202020202044
:100CD0002020002020202020202020202020202034
:100CE0002020200020202020202020202020202024
:100CF0002020202000202020202020202020202014
:100D00002020202000202020202020202020202003
:100D10002020202000233A53686F772F48696465AC
:100D2000204C4344002A3A546869732048656C702B
:100D30000044233A43616C6962726174696F6E00AA
:100D4000442A3A53657474696E67730044423A5298
:100D500065736574204C6F676765720044433A435E
:100D60006C656172204C43440044443A4D756C7488
:100D70006953656E736F72730044393A43757272CA
:100D8000656E7400566F6C746167652B4375727283
:100D9000656E740044383A456C656374726963002B
:100DA00044373A4D6F74696F6E0044363A445320AD
:100DB00054656D700044353A555620496E74656E21
:100DC000736974790044343A4F3220636F6E632E36
:100DD0000044333A434F3220636F6E632E00443237
:100DE0003A504D28313A322E353A313029004432CA
:100DF0003A504D28313A322E353A3130292A0044C2
:100E0000313A5475726269646974790044303A56B3
:100E10006F6C7461676500393A6F722033442061EA
:100E20006363656C2E00393A496E636C2E20616EE7
:100E3000672E00383A70482076616C756500373A45
:100E400049522054656D7000373A49522054656DFF
:100E5000702A00363A4D61676E6574696320666971
:100E6000656C6400353A476173204C6576656C00AB
:100E7000343A495220466C616D6500333A4C6967DB
:100E8000687420496E742E00323A616E64204865A1
:100E90006967687400323A54656D702050726573EA
:100EA0007375726500313A54656D702048756D69CF
:100EB0006469747900303A536F756E64204C6576BE
:100EC000656C00303A536F756E64204C6576656CC6
:100ED0002A0054696D65206C617073653A0057692A
:100EE00046692049503A004D6F74696F6E0055563F
:100EF00020496E742E00555620496E74656E7369D4
:100F00007479004F3220436F6E6300434F322043A9
:100F10006F6E630053656E736F72206572726F72CD
:100F20002100234E6F2073656E736F722100434F53
:100F30003220436F6E63004D6561737572696E6731
:100F400000234E6F2073656E736F7220666F722080
:100F5000504D21004E6F2073656E736F722100201B
:100F60006E672F4C00504D313A322E353A313000F9
:100F70004D6561737572696E672E2E00234E6F206A
:100F800054422073656E736F723F00234E6F20735F
:100F9000656E736F722100536F756E64204C6576B9
:100FA000656C004D6561737572696E672E2E002346
:100FB0004E6F2073656E736F722100536F756E6490
:100FC000204C6576656C00234E6F2073656E736FE1
:100FD0007220666F722074656D7020262068756DB2
:100FE000696469747921004E6F2053656E736F7266
:100FF000210020666F722074656D70202620687550
:101000006D696469747921002353656E736F722072
:101010004572726F72200053656E736F7220457255
:10102000726F7221002357726F6E672073656E7343
:101030006F7220666F722074656D7020262068754F
:101040006D6964697479210057726F6E672053650A
:101050006E736F72210054656D702048756D696400
:10106000697479004C6967687420496E74656E73A1
:1010700069747900466C616D6520495200234E6F9A
:101080002070482073656E736F722100704820765F
:10109000616C75650023496E76616C6964206B65CF
:1010A000792100204D756C746973656E736F72736E
:1010B000004D756C746973656E736F72730044696B
:1010C0007361626C6500456E61626C6500526562B9
:1010D0006F6F74696E672E2E2E002344413A2D32B5
:1010E000330050686F6E652053656E736F720041F8
:1010F0006363656C65726174696F6E004F726965D8
:101100006E742E2F496E636C2E00416E672E205632
:10111000656C6F6369747900436F6D702E202620B3
:10112000482D6669656C64004750530050726F78B3
:10113000696D697479004C6967687420496E7465DB
:101140006E736974790041697220507265737375AA
:1011500072650054656D7020262048756D6964695C
:10116000747900237265706C6965733D00676574FE
:1011700053656C665465737442697428293A20007B
:101180006973496E74657272757074456E61626CD4
:1011900065642831293A2000676574496E74657268
:1011A000727570744D617070696E672831293A20CC
:1011B00000676574496E74657272757074536F75EB
:1011C0007263652831293A2000676574496E746539
:1011D0007272757074536F7572636528293A2000B6
:1011E0006765745261746528293A20332E31343191
:1011F00035393F00616363656C2E69734C6F7750BE
:101200006F77657228293A2000616363656C2E69E7
:101210007341736C65657028293A200061636365CA
:101220006C2E6973546170536F757263654F6E5A9B
:1012300028293A2000616363656C2E6973546170DC
:10124000536F757263654F6E5928293A20006163A8
:1012500063656C2E6973546170536F757263654F6B
:101260006E5828293A2000616363656C2E697341CA
:1012700063746976697479536F757263654F6E5ADA
:1012800028293A2000616363656C2E697341637499
:101290006976697479536F757263654F6E59282941
:1012A0003A200069734163746976697479536F7584
:1012B0007263654F6E5828293A2000697354617033
:1012C000446574656374696F6E4F6E5A28293B20BC
:1012D00066616C73653F2000697354617044657486
:1012E000656374696F6E4F6E5A28293B207472755E
:1012F000653F200069735461704465746563746967
:101300006F6E4F6E5928293B2066616C73653F20D4
:10131000006973546170446574656374696F6E4FDE
:101320006E5928293B20747275653F2000697354FB
:101330006170446574656374696F6E4F6E582829D7
:101340003B2066616C73653F200069735461704493
:101350006574656374696F6E4F6E5828293B2074FD
:101360007275653F200067657453757070726573A0
:101370007342697428293B2066616C73653F2000C5
:101380006765745375707072657373426974282948
:101390003B20747275653F20006973416374697600
:1013A000697479416328293A20006973496E616341
:1013B0007469766974795A456E61626C656428292E
:1013C0003A20006973496E6163746976697479596A
:1013D000456E61626C656428293A20006973496E24
:1013E000616374697669747958456E61626C65648D
:1013F00028293A2000697341637469766974795ABF
:10140000456E61626C656428293A20006973416306
:1014100074697669747959456E61626C65642829CE
:101420003A20006973416374697669747958456E2E
:1014300061626C656428293A2000676574467265AC
:101440006546616C6C4475726174696F6E28293AE7
:1014500020006765744672656546616C6C546872FD
:101460006573686F6C6428293A2000676574546955
:101470006D65496E616374697669747928293A20CB
:1014800000676574496E616374697669747954683C
:10149000726573686F6C6428292000676574416306
:1014A0007469766974795468726573686F6C6428BE
:1014B000292000676574446F75626C6554617057CC
:1014C000696E646F7728292000676574446F7562C0
:1014D0006C655461704C6174656E637928293A209B
:1014E000006765745461704475726174696F6E2829
:1014F000293A2000676574417869734F66667365A1
:10150000742826782C2026792C20267A293A200047
:101510006765745461705468726573686F6C642891
:10152000293A200058595A2047733A200058595AEE
:1015300020434F554E54533A200073657420676121
:10154000696E735B5D3A006761696E735F6F7269A4
:10155000675B5D3A00416E676C65732F00496E638F
:101560006C2E20616E672E004E6F2073656E736F58
:1015700072210049522054656D70657261747572F4
:1015800065004D6561737572696E672E2E004E6F32
:101590002073656E736F723F0049522054656D7001
:1015A00065726174757265004D6561737572696EFF
:1015B000672E2E0000002100240027002A002D00A5
:1015C0003000330001010000040107010A0100009E
:1015D0002200250028002B002E00310034000201DB
:1015E0000000050108010B01000020002300260077
:1015F00029002C002F003200000100000301060129
:101600000901050505050705080808080202020288
:101610000A0A08080404040401010101010101018E
:101620000303030303030303040707070C0C0C0C59
:101630000C0C0C0C02020202060606060606060642
:101640000B0B0B0B0B0B0B0B0102102020080810CF
:101650002040102040800201020108040201010222
:1016600004081020408080402010080402018004FB
:101670000201804020100804020108040201010256
:10168000040810204080010204081020408000005F
:101690000A0B02090C0D0E080703040100000000EC
:1016A000000000000000000000000000000000003A
:1016B00000000000000000000000121110000000F7
:1016C000000000000000000000000000000000001A
:1016D0000000000023456E64206F66204D756C7419
:1016E0006973656E736F72204379636C652300497B
:1016F0006E76616C6964206B65792100482D66699E
:10170000656C640053656172636820446972656347
:1017100074696F6E00004EAD93AC11241FBECFEF05
:10172000D1E2DEBFCDBF00E00CBF1CE0A0E0B2E024
:10173000EEE8FFE701E00BBF02C007900D92A23177
:10174000B107D9F724E1A2E1BCE001C01D92A630A7
:10175000B207E1F71BE0CCE8DBE000E006C0219730
:101760000109802FFE010E94D5BCCB38D10780E053
:101770000807A9F70E94E1AF0C94B5BF0C940000D4
:1017800080915A0D90915B0D891B990B08950895D6
:10179000DC0180E0615090F09D919827E92FEF7077
:1017A000F0E0EB52F44F2491E92FE295EF70F0E076
:1017B000EB51F44FE491822F8E27ECCF08952091C6
:1017C000AC0C260F3327331F21323105ECF4209166
:1017D000D40DFC0190E080E0243069F082E00895AF
:1017E000A091AC0C2191AC014457534FA40FB52FDD
:1017F000B11D2C930196861798F38091AC0C680F5D
:101800006093AC0C80E0089581E0089508950895F8
:101810000895E0915B0D80915A0DE81730F4F0E0E7
:10182000E65CF24F808190E008958FEF9FEF08957E
:1018300090915B0D80915A0D2FEF3FEF981748F470
:10184000E92FF0E0E65CF24F208130E09F5F90935B
:101850005B0DC9010895CF92DF92EF92FF920F9333
:101860001F93CF93DF937C01CB018A012091DA0D86
:10187000222389F0EB016B01C40ED51ECC15DD05CA
:1018800069F06991D701ED91FC910190F081E02D13
:10189000C7011995F3CF642F0E94DF0BC801DF91B8
:1018A000CF911F910F91FF90EF90DF90CF9008950F
:1018B000CF93DF931F92CDB7DEB769832091DA0D06
:1018C0002223F9F02091FC0D203258F021E030E085
:1018D000FC013383228390E080E00F90DF91CF9171
:1018E00008958091DB0DE82FF0E0E452F24F9981EA
:1018F00090838F5F8093DB0D8093FC0D81E090E0FF
:10190000ECCF61E0CE0101960E94DF0BF7CF90E0B3
:1019100080E008950C94C3BD0F931F93CF93DF9382
:101920008C01EB0188E2FB0111928A95E9F74BE00B
:1019300050E067EB75E0CE010E948CBF1B8681E012
:1019400090E0A0E0B0E08C879D87AE87BF87F8016C
:1019500085899689A789B08D888B998BAA8BBB8B3B
:1019600082E090E0A0E0B0E08C8B9D8BAE8BBF8BD3
:101970001CA21DA21EA21FA280E090E0A8E4B4E475
:10198000888F998FAA8FBB8F80E090E0A8E4B4EC99
:101990008C8F9D8FAE8FBF8F8DEC9CECACE4BEE343
:1019A00088A399A3AAA3BBA3DF91CF911F910F9105
:1019B0000895AF92BF92CF92DF92EF92FF920F9372
:1019C0001F93CF93DF938C01EB0184E2FB01119213
:1019D0008A95E9F78EE10E94DB8D83E090E00E941A
:1019E000D68D0E94FCA266E08EE10E9414A31092A4
:1019F0005B0D80935A0D8630F0F30E941491A82E4F
:101A00000E941491B82E0E941491E82E0E94149105
:101A1000F82E0E941491C82E0E941491D82E60E0D6
:101A20007A2D6B29072E000C880B990B0E94B1B7F9
:101A3000F801658376838783908760E07C2D6D292C
:101A4000072E000C880B990B0E94B1B7F801618733
:101A500072878387948760E07E2D6F29072E000CA4
:101A6000880B990B0E94B1B7F80165877687878745
:101A7000908B118A128A138A148A84E290E0A0E083
:101A8000B0E088839983AA83BB8385899689A789D7
:101A9000B08D8C839D83AE83BF8382E090E0A0E015
:101AA000B0E088879987AA87BB87188A198A1A8A1B
:101AB0001B8AC090E004D090E104E090E204F09032
:101AC000E304A701960165817681878190850E9454
:101AD00029BA20E030E048EC52E40E9410B86C8B48
:101AE0007D8B8E8B9F8BA7019601F8016185728596
:101AF000838594850E9429BA20E030E048EC52E4C6
:101B00000E9410B8688F798F8A8F9B8F2091DC0498
:101B10003091DD044091DE045091DF04F8016585C9
:101B20007685878590890E9429BA20E030E048ECCC
:101B300052E40E9410B86C8F7D8F8E8F9F8F81E052
:101B4000DF91CF911F910F91FF90EF90DF90CF9099
:101B5000BF90AF900895862F0C94299F862F642FF5
:101B60000C94529F862F642F0C9441A01F93CF9307
:101B7000DF93EC01162F60E0812F0E9441A0612FBE
:101B800070E0FB01E85BF94EE491E883FB01EE5F56
:101B9000F94EE491F0E0EE0FFF1FE851FA4E859107
:101BA00094919A8389831B861D861C861A861986C2
:101BB00018861F821E821D821C821B82DF91CF919C
:101BC0001F910895EFE4F1E114A215A216A217A245
:101BD00010A611A612A613A681E084A729E130E081
:101BE00036A725A787A780E090E0A0EAB0E480AB05
:101BF00091ABA2ABB3AB80E090E0A8EAB1E484ABD8
:101C000095ABA6ABB7AB8093D8049093D904A093BF
:101C1000DA04B093DB0480E090E0A0E8BFE38093B7
:101C2000991190939A11A0939B11B0939C1180935A
:101C3000D4049093D504A093D604B093D704109203
:101C4000C6111092C5118BE090E09093C81180935B
:101C5000C7119093D3048093D2041092D61110929E
:101C6000D51190E080E00C947F902F923F924F929C
:101C70005F926F927F928F929F92AF92BF92CF921C
:101C8000DF92EF92FF920F931F93CF93DF936C013C
:101C9000CDE3D5E083E9882E84E0982E0FE411E1AE
:101CA000EE24E394F12C22E1222E312C33E1432E59
:101CB000512C40E1642E712C51E1A52EB12C809164
:101CC0009304909194048E159F050CF4C9C021E0F3
:101CD000C216D10409F0BDC0F80182AD93ADF40184
:101CE00093838283F40182819381009709F58A812D
:101CF0009B819093050280930402F4018281938179
:101D000084309105C1F52A813B81309307022093ED
:101D100006028531910509F47BC08631910509F0F1
:101D200040C02A813B8130937C0420937B044EC0C9
:101D30008130910539F48A819B8190938704809347
:101D40008604DBCF8230910539F48A819B819093A0
:101D5000030280930202D1CF039779F68A819B8197
:101D600090930102809300026BEF7BE080E493E1AB
:101D70000E945E98C2CF8530910539F42A813B815B
:101D800030937A0420937904C4CF8630910529F2E8
:101D900087309105B9F42A813B81309380042093E8
:101DA0007F048731910591F42A813B8128303105E8
:101DB000B1F570928F0460928E04B0928D04A0925F
:101DC0008C0404C08A30910509F0A3CF9C012B50EC
:101DD00031092A30310590F42A813B813093010288
:101DE0002093000239E1389FB001399F700D112412
:101DF000685F7D4F80E493E10E94C1988FEFE81AFD
:101E0000F80A2296E2E08E0E911C0E5F1F4F57CF0C
:101E10002A813B8130937E0420937D04D7CF2730E5
:101E2000310549F430928F0420928E0450928D0433
:101E300040928C04CBCF2630310541F621E030E0D2
:101E400030938F0420938E0410928D0410928C0492
:101E5000BDCFF40182819381F80193AF82AF42CF6D
:101E6000DF91CF911F910F91FF90EF90DF90CF9076
:101E7000BF90AF909F908F907F906F905F904F90AA
:101E80003F902F9008950F931F93CF93DF938C0172
:101E90001092130C1092120CC091120CD091130CD2
:101EA000C832D105A4F4809106020E94C4A1CC0FCF
:101EB000DD1FC25AD24F998388838091120C909172
:101EC000130C01969093130C8093120CE5CF0E9493
:101ED000238E20E030E040EA50E40E9410B820E079
:101EE00030E040E85AE30E9410B80430110599F43C
:101EF00020E030E040E650E40E9410B89B01AC01C5
:101F000060E070E080E890E40E944AB9DF91CF91F0
:101F10001F910F9108950A30110569F420E030E017
:101F200040E650E40E9410B89B01AC0160E070E014
:101F300080E291E4E9CF60E070E0CB01E7CF0F935E
:101F40001F9360E080918E040E94529F83E090E096
:101F50000197F1F761E080918E040E94529F83E225
:101F600090E00197F1F760E080918E040E94529F0B
:101F700080918C0490918D049927FC01E85BF94EC7
:101F80006491FC01EE5FF94EE491F0E0EE0FFF1F6B
:101F9000E851FA4E8591949100E717E120E030E096
:101FA000462F0E944EAC611571058105910529F0FF
:101FB0006F5F7F4F8F4F9F4F9F700E94B1B720E0A0
:101FC00030E44CE156E40E9429BA2091300C309163
:101FD000310C4091320C5091330C0E9410B820E02B
:101FE00030E048E453E40E9429BA1F910F9108950C
:101FF0002FB7F8946091D00C7091D10C8091D20CD5
:102000009091D30C2FBF08951F920F920FB60F928D
:1020100011242F933F938F939F93AF93BF938091FE
:10202000D00C9091D10CA091D20CB091D30C3091E6
:10203000CF0C23E0230F2D3758F50196A11DB11DBC
:102040002093CF0C8093D00C9093D10CA093D20C02
:10205000B093D30C8091220D9091230DA091240D6B
:10206000B091250D0196A11DB11D8093220D909375
:10207000230DA093240DB093250DBF91AF919F9197
:102080008F913F912F910F900FBE0F901F90189539
:1020900026E8230F0296A11DB11DD2CF0895DF922D
:1020A000EF92FF920F931F93CF93DF937C018B01ED
:1020B000D42EDC011696ED91FC91138615861486BC
:1020C0001286118610861782168215821482138258
:1020D000C0E0B801F701868197810E94C797D82F89
:1020E000882329F0DC1629F0CF5FDC1690F7D0E0CA
:1020F00009C067E0C8010E94C80BD80117969C91DF
:102100008913F2CF8D2FDF91CF911F910F91FF9007
:10211000EF90DF900895DC012C911196ED91FC91E8
:10212000F8948181822B81839281322F3095932381
:10213000928387E090E00197F1F781818323818387
:1021400083E290E00197F1F790817894EFECF0E072
:102150003197F1F7922381E009F480E00895FC01C2
:1021600090810180F281E02D292F209560FF14C01D
:10217000F8948281822382838181892B8183A3E2E7
:10218000B0E01197F1F78281982B9283789487EDD4
:1021900090E00197F1F70895F89482818223828379
:1021A0008181892B8183AFEFB0E01197F1F78281B4
:1021B000982B928378948FE090E0EBCFDF92EF92B0
:1021C000FF920F931F93CF93DF93EC01D62EE42E53
:1021D00008E010E0FF24F39461E08D2D8F2109F4D5
:1021E00060E0CE010E94AF10FF0C01501109A1F771
:1021F000E11010C0F894E981FA819181888180957D
:1022000089238183E981FA8192818881809589235C
:1022100082837894DF91CF911F910F91FF90EF907F
:10222000DF900895EF92FF920F931F93CF93DF9368
:102230008C017B0140E065E50E94DE10E70188E04B
:10224000E80EF11C699140E0C8010E94DE10CE1535
:10225000DF05C1F7DF91CF911F910F91FF90EF90B4
:102260000895FC0190810180F281E02DF894818134
:10227000292F20958223818378943DE743E050E025
:10228000315029F1DA011197F1F780818923C1F3E7
:10229000F8948281822382838181892B818378943F
:1022A000ABE7B7E01197F1F7F8948181822381833E
:1022B000A3E1B1E01197F1F78081982381E009F063
:1022C00080E07894E3E6F6E03197F1F7089580E056
:1022D00008958F929F92AF92BF92CF92DF92EF922A
:1022E000FF92CF93DF93EC018E819F810E94311189
:1022F00040E06CEC8E819F810E94DE10488164E496
:102300008E819F810E94DE108A81882371F1E9818C
:10231000E9508EEEC82E82E0D82EE33038F4F0E09B
:10232000EE0FFF1FEB5AFA4FC080D1808B818823BC
:1023300039F18881811124C00E94F80F4B015C01A2
:102340000D2C000CEE08FF088E819F810E948B10DF
:10235000813059F00E94F80F6C197D098E099F0990
:10236000681579058A059B0578F3DF91CF91FF9079
:10237000EF90DF90CF90BF90AF909F908F90089597
:10238000B601DD0C880B990BDF91CF91FF90EF9098
:10239000DF90CF90BF90AF909F908F900C9439A515
:1023A0006F927F928F929F92AF92BF92CF92DF9265
:1023B000EF92FF920F931F93CF93DF93EC017B017A
:1023C0008A018E819F810E943111811102C090E0AB
:1023D00037C0B7018E819F810E94121140E06EEBE1
:1023E0008E819F810E94DE107801680189E0C80E0D
:1023F000D11CAE80BF8088E0882E912C712C662481
:102400006394C5010E948B1081117628660CE1E06F
:102410008E1A9108B1F7F70171927F01EC15FD0555
:1024200041F78E819F810E943111813081F668E0F1
:10243000C8010E94C80B91E0F80120852813C7CF7E
:10244000892FDF91CF911F910F91FF90EF90DF9037
:10245000CF90BF90AF909F908F907F906F90089596
:10246000CF93DF9300D000D000D0CDB7DEB7AE0160
:102470004F5F5F4F0E94D011882331F08D818F33E1
:10248000A9F020F48F31A1F080E007C08F3521F052
:102490008F37D1F78CE001C08BE029960FB6F89406
:1024A000DEBF0FBECDBFDF91CF9108958AE0F5CF9B
:1024B00089E0F3CF0F931F93CF93DF93CDB7DEB7B0
:1024C00061970FB6F894DEBF0FBECDBF8C01462FCB
:1024D000BE01665F7F4F0E944F1081110FC060E008
:1024E00070E08EEF92EC61960FB6F894DEBF0FBEEF
:1024F000CDBFDF91CF911F910F910895AE014F5F36
:102500005F4FBE01665F7F4FC8010E94D0118823D4
:1025100031F36A8170E0762F6627770F770F770F98
:10252000298148E0249F90011124262B372B8A858E
:102530008031D1F4688570E08F81AB01481B51096F
:10254000CA019695982F8827979587950E94C1BCB8
:10255000CB014097B90153E0660F771F5A95E1F719
:1025600060789C01260F371F213854EE35070CF494
:10257000B6CFB901330F880B990B0E94B1B720E099
:1025800030E040E05CE30E9410B8ADCFEF92FF92E4
:102590000F931F93CF93DF9300D000D01F921F9211
:1025A000CDB7DEB78C01DC011696ED91FC91179743
:1025B0001386158614861286118610861782168257
:1025C00015821482138214961C92149715961C92ED
:1025D000EE24E394BE016F5F7F4FF80186819781FF
:1025E0000E94C797882309F46FC067E0CE01019667
:1025F0000E94C80B98858913EDCFD8018C91811169
:1026000025C016968D919C910E943111BE016F5F7D
:102610007F4FF801868197810E94121140E064EBA0
:10262000D80116968D919C910E94DE10F80186814A
:1026300097810E948B10F82ED80116968D919C914F
:102640000E943111F11002C0F801E082D801119608
:10265000FC9089818031A1F1BE016F5F7F4FC8017D
:102660000E9430128F15D0F4F8018181D8011196A3
:102670008C93119714968C9114978F5F14968C936A
:102680008981883231F0B0F4803119F0823209F05A
:10269000A1CFF80185818F5F85839CCF89818031AF
:1026A00011F48CE0E3CFBE016F5F7F4FC8010E9441
:1026B0003012DCCF8B3369F3823409F08BCFE9CF52
:1026C000FCE0FF1588F2EDCF28960FB6F894DEBF38
:1026D0000FBECDBFDF91CF911F910F91FF90EF9073
:1026E00008950F931F93CF938C01C62FFC01848113
:1026F0000E94DB8DF80183858C2B90E00E94D68DA3
:10270000CF911F910F910C94FCA20F931F93CF9325
:102710008C01C62F0E9471136C2F6460C8010E9447
:1027200071136C2F6B7FC8010E94711383EC90E0D2
:102730000197F1F7CF911F910F9108950F931F9378
:10274000CF938C01C62F607F61600E94851380E16A
:10275000C89FB00111246160C8010E94851381E007
:1027600090E0CF911F910F9108951F920F920FB695
:102770000F9211240BB60F922F933F934F935F93B9
:102780006F937F938F939F93AF93BF93EF93FF9339
:1027900080917E100E94299F20918110309182109B
:1027A0002F5F3F4F309382102093811090918010C3
:1027B000953618F096E090937D1090917D109430AE
:1027C00009F46EC0F8F4923031F1933009F44CC042
:1027D00090917F10992319F0811171C02F9AFF9168
:1027E000EF91BF91AF919F918F917F916F915F9189
:1027F0004F913F912F910F900BBE0F900FBE0F90F6
:102800001F901895953009F457C0963009F791E05C
:1028100090934D114FC08111DBCF209181103091E9
:1028200082102436310528F4109282101092811003
:10283000CFCF10924D1110928010E091801091E056
:102840009E0F90938010F0E02091811030918210C3
:10285000EE0FFF1FED57FF4E318320831092821041
:102860001092811093E019C0813009F0B1CFE0914E
:10287000801091E09E0F90938010F0E020918110E5
:1028800030918210EE0FFF1FED57FF4E31832083F2
:10289000109282101092811094E090937D1098CF46
:1028A000882359F22091811030918210253631050C
:1028B00008F48ECF95E0F1CF81118ACFB5CF2F9854
:1028C0008ECFCF92DF92EF92FF92CF93DF93EC0106
:1028D000072E000C880B990B0E94B1B76B017C018D
:1028E00020E030E040E45FE30E9410B820E030E0F8
:1028F00048E452E40E9429BA0E94D5BAC617D70705
:10290000D4F020E030E040EA5FE3C701B6010E9466
:1029100010B820E030E048E452E40E9429BA20E0F8
:1029200030E040E85FE30E944BB90E94D5BA21E055
:102930006C177D070CF420E0822F90E0DF91CF919F
:10294000FF90EF90DF90CF9008950F931F93CF9358
:10295000DF93082F61EA7BE084ED9FE00E94939D66
:10296000C7E0D0E010E0B8010C2E02C07595679565
:102970000A94E2F76170772742E050E084ED9FE02F
:102980000E94469D219778F7DF91CF911F910F917B
:1029900008951092D40D81E08093D30D1092AE0D66
:1029A00061E084E10E94529F61E085E10E94529FB4
:1029B000E9EBF0E080818E7F808380818D7F808352
:1029C00088E48093B80085E48093BC000895CF9399
:1029D000DF9391E090938B0C8823B9F0C091B800FD
:1029E000D091BA008091BC008A7B8093BC0060E0EB
:1029F00084E10E94529F60E085E10E94529F0E9404
:102A0000C914D093BA00C093B800DF91CF91089554
:102A100085ED8093BC008091D60D9091D70DA0914B
:102A2000D80DB091D90D0796A11DB11D23E0B69523
:102A3000A795979587952A95D1F72091BC0024FDFD
:102A400003C01092D40D08954091D60D5091D70D2A
:102A50006091D80D7091D90D452B462B472B69F30A
:102A60000097A105B10541F025E32A95F1F7000093
:102A70000197A109B109E1CF8091D50D0C94E7141C
:102A80001F920F920FB60F9211240BB60F922F9335
:102A90003F934F935F936F937F938F939F93AF93E6
:102AA000BF93EF93FF938091B900887F803609F43C
:102AB0004DC008F040C0883209F4A9C028F5803123
:102AC00009F49DC0C8F4882309F4FBC0883009F4D8
:102AD00096C0FF91EF91BF91AF919F918F917F91A0
:102AE0006F915F914F913F912F910F900BBE0F907F
:102AF0000FBE0F901F901895883109F488C080325E
:102B000041F78093D20D14C0803409F49DC040F485
:102B10008033B9F38833E9F68093D20D85ECB0C0E9
:102B2000803509F485C0883509F496C0883489F663
:102B30000E940815CECF883909F48CC038F5883743
:102B400029F050F4883611F0803719F683E080932D
:102B5000D40D1092CE0C57C0883809F47BC0803950
:102B600019F0803809F0B5CF8091CE0C803208F092
:102B700071C0E091CE0C81E08E0F8093CE0C8091DD
:102B8000BB00F0E0E255F34F80833DC0803B39F05D
:102B9000E0F4803A09F479C0883A09F09ACF84E0E9
:102BA0008093D40D1092AD0C1092AC0CE091380DC6
:102BB000F091390D19958091AC0C81110FC081E015
:102BC0008093AC0C10928C0C09C0803C09F4A6CF09
:102BD000883C09F4A3CF883B09F07BCFE091AD0C92
:102BE00081E08E0F8093AD0CF0E0E457F34F8081CD
:102BF0008093BB009091AD0C8091AC0C29C080916A
:102C0000AF0D8093BB0085EC8093BC0062CF9091A8
:102C1000D10D8091D00D981758F5E091D10D81E03C
:102C20008E0F8093D10DF0E0E055F24F8081E9CF17
:102C3000E091D10D81E08E0F8093D10D8091BB008A
:102C4000F0E0E055F24F80839091D10D8091D00D4E
:102C50009817C8F285E8D8CFE091D10D81E08E0FAA
:102C60008093D10D8091BB00F0E0E055F24F80835E
:102C70008091D30D81115CCF81E08093AE0D84EA09
:102C80008093BC001092D40D24CF85EC8093BC00BF
:102C90001092D40D8091CE0C803230F4E091CE0CA5
:102CA000F0E0E255F34F10826091CE0C70E0E091BD
:102CB000360DF091370D8EEA9CE019951092CE0CEE
:102CC00008CF1092D20D34CF23E333E948E853E420
:102CD0000E9429BA20E030E040E85FE30E944BB94F
:102CE0000E9453BC26E636EA45EA53E40E9410B837
:102CF0006093300C7093310C8093320C9093330CB2
:102D00000895CF92DF92EF92FF920E949F0F6B0186
:102D10007C0120E030E040E050E40E9432BB181615
:102D200024F40E949F0F6B017C0120E030E040E022
:102D300050E4C701B6010E9432BB181624F40E9469
:102D40009F0F6B017C0120E030E040E050E4C701C0
:102D5000B6010E9432BB181624F40E949F0F6B012B
:102D60007C0120E030E040E050E4C701B6010E9461
:102D700032BB181624F40E949F0F6B017C0120E0E7
:102D800030E040E050E4C701B6010E9432BB1816A3
:102D90002CF4C12CD12CE12C80E4F82EC701B60113
:102DA000FF90EF90DF90CF90089581E08093E5044D
:102DB00080918504882341F088E08093FE1360E0D1
:102DC00083EF93E10C947113089580918504811130
:102DD00010C081E0809385048093E5048091F9130D
:102DE000982F94609093F9138C600E94E58D0C9459
:102DF000D5168091E5048823D1F31092FE1360E08C
:102E000083EF93E10E9471131092E5048091F9130E
:102E10008B7F8093F91388600E94E58D1092850462
:102E200008952F923F924F925F926F927F928F926E
:102E30009F92AF92BF92CF92DF92EF92FF920F9349
:102E40001F93CF93DF93CDB7DEB766970FB6F89495
:102E5000DEBF0FBECDBF1C0187E39FE00E94F6904E
:102E600040E855E260E070E087E39FE00E94F4579D
:102E700064E670E080E090E00E9439A58CED95E07A
:102E8000A0E0B0E080933B0F90933C0FA0933D0FE8
:102E9000B0933E0F64E670E080E090E00E9439A5B8
:102EA0008FEF8A8781E08B8786E88C871D861E8658
:102EB0001F86188A198A89E78A8BC101880F991F92
:102EC0009E8B8D8BD12CC12CF12CE12C412C512CC3
:102ED000320187E39FE00E94EF8A08974CF049E0B7
:102EE00050E0BE01665F7F4F87E39FE00E94A98AA2
:102EF00065E070E080E090E00E9439A510E000E01D
:102F0000812C912C540187E39FE00E94208B892B18
:102F100039F4F4E08F169104A104B1040CF04EC012
:102F2000023011050CF04AC087E39FE00E94208B1D
:102F3000892B69F087E39FE00E94FE8AE1E0F0E0E0
:102F4000EC0FFD1FE00FF11F80830F5F1F4F65E047
:102F500070E080E090E00E9439A50230110509F090
:102F600073C099818A8598136FC09A818C85981354
:102F70006BC0FE013396FC8BEB8B87E39FE00E94D6
:102F8000208B892B39F4F4E08F169104A104B1044D
:102F90000CF053C00930110509F05CC08B8190E042
:102FA000982F88272C81820F911D092E000CAA0BC7
:102FB000BB0B480E591E6A1E7B1E43C08FEFC81AFA
:102FC000D80AE214F30434F4ED89FE89EC15FD050A
:102FD00009F07FCF87E39FE00E94F690E114F104AF
:102FE00009F47101C301B2010E94B1B74B015C0148
:102FF000B701FF0C880B990B0E94B1B79B01AC0184
:10300000C501B4010E9429BA66960FB6F894DEBFD6
:103010000FBECDBFDF91CF911F910F91FF90EF9029
:10302000DF90CF90BF90AF909F908F907F906F90E8
:103030005F904F903F902F900895043011050CF051
:10304000ADCFFFEFEF1AFF0A8FEF881A980AA80A90
:10305000B80A59CF87E39FE00E94FE8AEB89FC897A
:103060008193FC8BEB8B0F5F1F4F87CF4F925F924B
:103070006F927F929F92AF92BF92CF92DF92EF9228
:10308000FF920F931F93CF93DF93982E8EE0A82E7D
:10309000B12CEE24EA9493E0F92E0FEF13E0D12C3B
:1030A000C12CD0E0C0E0412C512C3201892D0E946E
:1030B000C4A1C817D90708F44AC0C816D90608F42D
:1030C0006C018017910708F444C08E159F0508F421
:1030D0007C01BC0190E080E00E94AFB79B01AC0195
:1030E000C301B2010E944BB92B013C0165E070E0C5
:1030F00080E090E00E9439A581E0A81AB108B1F6FD
:10310000BE016C0D7D1D6E0D7F1D600F711F90E067
:1031100080E00E94AFB79B01AC01C301B2010E94E5
:103120004AB920E030E040E251E40E9429BADF9140
:10313000CF911F910F91FF90EF90DF90CF90BF90B4
:10314000AF909F907F906F905F904F900895EC01AB
:10315000B8CF8C01BECF4F925F926F927F92AF92A9
:10316000BF92CF92DF92FF920F931F93CF93DF9383
:1031700000D000D0CDB7DEB75C0187E39FE00E94AE
:10318000F69040E052EC61E070E087E39FE00E943F
:10319000F4578CED95E0A0E0B0E080933B0F909366
:1031A0003C0FA0933D0FB0933E0F64E670E080E0CB
:1031B00090E00E9439A5D12CC12CF12C65E070E083
:1031C00080E090E00E9439A510E000E0412C512CF5
:1031D0003201F1103AC087E39FE00E94208B892BD7
:1031E00031F485E1481651046104710474F503302B
:1031F00011055CF587E39FE00E94208B892B69F025
:1032000087E39FE00E94FE8AE1E0F0E0EC0FFD1F03
:10321000E00FF11F80830F5F1F4F65E070E080E0DB
:1032200090E00E9439A5023011054CF089818B3B5A
:1032300031F4FF24F3948A818A3A09F0F12C8FEF5C
:10324000481A580A680A780AC4CF8FEFC81AD80AF1
:1032500064E670E080E090E00E9439A5AC14BD0403
:1032600009F0ACCF8F2D26960FB6F894DEBF0FBEB7
:10327000CDBFDF91CF911F910F91FF90DF90CF9045
:10328000BF90AF907F906F905F904F9008951F9385
:10329000CF93DF93182FCEE5DDE0812F0E94C4A1EC
:1032A000899399936CE370E080E090E00E9439A5E7
:1032B0008DE0CE3AD80789F70E94238E20E030E0D7
:1032C00040EA50E40E9410B820E030E040E85AE3C1
:1032D0000E9410B8DF91CF911F9108958F929F9215
:1032E000AF92BF92CF92DF92EF92FF920F931F9314
:1032F000CF93DF93CDB7DEB762970FB6F894DEBFFA
:103300000FBECDBF20913C0C222309F4D5C02091E3
:10331000610C3091620C263531050CF0CDC0E09087
:103320008304F090840449EDE4164FE0F4060CF0B9
:10333000C3C08C012F5F3F4F3093620C2093610C10
:103340000E94F80F8090340C9090350CA090360CB1
:10335000B090370C681979098A099B090E94AFB7A8
:1033600020E030E04AE754E40E9429BA6093380C28
:103370007093390C80933A0C90933B0C88E5E816D7
:1033800082E0F80634F488E592E090938404809318
:103390008304809183049091840438E3E32E3CE01D
:1033A000F32EFC01E853FC406F01C6018E0D9F1DFA
:1033B0009A838983F70161917F01CE0101960E9472
:1033C000DB57FCE3EF16FCE0FF0679F780918304FE
:1033D0009091840404969093840480938304B801AC
:1033E000CE0101960E94419BCE0101960E94499A0E
:1033F000BC01CE010D960E94419BCE0101960E9418
:10340000DE9AF80184819581849708F123E230E007
:1034100050E040E0B801CE0101960E945B9BBE01E6
:103420006F5F7F4FCE0107960E94419BCE010796AA
:103430000E94499ABC01CE010D960E948E9ACE013F
:1034400007960E94DE9ACE0101960E94DE9A498973
:103450005A894115510531F06DE37CE0CE010D969E
:103460000E94A990809183049091840421E6C22E49
:103470002CE0D22E0DE31CE09C012D533C40790141
:10348000C701800F911F9A838983F80161918F0191
:10349000CE0101960E94DB57C016D10689F78091B4
:1034A000830490918404849690938404809383048D
:1034B000CE010D960E94DE9A62960FB6F894DEBF9A
:1034C0000FBECDBFDF91CF911F910F91FF90EF9075
:1034D000DF90CF90BF90AF909F908F900895EF9224
:1034E000FF920F931F93CF93DF93CDB7DEB768970B
:1034F0000FB6F894DEBF0FBECDBF8C0161E67AE057
:10350000CE010D960E944A9B6FEB75E0CE0143966B
:103510000E944A9B63EA79E0C8010E94389BBE0181
:103520006D5E7F4FC8010E94629A6AE979E0C80126
:103530000E940B9A86EEE82E81E1F82EF701608159
:1035400070E0CE0101960E949598BE016F5F7F4F9B
:10355000CE0107960E94419BBE01635F7F4FCE0163
:1035600007960E94F899BC01C8010E94629ACE0198
:1035700007960E94DE9ACE0101960E94DE9A6DE8BF
:1035800079E0C8010E940B9AF7016181062E000CB8
:10359000770BCE0101960E949598BE016F5F7F4F19
:1035A000CE0107960E94419BBE01635F7F4FCE0113
:1035B00007960E94F899BC01C8010E94629ACE0148
:1035C00007960E94DE9ACE0101960E94DE9A63E879
:1035D00079E0C8010E940B9AF7016281062E000C67
:1035E000770BCE0101960E949598BE016F5F7F4FC9
:1035F000CE0107960E94419BBE01635F7F4FCE01C3
:1036000007960E94F899BC01C8010E94629ACE01F7
:1036100007960E94DE9ACE0101960E94DE9A6BE721
:1036200079E0C8010E940B9AF70163817481CE0191
:1036300001960E949598BE016F5F7F4FCE0107965D
:103640000E94419BBE016D5E7F4FCE0107960E9496
:10365000F899BC01C8010E94629ACE0107960E94A7
:10366000DE9ACE0101960E94DE9A64E679E0C801F6
:103670000E940B9AF70165817681CE0101960E9426
:103680009598BE016F5F7F4FCE0107960E94419BC8
:10369000BE01635F7F4FCE0107960E94F899BC017F
:1036A000C8010E94629ACE0107960E94DE9ACE015E
:1036B00001960E94DE9A6BE579E0C8010E940B9AA0
:1036C000F7016781062E000C770B6F5F7F4FCE01ED
:1036D00001960E949598BE016F5F7F4FCE010796BD
:1036E0000E94419BBE01635F7F4FCE0107960E94FF
:1036F000F899BC01C8010E94629ACE0107960E9407
:10370000DE9ACE0101960E94DE9A60E579E0C8015A
:103710000E940B9AF7016085062E000C770BCE01F4
:1037200001960E949598BE016F5F7F4FC8010E946D
:10373000629ACE0101960E94DE9ACE0143960E94C3
:10374000DE9ACE010D960E94DE9AC80168960FB6E9
:10375000F894DEBF0FBECDBFDF91CF911F910F91C7
:10376000FF90EF9008954F925F926F927F929F9299
:10377000AF92BF92CF92DF92EF92FF920F931F937F
:10378000CF93DF93CDB7DEB7A8970FB6F894DEBF1F
:103790000FBECDBF6AE073E184E093E10E948E9A90
:1037A0000E9447986FEE75E0CE0101960E944A9BF9
:1037B000BE016F5F7F4F84E093E10E94C799182F8D
:1037C000CE0101960E94DE9A112309F4F7C0809180
:1037D0000E1390910F134097B8F080E0A8960FB6A3
:1037E000F894DEBF0FBECDBFDF91CF911F910F9137
:1037F000FF90EF90DF90CF90BF90AF909F907F9021
:103800006F905F904F90089542E050E06AE073E15E
:10381000CE0101960E943858BE016F5F7F4F86EE41
:1038200092E10E94A59ACE0101960E94DE9A66EE70
:1038300072E1CE0101960E94419BCE0101960E9449
:10384000A359CE0101960E94DE9A86EE92E10E9473
:10385000D09820E030E048EC52E40E9410B80E947A
:10386000D5BAAB01BC014093C5045093C604609324
:10387000C7047093C804CE0101960E946898CE01D7
:1038800001960E94A359CE0101960E94DE9A609192
:10389000C5047091C6048091C7049091C8048B013F
:1038A0009C0100591F452140310901341C49210563
:1038B0003105C8F162EC75E0CE0101960E944A9B89
:1038C00066EE72E1CE0101960E94F89965ED75E011
:1038D0000E94E299BC018CEE92E10E948E9ACE0188
:1038E00001960E94DE9A60EC75E0CE0101960E947E
:1038F0004A9B6CEE72E1CE0101960E94F899BC01E0
:10390000CE0145960E94419BCE0145960E94F256FB
:10391000CE0145960E94DE9ACE0101960E94DE9A63
:103920001092EA0489C01A821982FE01339626E0B9
:10393000DF011D922A95E9F70E94B1B720E030E03F
:1039400048EC52E40E9429BA8E010F5F1F4F22E01B
:1039500047E00E9406B3BC018CEE92E10E94C19840
:1039600065EE75E0CE0145960E944A9B6CEE72E1D1
:10397000CE0145960E94F89962EF75E00E94E299A7
:10398000BC018CEE92E10E948E9ACE0145960E9477
:10399000DE9A8091C5049091C604A091C704B091AD
:1039A000C80480934F1190935011A0935111B0937C
:1039B000521190E080E00E947F9095CF6AED78E010
:1039C000CE0101960E94389BBE016F5F7F4F84E05D
:1039D00093E10E94C799182FCE0101960E94DE9AAA
:1039E000112389F142E050E06AE073E1CE010196D3
:1039F0000E943858BE016F5F7F4F86EE92E10E94B1
:103A0000A59ACE0101960E94DE9A86EE92E10E946E
:103A1000DB986330710590F470932F0C60932E0C3B
:103A200080912E0C90912F0C9093D6118093D511EC
:103A300090E080E00E947F9081E0D0CE10922F0C29
:103A400010922E0CEDCF65ED78E0CE0101960E942C
:103A5000389BBE016F5F7F4F84E093E10E94C7995E
:103A6000182FCE0101960E94DE9A1123A1F126E0C3
:103A700030E044E050E06AE073E1CE0101960E943C
:103A80005B9BBE016F5F7F4F86EE92E10E94A59A1D
:103A9000CE0101960E94DE9A86EE92E10E94DB98AA
:103AA0007093C8116093C7117093D3046093D204CC
:103AB0006AE073E1CE0101960E94419BCE0101961E
:103AC0000E94A359CE0101960E94DE9A90E080E008
:103AD0000E947F9025CF6EEC78E0CE0101960E9487
:103AE000389BBE016F5F7F4F84E093E10E94C799CE
:103AF000182FCE0101960E94DE9A1123A1F146E013
:103B000050E06AE073E1CE0101960E943858BE0190
:103B10006F5F7F4F86EE92E10E94A59ACE010196DB
:103B20000E94DE9A8091EA129091EB12892B61F04B
:103B300086EE92E10E94D098609388047093890485
:103B400080938A0490938B046AE073E1CE0101961E
:103B50000E94419BCE0101960E94A359CE0101967D
:103B60000E94DE9ADDCE67EF75E0CE0101960E94DD
:103B70004A9BBE016F5F7F4F84E093E10E94C7992B
:103B8000182FCE0101960E94DE9A112309F4BEC0BF
:103B90006AEC78E0CE0101960E94389BBE016F5F0F
:103BA0007F4F84E093E10E94C799182FCE010196C0
:103BB0000E94DE9A1123D1F184E090E00E94430F2D
:103BC0006093A9047093AA048093AB049093AC040F
:103BD0006AEB78E08CEE92E10E94699A4091A90428
:103BE0005091AA046091AB047091AC0422E0CE0124
:103BF00001960E94E69ABE016F5F7F4F8CEE92E1C4
:103C00000E94629ACE0101960E94DE9A8091A904D8
:103C10009091AA04A091AB04B091AC04809373116D
:103C200090937411A0937511B09376116AEF75E0BB
:103C3000CE0101960E944A9BBE016F5F7F4F84E0D8
:103C400093E10E94C799182FCE0101960E94DE9A37
:103C50001123F1F18AE090E00E94430F6093A504E4
:103C60007093A6048093A7049093A80469EA78E06F
:103C70008CEE92E10E94699A4091A5045091A604AD
:103C80006091A7047091A80422E0CE0101960E94E1
:103C9000E69ABE016F5F7F4F8CEE92E10E94629ABE
:103CA000CE0101960E94DE9A8091A5049091A6040F
:103CB000A091A704B091A8048093771190937811F4
:103CC000A0937911B0937A1190E080E00E947F90E8
:103CD00060EC75E0CE0101960E944A9B6CEE72E1A9
:103CE000CE0101960E94F899BC01CE0145960E9432
:103CF000419BCE0145960E94F256CE0145960E9408
:103D0000DE9ACE0101960E94DE9A96CE6FEF75E0A4
:103D1000CE0101960E944A9BBE016F5F7F4F84E0F7
:103D200093E10E94C799182FCE0101960E94DE9A56
:103D3000112309F4BDC080910E1390910F130797C2
:103D4000F8F046E050E06AE073E1CE0101960E948F
:103D50003858BE016F5F7F4F86EE92E10E94A59AB0
:103D6000CE0101960E94DE9A86EE92E10E94D098E2
:103D70006093D8047093D9048093DA049093DB04A1
:103D800080917F049091800499270E9436182DE03D
:103D900038E643E55BE30E9410B86B017C0120919B
:103DA0000705309108054091090550910A050E94C8
:103DB000AAB718160CF460C06091EF047091F0047B
:103DC0008091F1049091F20420E030E048EC52E45C
:103DD0000E9410B86B017C0120E030E0A9010E9434
:103DE000AAB7181634F0C12CD12C38EAE32E31E4EE
:103DF000F32EC092D804D092D904E092DA04F09263
:103E0000DB04C0928311D0928411E0928511F0926C
:103E100086118091310D882381F067E978E084ED87
:103E20009FE00E94B59D6091D8047091D904809163
:103E3000DA049091DB040E94379D90E080E00E94BC
:103E40007F906DE878E08CEE92E10E94699A409153
:103E5000D8045091D9046091DA047091DB0422E017
:103E6000CE0101960E94E69ABE016F5F7F4F8CEEF5
:103E700092E10E94629AA7C020911B0530911C0517
:103E800040911D0550911E05C701B6010E9432BB2D
:103E900087FF05C0C701B6010E944D8F95CF609185
:103EA00003057091040580910505909106058CCF5E
:103EB00069E878E0CE0101960E94389BBE016F5FF1
:103EC0007F4F84E093E10E94C799182FCE0101969D
:103ED0000E94DE9A112309F47BC060E080917D048A
:103EE0000E9441A009E110E0C12CD12C7601809103
:103EF0007D040E94C4A1BC01990F880B990B0E94FC
:103F0000B1B79B01AC01C701B6010E944BB96B016F
:103F10007C016AE070E080E090E00E9439A50150E9
:103F2000110929F720E030E040EA50E4C701B6016A
:103F30000E9410B820E030EC4FE754E40E9429BA08
:103F400020E030E048EC51E40E9429BA6093D404A8
:103F50007093D5048093D6049093D70460939911FD
:103F600070939A1180939B1190939C1190E080E044
:103F70000E947F9066E778E08CEE92E10E94699A59
:103F80004091D4045091D5046091D6047091D70427
:103F900022E0CE0101960E94E69ABE016F5F7F4F3C
:103FA000CE0145960E94419B65E076E0CE014596A4
:103FB0000E94E299BC018CEE92E10E94629ACE01CD
:103FC00045960E94DE9ACE0101960E94DE9A56C066
:103FD00068E076E0CE0101960E944A9BBE016F5FC9
:103FE0007F4F84E093E10E94C799182FCE0101967C
:103FF0000E94DE9A112309F44CC080917E11082E94
:10400000000C990B0197039798F589E390E00E94C3
:1040100036182AE137E64CE950E40E9410B8609364
:104020007F1170938011809381119093821190E0A1
:1040300080E00E947F9065E578E08CEE92E10E943E
:10404000699A40917F115091801160918111709116
:10405000821122E0CE0101960E94E69ABE016F5FB6
:104060007F4FCE0145960E94419B6EE076E09ECF49
:104070006FE278E08CEE92E10E94699A6CEE72E158
:10408000CE0101960E94419BCE0101960E94F256FC
:1040900065CD6BE278E0CE0101960E94389BBE01AF
:1040A0006F5F7F4F84E093E10E94C799182FCE0184
:1040B00001960E94DE9A112309F43CC126E030E00B
:1040C00044E050E06AE073E1CE0101960E945B9B00
:1040D000BE016F5F7F4F86EE92E10E94A59ACE01EE
:1040E00001960E94DE9A86EE92E10E94DB986B01B7
:1040F0005B016BE679E0CE0101960E944A9BBE010E
:104100006F5F7F4F8AE093E10E9491998E010B5E71
:104110001F4FAC014F5F5F4F6AE073E1C8010E941F
:104120003858B80186EE92E10E94A59AC8010E9413
:10413000DE9ACE0101960E94DE9A90907B0486EE74
:1041400092E10E94D0982B013C018091310D88238F
:10415000B9F064E477E084ED9FE00E94B59D4AE009
:1041600050E0B60184ED9FE00E94469D61E67AE052
:1041700084ED9FE00E94939DC301B2010E94379D90
:10418000692DC8010E94B60D18870F831D821E82FB
:10419000198289E08A8381E08B838C831C8A1B8A45
:1041A000CE0101960E94C612CE0101960E946911AD
:1041B000CE0101960E94A2A80E8110E00B301105DD
:1041C00014F00AE010E0BBE5CB16D10408F44EC0B1
:1041D00023E6C22E2CE0D22E5601412C512C320166
:1041E000F12CE12C0E151F05B9F06E2DCE010196B4
:1041F0000E945A129B01AC01F50121933193419326
:1042000051935F01C301B2010E944BB92B013C01E4
:10421000FFEFEF1AFF0AE6CFB7010F2C000C880B57
:10422000990B0E94B1B79B01AC01C301B2010E947E
:1042300029BA2B013C0110E000E0E016F106B9F1CB
:10424000D6012D913D914D915D916D015D01B4E0DF
:10425000AB1AB108C301B2010E944AB9F5016083EB
:104260007183828393830F5F1F4FE7CF1A141B0460
:104270000CF041C00A151B050CF086010150110914
:10428000602FCE0101960E945A129B01AC01000FD3
:10429000111F000F111F0D59134FC301B2010E94CE
:1042A0004AB9D8016D937D938D939C931397E3E660
:1042B000FCE0ADE9B1E18BE89CE041915191619165
:1042C00071914D935D936D937D938E179F07A9F721
:1042D00090E080E00E947F906AE078E08CEE92E1CE
:1042E0000E94699A44E050E06AE073E1CE010196D1
:1042F0000E943858B9CDA114B104C9F683E6E82E5E
:104300008CE0F82E0A151B0591F26A2DCE0101965C
:104310000E945A129B01AC01C301B2010E944AB92A
:10432000F70161937193819391937F01FFEFAF1A2E
:10433000BF0AE8CF61E176E0CE0101960E944A9B78
:10434000BE016F5F7F4F84E093E10E94C799182FF1
:10435000CE0101960E94DE9A112309F423C127E0C1
:1043600030E046E050E06AE073E1CE0101960E9441
:104370005B9BBE016F5F7F4F86EE92E10E94A59A24
:10438000CE0101960E94DE9A86EE92E10E94DB98B1
:104390007B0160937E118AE093E10E94E69861E6DA
:1043A0007AE0CE0101960E944A9BBE016F5F7F4F6B
:1043B0008AE093E10E949199AC014F5F5F4F6AE000
:1043C00073E1CE0145960E943858CE0145960E9471
:1043D000D09860937F117093801180938111909396
:1043E0008211CE0145960E94DE9ACE0101960E946E
:1043F000DE9A69EF77E08CEE92E10E94699A44E0E0
:10440000E416F1041CF582E0E816F1040CF09FC0FC
:10441000E114F10431F1EA94EF2809F471C06091DC
:104420007E11062E000C770BCE0145960E949598C2
:1044300063E276E0CE0101960E944A9BBE016B5E6C
:104440007F4FCE0101960E94F8994CC0B4E0EB1664
:10445000F10429F768ED77E08CEE92E10E940B9A67
:1044600071C020E030E0A90160917F11709180114E
:1044700080918111909182110E94AAB7181664F060
:1044800080E090E0A0E8BFE380937F1190938011DB
:10449000A0938111B093821120917F1130918011EE
:1044A000409181115091821160E070E080EA90E4C7
:1044B0000E9429BAAB01BC0122E0CE0145960E94C0
:1044C000E69A68E176E0CE0101960E944A9BBE0121
:1044D0006B5E7F4FCE0101960E94F8996CE17BE004
:1044E0000E94E299BC018CEE92E10E94629ACE0198
:1044F00001960E94DE9ACE0145960E94DE9A22C065
:104500006BEE77E08CEE92E10E940B9A20E030E0B7
:1045100048E453E460917F11709180118091811182
:10452000909182110E94AAB7181664F080E090E47E
:10453000ACE1B5E480937F1190938011A093811139
:10454000B093821190E080E00E947F9097CD6FED54
:1045500077E08CEE92E10E940B9A8AE08E9DB0018A
:104560008F9D700D1124CE0101960E949598BE0179
:104570006F5F7F4FCE0145960E94419B65E17BE0D6
:10458000CE0145960E94E299BC018CEE92E10E9418
:10459000629ACE0145960E94DE9ACE0101960E9453
:1045A000DE9AB4CF6AE276E0CE0101960E944A9B81
:1045B000BE016F5F7F4F84E093E10E94C799182F7F
:1045C000CE0101960E94DE9A112309F4CCC027E0A7
:1045D00030E046E050E06AE073E1CE0101960E94CF
:1045E0005B9BBE016F5F7F4F86EE92E10E94A59AB2
:1045F000CE0101960E94DE9A86EE92E10E94DB983F
:1046000060937B118AE093E10E94E69886EE92E146
:104610000E94DB98611571058105910509F074C050
:1046200085E090E090937D1180937C1190E080E094
:104630000E947F9067EC77E08CEE92E10E94699A8D
:1046400080917B11833044F56CEB77E08CEE92E146
:104650000E940B9A60917C1170917D11CE010196A0
:104660000E949598BE016F5F7F4FCE0145960E94D4
:10467000419B6BE37AE0CE0145960E94E299BC0132
:104680008CEE92E10E94629ACE0145960E94DE9ADB
:10469000CE0101960E94DE9A80917B1183300CF44A
:1046A000EDCC60917C1170917D11CE0183960E94BA
:1046B000959860917B11062E000C770BCE014596E4
:1046C0000E94959863E276E0CE0101960E944A9B93
:1046D000BE016B5E7F4FCE0101960E94F899BE012C
:1046E0006D5D7F4F0E94F899BC018CEE92E10E94B3
:1046F000629ACE0101960E94DE9ACE0145960E94F2
:10470000DE9ACE01839661CC6130710581059105F9
:1047100019F489E190E086CF61E67AE0CE01019656
:104720000E944A9BBE016F5F7F4F8AE093E10E9427
:104730009199AC014F5F5F4F6AE073E1CE014596FE
:104740000E943858CE0145960E94DB9870937D11E7
:1047500060937C11CE0145960E94DE9ACE010196AF
:104760000E94DE9A63CF61E376E0CE0101960E945B
:104770004A9BBE016F5F7F4F84E093E10E94C7991F
:10478000182FCE0101960E94DE9A112309F468C009
:104790008091790490917A040E9447196093AD0446
:1047A0007093AE048093AF049093B004609367114C
:1047B000709368118093691190936A1180E090E57D
:1047C000A3ECB7E48093B5049093B604A093B70428
:1047D000B093B80480935F1190936011A09361111E
:1047E000B09362118091310D882381F06EE977E0FA
:1047F00084ED9FE00E94B59D6091AD047091AE0480
:104800008091AF049091B0040E94379D90E080E0C9
:104810000E947F904091AD045091AE046091AF042E
:104820007091B00422E0CE0145960E94E69A65E3BD
:1048300076E0CE0101960E944A9BBE016B5E7F4FDF
:10484000CE0101960E94F899BC018CEE92E10E9483
:104850008E9ACE0101960E94DE9ACE014596B5CB86
:1048600060E476E0CE0101960E944A9BBE016F5F34
:104870007F4F84E093E10E94C799182FCE010196E3
:104880000E94DE9A112309F488C080910E13909142
:104890000F130497F8F044E050E06AE073E1CE01B2
:1048A00001960E943858BE016F5F7F4F86EE92E1FD
:1048B0000E94A59ACE0101960E94DE9A86EE92E1B0
:1048C0000E94D0986093B9047093BA048093BB049B
:1048D0009093BC048091B9049091BA04A091BB0458
:1048E000B091BC0480935B1190935C11A0935D1117
:1048F000B0935E118091310D882389F065E877E0EF
:1049000084ED9FE00E94B59D6091B9047091BA0456
:104910008091BB049091BC0442E00E94559C809120
:10492000790490917A040E9447196093B1047093BE
:10493000B2048093B3049093B404609363117093B2
:10494000641180936511909366118091310D8823D5
:1049500081F06BE777E084ED9FE00E94B59D609168
:10496000B1047091B2048091B3049091B4040E9498
:10497000379D90E080E00E947F904091B10450917B
:10498000B2046091B3047091B40422E0CE01459664
:104990000E94E69A64E476E04CCF6CE476E0CE01C7
:1049A00001960E944A9BBE016F5F7F4F84E093E1B6
:1049B0000E94C799182FCE0101960E94DE9A1123FA
:1049C00011F40C94ED1B80910E1390910F1304972A
:1049D000F8F044E050E06AE073E1CE0101960E94F5
:1049E0003858BE016F5F7F4F86EE92E10E94A59A14
:1049F000CE0101960E94DE9A86EE92E10E94D09846
:104A00006093B5047093B6048093B7049093B80490
:104A10008091B5049091B604A091B704B091B80408
:104A200080935F1190936011A0936111B093621114
:104A30008091310D882389F062E677E084ED9FE074
:104A40000E94B59D6091B5047091B6048091B70441
:104A50009091B80442E00E94559C80917904909115
:104A60007A040E9447196093AD047093AE0480935A
:104A7000AF049093B00460936711709368118093B2
:104A8000691190936A118091310D882381F068E556
:104A900077E084ED9FE00E94B59D6091AD04709138
:104AA000AE048091AF049091B0040E94379D90E0D5
:104AB00080E00E947F904091AD045091AE046091DF
:104AC000AF047091B00461CFCF93DF93CDB7DEB761
:104AD0002C970FB6F894DEBF0FBECDBF8130910585
:104AE00009F06EC09093C6118093C51164EE75E015
:104AF000CE0101960E94389BCE0101960E94A359D7
:104B0000CE0101960E94DE9A60E576E0CE01019624
:104B10000E944A9B6BED73E1CE0101960E94F899C9
:104B2000BC01CE0107960E94419B48EC50E06FEF1C
:104B30007FEFCE0107960E94885ACE0107960E9409
:104B4000DE9ACE0101960E94DE9A8DEF9DE00E94D2
:104B5000F69040E052EC61E070E08DEF9DE00E9445
:104B6000F45790E080E00E947F906FE576E0CE0100
:104B700001960E944A9B67EE73E1CE0101960E9466
:104B8000F899BC01CE0107960E94419B40ED57E089
:104B90006FEF7FEFCE0107960E946857CE01079610
:104BA0000E94DE9ACE0101960E94DE9A81E02C9648
:104BB0000FB6F894DEBF0FBECDBFDF91CF91089541
:104BC0000097E1F51092C6111092C51166ED75E0DF
:104BD000CE0101960E94389BCE0101960E94A359F6
:104BE000CE0101960E94DE9A66E576E0CE0101963E
:104BF0000E944A9B6BED73E1CE0101960E94F899E9
:104C0000BC01CE0107960E94419B48EC50E06FEF3B
:104C10007FEFCE0107960E94885ACE0107960E9428
:104C2000DE9ACE0101960E94DE9A8DEF9DE00E94F1
:104C3000F69040E855E260E070E08FCF8230910559
:104C4000A9F49093C6118093C51165EC75E0CE016F
:104C500001960E94389BCE0101960E94A359CE0175
:104C600001960E94DE9A6AE576E0C0CF80E09FCF91
:104C70000F931F93CF93DF93CDB7DEB72C970FB66B
:104C8000F894DEBF0FBECDBF8C016BEF7BE08AE0F6
:104C900093E10E945E980830110509F0F8C06BEBB3
:104CA00075E0CE0101960E94389B44E650E06FEF1C
:104CB0007FEFCE0101960E94885ACE0101960E9494
:104CC000DE9A6FEA75E0CE0101960E94389B44E6B9
:104CD00050E070E060E0CE0101960E946857CE017E
:104CE00001960E94DE9A8DEF9DE00E94C38B4CE2FC
:104CF00051E061E070E0CE0107960E947FA98091AB
:104D0000310D8823D1F064E676E0CE0101960E9451
:104D10004A9BBE01695F7F4FCE0101960E94F899C0
:104D200067E676E00E94E299BC0184ED9FE00E9474
:104D3000A39DCE0101960E94DE9A65E17BE0CE0143
:104D400001960E944A9BBE016F5F7F4FCE0107967E
:104D50000E94C799182FCE0101960E94DE9A112356
:104D600009F478C069E676E08AE093E10E945E98F3
:104D700088E090E090932B0C80932A0C0E94B31B48
:104D8000182F62EA75E0CE0101960E94389B44E636
:104D900050E070E060E0CE0101960E946857CE01BD
:104DA00001960E94DE9A8DEF9DE00E94C38B48E53C
:104DB00052E061E070E0CE0101960E947FA9BE0141
:104DC0006F5F7F4FCE0107960E94A59ACE01019694
:104DD0000E94DE9A8091310D8823D1F064E676E05E
:104DE000CE0101960E944A9BBE01695F7F4FCE01B2
:104DF00001960E94F89967E676E00E94E299BC016C
:104E000084ED9FE00E94A39DCE0101960E94DE9A50
:104E100061EA7BE0CE0101960E944A9BBE016F5F72
:104E20007F4FCE0107960E94C799082FCE010196A9
:104E30000E94DE9A002371F06EE676E08AE093E14C
:104E40000E945E980E94B31B882321F065E975E0FB
:104E5000111102C06EE875E0CE0101960E94389BE8
:104E600044E650E070E060E0CE0101960E94685791
:104E7000CE0101960E94DE9A6BEF7BE08AE093E11F
:104E80000E945E98CE0107960E94DE9AA0C2093F5A
:104E90002FEF120709F00CC164E875E0CE0101960E
:104EA0000E94389B44E650E06FEF7FEFCE01019601
:104EB0000E94885ACE0101960E94DE9A66E775E04C
:104EC000CE0101960E94389B44E650E070E060E01D
:104ED000CE0101960E946857CE0101960E94DE9A8B
:104EE0008DEF9DE00E94C38B4CE251E064E070E0E6
:104EF000CE0101960E947FA98091310D8823D1F0C7
:104F000064E676E0CE0107960E944A9BBE016F5F81
:104F10007F4FCE0107960E94F89967E676E00E94DF
:104F2000E299BC0184ED9FE00E94A39DCE0107960B
:104F30000E94DE9A70E060E0CE0101960E94B69970
:104F4000082E000C990BC0970A9708F096C064E7EA
:104F500076E0CE0107960E944A9BBE016F5F7F4FAD
:104F6000CE0107960E94F899BC018AE093E10E9465
:104F70008E9ACE0107960E94DE9A89EF9FEF90935A
:104F80002B0C80932A0C0E94B31B182F68E675E047
:104F9000CE0107960E94389B44E650E070E060E046
:104FA000CE0107960E946857CE0107960E94DE9AAE
:104FB0008DEF9DE00E94C38B48E552E065E070E014
:104FC000CE0107960E947FA9BE01695F7F4FCE0187
:104FD00001960E94A59ACE0107960E94DE9A8091C2
:104FE000310D8823D1F064E676E0CE0107960E9469
:104FF0004A9BBE016F5F7F4FCE0107960E94F899D2
:1050000067E676E00E94E299BC0184ED9FE00E9491
:10501000A39DCE0107960E94DE9A70E060E0CE016B
:1050200001960E94B699082E000C990BC0970A971A
:1050300020F569E776E0CE0107960E944A9BBE0103
:105040006F5F7F4FCE0107960E94F899BC018AE0FE
:1050500093E10E948E9ACE0107960E94DE9A89EF14
:105060009FEF90932B0C80932A0C0E94B31B8823F4
:1050700021F06BE575E0111102C064E575E0CE0129
:1050800007960E94389B44E650E070E060E0CE0155
:1050900007960E946857CE0107960E94DE9A6BEF32
:1050A0007BE08AE093E10E945E98CE010196ECCE0F
:1050B0006AE475E0CE0101960E94389B44E650E018
:1050C0006FEF7FEFCE0101960E94885ACE010196C4
:1050D0000E94DE9A6BEF7BE08AE093E10E945E988B
:1050E000053F8FEF180709F044C06EE776E08AE0CD
:1050F00093E10E945E9860E475E0CE0101960E9403
:10510000389B44E650E06FEF7FEFCE0101960E949E
:105110006857CE0101960E94DE9A80910E139091FD
:105120000F13892B09F453C10E94B31B882309F480
:1051300059C168EC70E080E090E00E9439A560EC15
:1051400074E0CE0101960E94389B44EF51E06FEF6E
:105150007FEFCE0101960E946857CE0101960E9412
:10516000DE9A10932B0C00932A0CC8010E941A7728
:105170002EC1063F2FEF120749F46FEF75E08AE06A
:1051800093E10E945E9866E375E0B7CF013F8FEF31
:10519000180749F468E076E08AE093E10E945E989F
:1051A00067E275E0AACF023F2FEF120749F462E8E9
:1051B00076E08AE093E10E945E9867E175E09DCF1A
:1051C000033F8FEF180709F04DC06BE075E0CE018B
:1051D00001960E94389B44E650E06FEF7FEFCE01CE
:1051E00001960E94885ACE0101960E94DE9A6DEFC8
:1051F00074E0CE0101960E94389B44E650E06FEFC8
:105200007FEFCE0101960E946857CE0101960E9461
:10521000DE9A44EF51E062E070E0CE0101960E9418
:105220007FA9BE016F5F7F4F8AE093E10E94A59A3C
:10523000CE0101960E94DE9A6EE876E0CE010196DC
:105240000E944A9B6AE073E1CE0101960E94F899A0
:10525000BC018AE093E10E948E9ACE0101960E94E1
:10526000DE9A5BCF0230110509F094C061EF74E063
:10527000CE0101960E94389B44E650E06FEF7FEF2D
:10528000CE0101960E94885ACE0101960E94DE9AB4
:1052900061EE74E0CE0101960E94389B44E650E036
:1052A0006FEF7FEFCE0101960E946857CE01019605
:1052B0000E94DE9A44EF51E066E070E0CE01019674
:1052C0000E947FA9BE016F5F7F4F8AE093E10E9439
:1052D000A59ACE0101960E94DE9A80910E139091BC
:1052E0000F130597B0F070E060E08AE093E10E9450
:1052F000B699082E000C990BC0970A9750F48AE0D3
:1053000093E10E94DB98613523EC720781059105DA
:10531000CCF463ED74E0CE0101960E94389B48EE18
:1053200053E06FEF7FEFCE0101960E946857CE01E8
:1053300001960E94DE9A6BEF7BE08AE093E10E9487
:105340005E98EBCE0E94B1B720E030E048EC52E42A
:105350000E9429BAAB01BC0122E0CE0107960E944F
:10536000E69A6FEE75E0CE0101960E944A9BBE015F
:10537000695F7F4FCE0101960E94F899BC018AE0D7
:1053800093E10E948E9ACE0101960E94DE9ACE0190
:105390000796C1CE6AEC74E0CE0101960E94389B5C
:1053A00044E650E06FEF7FEFCE0101960E94685710
:1053B000CE0101960E94DE9A6BEF7BE08AE093E1DA
:1053C0000E945E980B3E8FEF180709F0A6CE2C9630
:1053D0000FB6F894DEBF0FBECDBFDF91CF911F9106
:1053E0000F91089568EC70E080E090E00E9439A58C
:1053F00064EB74E0CE0101960E94389B44EF51E0CB
:105400006FEF7FEFCE0101960E9468574ECEBF929C
:10541000CF92DF92EF92FF920F931F93CF93DF9380
:10542000CDB7DEB762970FB6F894DEBF0FBECDBF23
:105430008C016B0161E67AE0CE010D960E944A9BD9
:1054400062EB74E0C8010E94389B76012FEFE21AEC
:10545000F20AB701CE0101960E949598BE016F5FD6
:105460007F4FCE0107960E94419B6CE978E0CE0108
:1054700007960E94E299BC01C8010E94629ACE017F
:1054800007960E94DE9ACE0101960E94DE9A8AE07B
:10549000B82EBE9CC001BF9C900D1124FC01EA51A6
:1054A000FE4E7F018081082E000C990B0E9444BFA4
:1054B000892B09F4B2C0B701CE0101960E944A9B24
:1054C000BE016F5F7F4FCE0107960E94419B60E94E
:1054D00079E0CE0107960E94E299BC01C8010E94C2
:1054E000629ACE0107960E94DE9ACE0101960E9432
:1054F000DE9ABC9CC001BD9C900D11249C012A51D8
:105500003E4E7901F9016685062E000C770BCE011F
:1055100001960E949598BE016F5F7F4FCE0107965E
:105520000E94419B65E976E0CE0107960E94E299D0
:10553000BE01635F7F4F0E94F899BC01C8010E94C1
:10554000629ACE0107960E94DE9ACE0101960E94D1
:10555000DE9A6BEA74E0C8010E940B9AF701678536
:10556000062E000C770BCE0101960E949598BE0185
:105570006F5F7F4FCE0107960E94419BBE01635F24
:105580007F4FCE0107960E94F899BC01C8010E9486
:10559000629ACE0107960E94DE9ACE0101960E9481
:1055A000DE9A65EA74E0C8010E940B9AF7016089EF
:1055B0007189CE0101960E949598BE016F5F7F4F61
:1055C000CE0107960E94419BBE01635F7F4FCE01D3
:1055D00007960E94F899BC01C8010E94629ACE0108
:1055E00007960E94DE9ACE0101960E94DE9A60EA3A
:1055F00074E0C8010E940B9AF70162897389CE0199
:1056000001960E949598BE016F5F7F4FC8010E946E
:10561000629ACE0101960E94DE9ACE010D960E94FA
:10562000DE9AC80162960FB6F894DEBF0FBECDBFFA
:10563000DF91CF911F910F91FF90EF90DF90CF906E
:10564000BF9008952F923F924F925F926F927F92F8
:105650008F929F92AF92BF92CF92DF92EF92FF9282
:105660000F931F93CF93DF93CDB7DEB768970FB635
:10567000F894DEBF0FBECDBF2B013C010E94F80F96
:105680006D877E878F87988B8AE99EE00E94F690CF
:1056900062E370E080E090E00E9439A561E08091D3
:1056A0008E040E9441A060E080918C040E9441A081
:1056B00064E670E080E090E00E9439A56091880483
:1056C0007091890480918A0490918B040E946416E1
:1056D0000E9481167B018C010E94E7A14B015C01B5
:1056E00060E570E080E090E00E9439A567E976E02F
:1056F0008CEE92E10E945E9820E030E04AE754E4AC
:10570000C301B2010E9410B86D8B7E8B8F8B988F76
:10571000412C512C320160E070E0CB010E94B1B706
:105720002D893E894F89588D0E94AAB787FF87C16E
:105730000E94F80F2D853E854F855889621B730B9B
:10574000840B950B0E94AFB720E030E04AE754E4A9
:105750000E9429BAAB01BC0123E0CE0101960E9450
:10576000E69ABE016F5F7F4F86EE92E10E94A59A96
:10577000CE0101960E94DE9A0E948116D62EC72E77
:10578000382E292E0E94E7A1698B7A8B8B8B9C8BFC
:10579000DC01CB0188199909AA09BB094C015D01FB
:1057A00091ED891697E09906A104B104BCF020E0C0
:1057B00030E0A9016D2D7C2D832D922D0E9432BBEE
:1057C000181684F426EA3BE944EC5BE36D2D7C2D4E
:1057D000832D922D0E94AAB787FF10C0812C912C97
:1057E00054012EC026EA3BE944EC5BEB6D2D7C2D89
:1057F000832D922D0E9432BB181684F3C501B4018B
:1058000028EE33E040E050E00E94E7B8CA01B90159
:105810000E94B1B74B015C019701A8016D2D7C2D51
:10582000832D922D0E944AB920E030E04AE754E4EB
:105830000E9410B8A50194010E9429BA4B015C0195
:1058400066EE72E1CE0101960E94419B6EEB76E01E
:10585000CE0101960E94E299BC0186EE92E10E947F
:105860008E9ACE0101960E94DE9A23E04D2D5C2D8A
:10587000632D722DCE0101960E94E69ABE016F5FE4
:105880007F4FCE0107960E94419B65EB76E0CE01EB
:1058900007960E94E299BC0180EE92E10E948E9AE6
:1058A000CE0107960E94DE9ACE0101960E94DE9AF2
:1058B00022E0B501A401CE0107960E94E69A6EEBA4
:1058C0007AE0CE0101960E944A9B66EE72E1CE011B
:1058D00001960E94F89968EB76E00E94E29960EEEA
:1058E00072E10E94F8996FE37BE00E94E299BE01A9
:1058F000695F7F4F0E94F8996CEB76E00E94E29915
:10590000BC018CEE92E10E94629ACE0101960E9447
:10591000DE9ACE0107960E94DE9A20E030E0A901CF
:10592000C501B4010E9432BB87FD06C061E67AE082
:1059300080EE92E10E94589A22E0B501A401CE01C6
:1059400001960E94E69ABE016F5F7F4FCE010796D7
:105950000E94419B6CEB76E0CE0107960E94E29993
:10596000BC0180EE92E10E94629ACE0107960E94ED
:10597000DE9ACE0101960E94DE9A6CEE72E1CE01B3
:1059800001960E94419BCE0101960E94F256CE01E3
:1059900001960E94DE9AC301B20125E030E040E0AA
:1059A00050E00E94E7B8672B682B692B21F569E866
:1059B00074E0CE0101960E94389B45E050E070E013
:1059C00060E0CE0101960E94885ACE0101960E94A5
:1059D000DE9A60EE72E1CE0101960E94419B45E0A5
:1059E00050E06FEF7FEFCE0101960E946857CE0125
:1059F00001960E94DE9A6BEF7BE08CEE92E10E94B2
:105A00005E9862E370E080E090E00E9439A50E9419
:105A1000F80F2D853E854F855889621B730B840BCB
:105A2000950B3FEF431A530A630A730A89889A88D1
:105A3000AB88BC88ED2CFC2C032D122D6FCE60E0C2
:105A400080918E040E9441A068960FB6F894DEBF44
:105A50000FBECDBFDF91CF911F910F91FF90EF90BF
:105A6000DF90CF90BF90AF909F908F907F906F907E
:105A70005F904F903F902F9008958F929F92AF929A
:105A8000BF92CF92DF92EF92FF920F931F93CF932B
:105A9000DF93CDB7DEB7EA970FB6F894DEBF0FBE3F
:105AA000CDBFF82E6BEF7BE0CE01C5960E944A9BDE
:105AB0008E010B5E1F4F6F2DC8010E94B60D188717
:105AC0000F831D821E82198289E08A8381E08B8385
:105AD0008C831C8A1B8ACE0101960E94C612CE01BD
:105AE00001960E946911CE0101960E94A2A80E8122
:105AF00010E00330110509F488C16FE774E0CE01AE
:105B0000C5960E94699A6BEF7BE08CEE92E10E9451
:105B10005E98BE016B5C7F4FCE0183960E94419BD5
:105B20004AE050E070E060E0CE0183960E94885A1F
:105B3000CE0183960E94DE9A61E080E00E94F68D9D
:105B400062EE76E0CE01C5960E945E9883E6C82E8E
:105B50008CE0D82EF12CE12CE016F1060CF0F0C010
:105B60006E2DCE0101960E945A12F60121913191BB
:105B7000419151916F010E944BB94B015C01FFEFC4
:105B8000EF1AFF0A20E030E04CEF52EC0E94AAB777
:105B900087FF33C0B701CE0189960E94959864E3D0
:105BA00078E0CE0183960E944A9BBE01675D7F4FDD
:105BB000CE0183960E94F89960EC76E00E94E2990B
:105BC000BC018CEE92E10E94629ACE0183960E9403
:105BD000DE9ACE0189960E94DE9A0130110509F005
:105BE00055C081E0E816F10409F0B6CF6CEE72E121
:105BF000CE01C5960E948E9AAFCF22E0B501A401D6
:105C0000CE018F960E94E69AB701CE0189960E9436
:105C1000959864E378E0CE0183960E944A9BBE018A
:105C2000675D7F4FCE0183960E94F8996BE679E01D
:105C30000E94E299BE01615D7F4F0E94F899BC010C
:105C400080EE92E10E948E9ACE0183960E94DE9AA7
:105C5000CE0189960E94DE9ACE018F960E94DE9A2E
:105C600060EE72E1CE0183960E94419B61E67AE08C
:105C7000CE0183960E94E299BC018CEE92E10E94D3
:105C8000629ACE0183960E94DE9AA7CF0230110558
:105C900011F522E0B501A401CE0183960E94E69A97
:105CA000BE016D5D7F4FCE0189960E94419B61E6EA
:105CB0007AE0CE0189960E94E299BC01CE01C59698
:105CC0000E94629ACE0189960E94DE9ACE01839646
:105CD0000E94DE9A41CF0330110509F43DCF60EEFA
:105CE00072E1CE0183960E94419B44E150E06FEF48
:105CF0007FEFCE0183960E946857CE0183960E9463
:105D0000DE9A6BEA77E0CE0183960E944A9BCE0131
:105D100083960E944A57CE0183960E94DE9A809114
:105D20008504882309F418CF8091E504882309F4B9
:105D300013CF60ED77E080E090E00E9439A50CCFB2
:105D4000CE01C5960E94E6988CEE92E10E94E698FC
:105D50000115110579F56CE674E08CEE92E10E9474
:105D6000699A61E674E0CE0183960E94389B4AE00E
:105D700050E06FEF7FEFCE0183960E946857CE010F
:105D800083960E94DE9ACE01C5960E94DE9AEA961C
:105D90000FB6F894DEBF0FBECDBFDF91CF911F913C
:105DA0000F91FF90EF90DF90CF90BF90AF909F90BA
:105DB0008F900895043011050CF5BE016B5C7F4F88
:105DC000CE0183960E94419B4AE050E06FEF7FEF47
:105DD000CE0183960E946857CE0183960E94DE9A78
:105DE0006BEA77E0CE0183960E944A9BCE018396B0
:105DF0000E944A57CE0183960E94DE9A6CEC76E0B0
:105E00008CEE92E10E94589ABECF6FED76E0CE0103
:105E1000C5960E945E98BE016B5C7F4FCE01839653
:105E20000E94419B4AE050E070E060E0CE01839622
:105E30000E94885ACE0183960E94DE9A6BEF7BE027
:105E40008CEE92E10E945E986CEE72E1CE01C596F6
:105E50000E948E9A10E000E0602FCE0101960E9411
:105E60005A126B017C0122E0BC01A601CE0183968F
:105E70000115110509F077C00E94E69ABE016D5D1B
:105E80007F4F83EF93E10E94959DCE0183960E9400
:105E9000DE9A22E0B701A601CE0183960E94E69A1F
:105EA000BE016D5D7F4FCE0189960E94419B61E6E8
:105EB0007AE0CE0189960E94E299BC018CEE92E1D3
:105EC0000E94629ACE0189960E94DE9ACE01839644
:105ED0000E94DE9A0F5F1F4F0330110509F0BCCFFF
:105EE000CE01C5960E94E698BE016B5C7F4FCE0145
:105EF00083960E94419B4AE050E06FEF7FEFCE0116
:105F000083960E946857CE0183960E94DE9A6BEAC0
:105F100077E0CE0183960E944A9BCE0183960E9431
:105F20004A57CE0183960E94DE9A8CEE92E10E943F
:105F3000E69865EE76E0CE0183960E944A9B6CEE71
:105F400072E1CE0183960E94F8996CEC76E00E9493
:105F5000E299BC018CEE92E10E948E9ACE0183966A
:105F60000E94DE9A10CF0E94E69ABE016D5D7F4FBF
:105F7000CE0189960E94419B61E67AE0CE01899626
:105F80000E94E299BC01CE01C5960E94629ACE01A0
:105F900089960E94DE9A79CF8F929F92AF92BF929C
:105FA000CF92DF92EF92FF920F931F93CF93DF93E5
:105FB000CDB7DEB768970FB6F894DEBF0FBECDBF82
:105FC0006C018091C5119091C6110197C9F06BEFDA
:105FD0007BE0C6010E944A9BC60168960FB6F89402
:105FE000DEBF0FBECDBFDF91CF911F910F91FF900C
:105FF000EF90DF90CF90BF90AF909F908F900895DB
:106000006FEE76E0CE010D960E944A9BBE01635F63
:106010007F4F8DEF9DE00E94959D6CE271E080E0E6
:1060200090E00E9439A5CE0143960E94BC7064E6C0
:1060300070E080E090E00E9439A510E000E085E08B
:10604000A82EB12C9AE0892E912C6AEF76E0CE0131
:1060500001960E944A9BBE016F5F7F4FCE0143961F
:106060000E949B997C01CE0101960E94DE9AA701B5
:106070004F5F5F4FBE016D5E7F4FCE0101960E9464
:106080003858BE016F5F7F4FCE010D960E94A59AD2
:10609000CE0101960E94DE9A89899A89892B09F19D
:1060A00070E060E0CE010D960E94B699082E000CBB
:1060B000990BC0970A97A8F46CEF76E0CE01019691
:1060C0000E944A9BBE016F5F7F4FCE010D960E94DA
:1060D000C799E82ECE0101960E94DE9AFF24F39420
:1060E000E110F12C60E974E0CE0101960E94389B2A
:1060F00044E150E06FEF7FEFCE0101960E94CF594F
:10610000CE0101960E94DE9A0F5F1F4F62E370E09E
:1061100080E090E00E9439A5C801B5010E94C1BC91
:106120000197C1F4CE0101960E946F6F8D819E810F
:10613000892B09F46AC0BE016F5F7F4F8AE093E14B
:106140000E948E9A0E947C4AFF24F394CE0101960D
:106150000E94DE9ACE0101960E94BC70BE016F5F64
:106160007F4FCE0143960E94A59ACE0101960E94D0
:10617000DE9A62E370E080E090E00E9439A5043688
:10618000110519F0FF2009F460CF8091310D8823AB
:10619000F1F060EC75E0CE0101960E944A9BBE01D1
:1061A000635F7F4FCE0101960E94F899BC01CE013A
:1061B00007960E94419BCE0107960E94F256CE019F
:1061C00007960E94DE9ACE0101960E94DE9A898986
:1061D0009A89892B61F070E060E0CE010D960E94F3
:1061E000B699082E000C990BC0970A9738F164E015
:1061F00077E0C6010E944A9BCE0143960E94DE9A38
:10620000CE010D960E94DE9AE7CE043111050CF402
:106210009DCFC801B4010E94C1BC892B09F096CF63
:10622000BE01635F7F4F8DEF9DE00E94959D68ECFE
:1062300070E080E090E00E9439A588CF6CEF76E0B6
:10624000CE0101960E944A9BBE016F5F7F4FCE0137
:106250000D960E94C799182FCE0101960E94DE9AD2
:106260001111C5CFBE01635F7F4FC6010E942F9BF6
:10627000C3CF2F923F924F925F926F927F928F92F5
:106280009F92AF92BF92CF92DF92EF92FF920F93C5
:106290001F93CF93DF93CDB7DEB76D970FB6F8940A
:1062A000DEBF0FBECDBF61E089E10E9441A061E089
:1062B00089E10E94529F0E94B09760E177E084EDEF
:1062C0009FE00E94089CF12CE12C17E2812F0E9494
:1062D000DB8D0E94FCA2811195C16CE177E084ED19
:1062E0009FE00E94939D40E150E0612F84ED9FE08C
:1062F0000E94F19B1093F71368E377E084ED9FE031
:106300000E94939D40E150E0612F84ED9FE00E9448
:10631000F19B2FEFE21AF20A1F5F1034B9F66DE617
:1063200077E0EF2811F063E877E084ED9FE00E94CA
:10633000089C0E94E4AB80E40E94E58D0AEC14E026
:10634000D8016D918D0183EF93E10E949E13B4E01B
:10635000023D1B07A9F70E9426570E94D5168EE41E
:1063600092E00E94D1B880935C0D8FE492E00E948D
:10637000D1B880935D0D80915C0D90915D0D1816E4
:10638000190664F41092C904019741F410925D0D4E
:1063900010925C0D8EE492E00E942A9064EC7BE007
:1063A000CE0101960E94389B4AE050E06FEF7FEFEC
:1063B000CE0101960E94885ACE0101960E94DE9A73
:1063C00040E052EC61E070E084ED9FE00E94F45701
:1063D0008091C904882331F068EE73E080E090E09A
:1063E0000E9439A584ED9FE00E94FE8A8B8B66EEA9
:1063F000E62E61E1F62E0CE211E0C8010E94D1B850
:10640000F70181937F010F5F1F4F0632F2E01F07F4
:10641000A1F78091E711181624F42B892D3609F085
:1064200021C16BEF7BE0CE010D960E944A9B10923A
:10643000E61188E18093E71184E08093E8111092DF
:10644000ED111092EE116AE17AE0CE010D960E94F4
:106450005E9880EF91E1009739F044E050E0BC0194
:10646000CE010D960E94A99081E08093F41183E003
:106470008093F51182E090E09093F7118093F611EC
:1064800085E090E09093F9118093F81167E17AE04C
:10649000CE010D960E945E988AEF91E1009739F047
:1064A00044E050E0BC01CE010D960E94A99082E02C
:1064B0008093FE1183E08093FF1182E090E090933F
:1064C00001128093001285E090E090930312809374
:1064D000021264E17AE0CE010D960E945E9884E09B
:1064E00092E1009739F044E050E0BC01CE010D96F6
:1064F0000E94A99083E0809308128093091282E0A1
:1065000090E090930B1280930A1285E090E09093B4
:106510000D1280930C126AE877E0CE010D960E946E
:106520005E988EE092E1009739F044E050E0BC01C3
:10653000CE010D960E94A99085EF8093121283E000
:106540008093131282E090E09093151280931412BE
:1065500085E090E090931712809316128CE291E000
:106560000E94CC908091310D882311F1CE010196CB
:106570000E946F1ABE016F5F7F4F84ED9FE00E9403
:10658000A39DCE0101960E94DE9A61E07AE084ED3F
:106590009FE00E94B59D2AE04AE050E060E070E094
:1065A00084ED9FE00E94A19B84ED9FE00E94ED9B03
:1065B00067EC79E0CE0107960E94389BBE01695FC7
:1065C0007F4F84ED9FE00E94A39D10E000E080914A
:1065D000E811082E000C990B0817190724F5B801CB
:1065E000CE0101960E94072ABE016F5F7F4F84EDA6
:1065F0009FE00E94A39DCE0101960E94DE9A0F5F4C
:106600001F4FE5CF843009F087CE62E577E084ED57
:106610009FE00E94939D40E150E0612F84ED9FE058
:106620000E94F19B79CECE0107960E94DE9A80915E
:10663000310D882399F061EE79E084ED9FE00E94AE
:10664000B59D2AE04AEF50E060E070E084ED9FE005
:106650000E94A19B84ED9FE00E94ED9BCE010D96D0
:106660000E94DE9A8091EF1181118091E611809352
:10667000E1110E94F80F6093DD117093DE11809399
:10668000DF119093E0113B8910E0323709F499C58E
:106690005FE4252E51E1352E710110E000E0C801C4
:1066A0000E94D1B8D7018D937D010F5F1F4F08382D
:1066B0001105A9F780914F1190915011A09151119E
:1066C000B091521185369105A105B1050CF49BC11D
:1066D0008093C5049093C604A093C704B093C804E4
:1066E0008091531190915411A0915511B091561170
:1066F0008093C1049093C204A093C304B093C404D4
:106700008091571190915811A0915911B0915A113F
:106710008093BD049093BE04A093BF04B093C004C3
:106720006BE671E1CE0101960E944A9BBE016F5F4C
:106730007F4F81EE93E10E94A59ACE0101960E94BF
:10674000DE9A69EC71E1CE0101960E944A9BBE017E
:106750006F5F7F4F8BED93E10E94A59ACE0101966A
:106760000E94DE9A23E030E050E040E061EE73E109
:10677000CE0107960E945B9B23E030E050E040E0B2
:106780006BED73E1CE0101960E945B9B2D813E81F2
:106790008B859C852817390709F589819A816F8136
:1067A0007885009759F06115710509F0F1C0232B28
:1067B00009F4F1C0DC018C9190E00DC06115710508
:1067C00009F4E9C0232B09F4E6C0FB01808190E0C5
:1067D00091958195910911E0892B09F010E0CE0186
:1067E00001960E94DE9ACE0107960E94DE9A111150
:1067F00006C061EE73E18BED93E10E948E9A809169
:106800005B1190915C11A0915D11B0915E1180932C
:10681000B9049093BA04A093BB04B093BC048091D4
:106820005F1190916011A0916111B09162118093FC
:10683000B5049093B604A093B704B093B8048091C4
:10684000631190916411A0916511B09166118093CC
:10685000B1049093B204A093B304B093B4048091B4
:10686000671190916811A0916911B0916A1180939C
:10687000AD049093AE04A093AF04B093B004E09144
:10688000C711F091C811FD8FEC8FF093D304E09302
:10689000D2048091831190918411A0918511B091BF
:1068A00086118C8B9D8BAE8BBF8B8093D80490937D
:1068B000D904A093DA04B093DB04809199119091EC
:1068C0009A11A0919B11B0919C11888F998FAA8FDA
:1068D000BB8F8093D4049093D504A093D604B09337
:1068E000D70440907311509074116090751170909E
:1068F00076114092A9045092AA046092AB0470925F
:10690000AC048090771190907811A0907911B0909C
:106910007A118092A5049092A604A092A704B09246
:10692000A8040091D5111091D611B801012E000CC8
:10693000880B990B0E94B1B76B017C01AC019B01E4
:106940000E9497BC811104C010932F0C00932E0C51
:10695000209193043091940490E080E02817390747
:10696000E4F0D101D8964D915C91D99757FF0BC0B7
:10697000FC01EE0FFF1FED56FB4F40815181D99670
:106980005C934E93D8970196B2E02B0E311CE6CF64
:106990000E946EBF20CF11E022CFA3019201C3015C
:1069A000B2010E9497BC811109C0A5019401C501E3
:1069B000B4010E9497BC882309F472C30E94E20DBF
:1069C0003DE9A32E31E1B32E03E61CE0D501CD90C5
:1069D000DD90ED90FD905D01A7019601C701B60124
:1069E0000E9497BC811105C0F801C082D182E28269
:1069F000F3820C5F1F4FFCE00B381F0739F781E073
:106A000090E00E94350E1B891257113009F4D9C34A
:106A10002B892E3609F4D4C380914F1190915011D7
:106A2000A0915111B091521185369105A105B10582
:106A30000CF4C7C38091C5119091C6118D7F892B2D
:106A400041F440E855E260E070E08DEF9DE00E9487
:106A5000F4578091C5119091C611019741F440E01F
:106A600052EC61E070E08DEF9DE00E94F45764E627
:106A700070E080E090E00E9439A58091C51190916E
:106A8000C611892B09F0B8C02B892E3671F0809180
:106A90004F1190915011A0915111B0915211853622
:106AA0009105A105B1050CF0A7C06BEF7BE0CE010D
:106AB00007960E944A9B62E977E0CE0101960E9408
:106AC0004A9B6BED73E1CE0101960E94F899BC01DF
:106AD000CE0107960E948E9ACE0101960E94DE9A00
:106AE000BE01695F7F4F8DEF9DE00E94959D68EB31
:106AF0007BE080E090E00E9439A5BE01695F7F4F96
:106B0000CE0101960E94419BCE0101960E94A3599D
:106B1000CE0101960E94DE9A6CE271E080E090E086
:106B20000E9439A54091DF135091E0134250510962
:106B30006BED73E1CE0101960E943858BE016F5F84
:106B40007F4FCE0107960E94A59ACE0101960E9422
:106B5000DE9ABE01695F7F4FCE0101960E94419B84
:106B6000BE01695F7F4FCE0101960E94F899BC017A
:106B7000CE0107960E948E9ACE0101960E94DE9A5F
:106B80006AE977E0CE0101960E944A9BBE01695FE7
:106B90007F4FCE0101960E94F899BC01CE01079665
:106BA0000E948E9ACE0101960E94DE9ABE01695F14
:106BB0007F4F8DEF9DE00E94959D68EB7BE080E02C
:106BC00090E00E9439A5BE01695F7F4FCE0101961A
:106BD0000E94419BCE0101960E94A359CE010196CD
:106BE0000E94DE9A6CE271E080E090E00E9439A59C
:106BF000CE0107960E94DE9A64E670E080E090E0A5
:106C00000E9439A5F89482E08093B0008093B1008F
:106C100094E69093B3001092B20080937000789441
:106C200080937D101092801080917E1060E00E9411
:106C300041A06EE97BE0CE0101960E94389B4AE0BC
:106C400050E06FEF7FEFCE0101960E94885ACE018F
:106C500001960E94DE9A6BEF7BE08CEE92E10E943F
:106C60005E988091C5119091C611892B31F466E52B
:106C700076E08CEE92E10E945E988091C511909131
:106C8000C611019731F460E576E08CEE92E10E9446
:106C90005E988091C5119091C611029731F46AE512
:106CA00076E08CEE92E10E945E988091F0129091D5
:106CB000F112892BC1F06BED73E18CEE92E10E9431
:106CC000629A6CEE72E1CE0101960E94419B4AE00D
:106CD00050E06FEF7FEFCE0101960E946857CE0122
:106CE00001960E94DE9A8091C5119091C61101977C
:106CF00009F05CC0CE0107960E94CC2F8B859C8545
:106D0000009709F449C0EF81F8852081222309F416
:106D100043C0079708F440C06BE87BE08CEE92E13B
:106D20000E94699ABE01695F7F4F8CEE92E10E94DA
:106D3000629A6CEE72E1CE0101960E94419BCE01F7
:106D400001960E94F256CE0101960E94DE9A62E8F8
:106D50007BE0CE0101960E94389B48EC50E06FEF3B
:106D60007FEFCE0101960E94CF59CE0101960E947D
:106D7000DE9ABE01695F7F4FCE0101960E94419B62
:106D800048EC50E06FEF7FEFCE0101960E9468570C
:106D9000CE0101960E94DE9A68EE73E080E090E0FA
:106DA0000E9439A5CE0107960E94DE9A66E67BE036
:106DB0008CEE92E10E94699A60EC75E0CE0101963A
:106DC0000E944A9B6BED73E1CE0101960E94F899F7
:106DD0006CEE72E10E94F899BC018CEE92E10E9487
:106DE0008E9ACE0101960E94DE9A6CEE72E1CE017F
:106DF00001960E94419BCE0101960E94F256CE015F
:106E000001960E94DE9A6BEF7BE08CEE92E10E948D
:106E10005E9864E670E080E090E00E9439A50E94F0
:106E2000B09764E670E080E090E00E9439A583E2CC
:106E30000E94DB8D81E090E00E94D68D0E94FCA232
:106E400083E090E090932D0C80932C0C8CE40E94B6
:106E5000809F6B017C0162E370E080E090E00E9423
:106E600039A5A7019601C701B6010E9497BC8823E6
:106E7000B9F086E60E94809F6B017C0162E370E0BE
:106E800080E090E00E9439A5A7019601C701B601F4
:106E90000E9497BC882321F010922D0C10922C0C8C
:106EA00080912C0C90912D0C039709F08CC261E518
:106EB0007BE0CE0101960E94389BCE0101960E9494
:106EC000A359CE0101960E94DE9A83E080931013AD
:106ED0000E94B09780ED0E94EAA3853509F096C222
:106EE0008AEA0E9407A490931213809311138CEAEC
:106EF0000E9407A490931413809313138EEA0E94A8
:106F000007A4909316138093151380EB0E9407A497
:106F1000909322138093211382EB0E9407A49093F5
:106F200024138093231384EB0E9407A490932613C9
:106F30008093251386EB0E9407A4909318138093E7
:106F4000171388EB0E9407A490931A1380931913C8
:106F50008AEB0E9407A490931C1380931B138CEB65
:106F60000E9407A490931E1380931D138EEB0E9422
:106F700007A49093201380931F1368E17BE08CEEAD
:106F800092E10E94699A0E94D9A50E94B1B70E941D
:106F9000D5BA0E94B1B720E030E048EC52E40E943C
:106FA00029BAAB01BC0122E0CE0101960E94E69A0B
:106FB000BE016F5F7F4FCE0107960E94419B63EF3A
:106FC00075E0CE0107960E94E299BC018CEE92E139
:106FD0000E94629ACE0107960E94DE9ACE01019627
:106FE0000E94DE9A6CEE72E1CE0101960E94419BF6
:106FF000CE0101960E94A359CE0101960E94DE9A0D
:1070000062E07BE08CEE92E10E94699A6091C50497
:107010007091C6048091C7049091C8040E94B1B7D2
:1070200020E030E048EC52E40E9429BAAB01BC01F8
:1070300022E0CE0101960E94E69ABE016F5F7F4F6B
:10704000CE0107960E94419B63EF75E0CE01079643
:107050000E94E299BC018CEE92E10E94629ACE01FC
:1070600007960E94DE9ACE0101960E94DE9A6CEE8F
:1070700072E1CE0101960E94419BCE0101960E94D1
:10708000A359CE0101960E94DE9A3B89313609F060
:107090004EC281E00E94CD6881E00E94876EC6C129
:1070A00000917B11602F002E000C770B880B990B41
:1070B0000E94B1B79B01AC010E9497BC81117ECCAC
:1070C00060907C1170907D11B301072C000C880B2F
:1070D000990B0E94B1B79B01AC010E9497BC811132
:1070E0006DCC10917E11612F012E000C770B880B57
:1070F000990B0E94B1B79B01AC010E9497BC811112
:107100005DCC80907F1190908011A0908111B09003
:107110008211A5019401C501B4010E9497BC81119F
:107120004DCC2C893D894E895F89CA01B9010E94E5
:1071300097BC811143CC288D398D4A8D5B8DCA0156
:10714000B9010E9497BC811139CC6091C511709131
:10715000C611072E000C880B990B0E94B1B79B013A
:10716000AC010E9497BC811129CCEC8DFD8DBF0133
:10717000FF0F880B990B0E94B1B79B01AC010E94D5
:1071800097BC81111BCCA7019601C701B6010E94D3
:1071900097BC811113CC04300CF010CC15300CF0DE
:1071A0000DCCFBEF6F1671040CF008CC20E030E042
:1071B000A901C501B4010E94AAB787FDFFCB00CC8D
:1071C0001CEF8091C5049091C604A091C704B091B2
:1071D000C80480934F1190935011A0935111B09314
:1071E00052118091C1049091C204A091C304B09146
:1071F000C4048093531190935411A0935511B093EC
:1072000056118091BD049091BE04A091BF04B0912D
:10721000C0048093571190935811A0935911B093C3
:107220005A113B89333751F160E081EE93E10E94BE
:10723000359A60E08BED93E10E94359A4091E51319
:107240005091E6134115510549F08BE691E1009705
:1072500029F0BC0181EE93E10E94A9904091DF13D7
:107260005091E0134115510549F089EC91E10097E7
:1072700029F0BC018BED93E10E94A9908091B904A3
:107280009091BA04A091BB04B091BC0480935B11AF
:1072900090935C11A0935D11B0935E118091B50441
:1072A0009091B604A091B704B091B80480935F1197
:1072B00090936011A0936111B09362118091B10419
:1072C0009091B204A091B304B091B404809363117F
:1072D00090936411A0936511B09366118091AD04F1
:1072E0009091AE04A091AF04B091B0048093671167
:1072F00090936811A0936911B0936A1190E080E0B7
:107300000E947F90E3E6FCE0ADE9B1E18BE89CE010
:1073100041915191619171914D935D936D937D93E5
:107320008E179F07A9F76EEA7BE0CE0101960E94B7
:10733000389BCE0101960E94A359CE0101960E946E
:10734000DE9A93E9C92E94E0D92E27E8A22E21E1F6
:10735000B22EF12CE12C80919304909194048E151F
:107360009F054CF1D6018D919D916D01F5018193A1
:1073700091935F018091310D8823C9F060EC75E035
:1073800084ED9FE00E94939D4AE050E0B70184EDB8
:107390009FE00E94469D6DE877E084ED9FE00E94AB
:1073A000939DF6013297808191810E94809DFFEF2D
:1073B000EF1AFF0AD0CF123008F03CCB90E080E00B
:1073C0000E947F9037CB86E00E9414A5BC0190E01C
:1073D00080E00E94AFB72AE037ED43EA5CE30E9409
:1073E00010B823E333E948E853E40E944AB920E0A7
:1073F00030E048E453E40E94AAB787FF66CD82E0FC
:1074000090E090939204809391045FCD6BE27BE0D7
:10741000CE0101960E94389BCE0101960E94F25641
:10742000CE0101960E94DE9A1092900464E670E00C
:1074300080E090E00E9439A580912C0C90912D0C59
:10744000892BA1F461E080918E040E9441A060E04C
:1074500080918C040E9441A06091880470918904FD
:1074600080918A0490918B040E94641660E0809160
:107470008E040E9441A08091C904882331F068EEF7
:1074800073E080E090E00E9439A567E17AE088EF40
:1074900092E10E945E9882E090E090932B0C8093A2
:1074A0002A0C8091C904882309F494C168EC7AE01D
:1074B000CE0101960E94389B4CE251E06FEF7FEFC6
:1074C000CE0101960E946857CE0101960E94DE9A75
:1074D00060918604709187048091D2049091D304C6
:1074E0000E94B55484E1C82ED12CE12CF12C10E07F
:1074F00000E00F5F1F4FC701B6010E9439A56091E0
:107500008604709187048091D2049091D3040E94E4
:10751000B554033011052CF00A301105DCF4892B29
:10752000E1F044E1C40ED11CE11CF11CE2CF84ED7A
:107530009FE00E94FE8A182F64E670E080E090E0F1
:107540000E9439A5113609F4A4CD80E00E94CD68CF
:1075500080E0A3CD892B09F0EDC18091D2049091F8
:10756000D3048B30910509F095C180914A13909115
:107570004B13A0914C13B0914D138093260C909314
:10758000270CA093280CB093290C8091461390915E
:107590004713A0914813B09149138093220C909304
:1075A000230CA093240CB093250C4091260C5091F1
:1075B000270C6091280C7091290C21E0CE010196D6
:1075C0000E94E69A62EE76E0CE0107960E944A9B00
:1075D000BE016F5F7F4FCE0107960E94F899BC01F4
:1075E0008CEE92E10E948E9ACE0107960E94DE9A5E
:1075F000CE0101960E94DE9A4091220C5091230CFC
:107600006091240C7091250C21E0CE0101960E941E
:10761000E69A61EA77E0CE0107960E944A9BBE0196
:107620006F5F7F4FCE0107960E94F899BC018CEEE8
:1076300092E10E94629ACE0107960E94DE9ACE01E4
:1076400001960E94DE9A65E67BE08CEE92E10E9454
:10765000589A6BEF7BE0CE0101960E944A9B44E171
:1076600050E070E060E0CE0101960E94885ACE01A1
:1076700001960E94DE9AC090260CD090270CE090D4
:10768000280CF090290C20E030E0A901C701B601D8
:107690000E9432BB20E030E040E05FE387FD1AC18A
:1076A000C701B6010E944BB90E94D5BAAB01BC011B
:1076B000CE0101960E946898BE016F5F7F4F86EEF3
:1076C00092E10E94A59ACE0101960E94DE9A60E0A6
:1076D00087E00E94F68D66EE72E183EF93E10E94EF
:1076E000959D6FED83EF93E10E941A9C67EA77E026
:1076F00083EF93E10E94939D6091220C7091230C83
:107700008091240C9091250C0E94D5BA4AE050E05B
:1077100083EF93E10E94469D65E67BE083EF93E172
:107720000E94939D64E670E080E090E00E9439A59D
:10773000C090260CD090270CE090280CF090290CDB
:1077400020E030E040EF51E4C701B6010E9432BBB7
:1077500069EB7AE087FF28C020E030E040ED51E49B
:10776000C701B6010E9432BB87FDB9C069EA7AE061
:10777000CE0101960E94389B4AE050E06FEF7FEF08
:10778000CE0101960E946857CE0101960E94DE9AB2
:107790008091C904882331F06CED75E080E090E0C1
:1077A0000E9439A569E97AE0CE0101960E94389BD2
:1077B0004AE050E06FEF7FEFCE0101960E946857DC
:1077C000CE0101960E94DE9A62E370E080E090E0D4
:1077D0000E9439A56AEE7AE08CEE92E10E94699AE5
:1077E00060EC75E0CE0101960E944A9B6BED73E15F
:1077F000CE0101960E94F8996CEE72E10E94F89910
:10780000BC018CEE92E10E948E9ACE0101960E94FC
:10781000DE9A6CEE72E1CE0101960E94419BCE0190
:1078200001960E94F256CE0101960E94DE9A66ED04
:107830007AE08CEE92E10E94699A6CEE72E1CE01E0
:1078400001960E94419BCE0101960E94F256CE0104
:1078500001960E94DE9A6BEF7BE08CEE92E10E9433
:107860005E986D960FB6F894DEBF0FBECDBFDF9168
:10787000CF911F910F91FF90EF90DF90CF90BF902D
:10788000AF909F908F907F906F905F904F903F90C0
:107890002F9008958631910509F467CE0C9709F071
:1078A00084CE8091190C90911A0CA0911B0CB09170
:1078B0001C0C8093260C9093270CA093280CB0935B
:1078C000290C8091150C9091160CA091170CB09179
:1078D000180C63CEC701B6010E944AB9E5CE20E07C
:1078E00030E040EB51E4C701B6010E9432BB6BE8C7
:1078F0007AE087FF59CF6CE77AE0CE0101960E94CB
:10790000389B4AE050E06FEF7FEFCE0101960E9476
:107910006857CE0101960E94DE9A8091C90488239F
:1079200031F06CED75E080E090E00E9439A56EE6E4
:107930007AE03ACF0E9426576EE170E080E090E056
:107940000E9439A50E9484A56B017C0164E670E069
:1079500080E090E00E9439A562EE76E08CEE92E144
:107960000E945E9821E0B701A601CE0101960E9417
:10797000E69ABE016F5F7F4F8CEE92E10E94629AA1
:10798000CE0101960E94DE9A6CEE72E1CE01019664
:107990000E94419B4AE050E070E060E0CE01019619
:1079A0000E94885ACE0101960E94DE9A8091850439
:1079B000882379F08091E504882359F06FED83EFF7
:1079C00093E10E941A9C6BEA77E083EF93E10E94B7
:1079D000939D6AEA77E08CEE92E10E94589AC092F9
:1079E000260CD092270CE092280CF092290C20E073
:1079F00030E040EF51E4C701B6010E9432BB6EE5B2
:107A00007AE087FF28C020E030E040ED51E4C70174
:107A1000B6010E9432BB87FD3EC06EE47AE0CE0123
:107A200001960E94389B4AE050E06FEF7FEFCE0155
:107A300001960E946857CE0101960E94DE9A8091BD
:107A4000C904882331F06CED75E080E090E00E947D
:107A500039A56EE37AE0CE0101960E94389B4AE098
:107A600050E06FEF7FEFCE0101960E946857CE0184
:107A700001960E94DE9A6CE271E080E090E00E9444
:107A800039A58091C904882309F4A4CE68EE73E077
:107A900080E090E09DCE20E030E040EB51E4C70173
:107AA000B6010E9432BB60E37AE087FFD4CF61E287
:107AB0007AE0CE0101960E94389B4AE050E06FEFD9
:107AC0007FEFCE0101960E946857CE0101960E9479
:107AD000DE9A8091C904882331F06CED75E080E076
:107AE00090E00E9439A563E17AE0B5CF2F923F92F2
:107AF0004F925F926F927F928F929F92AF92BF92BE
:107B0000CF92DF92EF92FF920F931F93CF93DF9369
:107B1000CDB7DEB7E6970FB6F894DEBF0FBECDBF88
:107B20006AE073E184E093E10E948E9A0E94479894
:107B30006DEA77E0CE0101960E944A9BBE016F5F1D
:107B40007F4F84E093E10E94C799182FCE010196E0
:107B50000E94DE9A112309F48FC026E030E045E050
:107B600050E06AE073E1CE0101960E945B9BBE018A
:107B70006F5F7F4F86EE92E10E94A59ACE0101963B
:107B80000E94DE9A86EE92E10E94DB986B016BE622
:107B900079E0CE0101960E944A9BBE016F5F7F4F44
:107BA0008AE093E10E949199AC014F5F5F4F6AE0D8
:107BB00073E1CE010B960E943858BE01655F7F4F7E
:107BC00086EE92E10E94A59ACE010B960E94DE9A63
:107BD000CE0101960E94DE9A86EE92E10E94DB9829
:107BE0009B01E3E9F4E041E050E0A0919304B091FF
:107BF0009404A417B5075CF0A281B381A217B30760
:107C000011F4138212824F5F5F4F3296EECFF6016E
:107C1000EE0FFF1FED56FB4F7183608382E090E013
:107C20000E94350E6AE073E1CE0101960E94419BED
:107C3000CE0101960E94A359CE0101960E94DE9AC0
:107C400090E080E00E947F901092EA041091EA0494
:107C5000112311F40C947A4A6AE073E1CE01019683
:107C60000E94419BCE0101960E94A359CE0101962C
:107C70000E94DE9A0C94324863EB77E0CE010196C5
:107C80000E944A9BBE016F5F7F4F84E093E10E9498
:107C9000C799182FCE0101960E94DE9A1123F1F0A8
:107CA000E3E9F4E081E090E02091930430919404C2
:107CB0002817390774F0863091052CF4938382835A
:107CC00001963296F1CF9C012E5F3F4F3383228382
:107CD000F7CF82E090E00E94350EB2CF69EB77E0FB
:107CE000CE0101960E944A9BBE016F5F7F4F84E0E8
:107CF00093E10E94C799182FCE0101960E94DE9A47
:107D00001123D1F080915C0D90915D0D892B81F450
:107D100081E090E090935D0D80935C0D8EE492E0A5
:107D20000E942A9068EC70E080E090E00E9439A503
:107D3000F0E0E0E019958ACF60EC77E0CE010196A3
:107D40000E944A9BBE016F5F7F4F84E093E10E94D7
:107D5000C799182FCE0101960E94DE9A112399F13E
:107D600068EC77E0CE0101960E944A9B67EE73E1D2
:107D7000CE0101960E94F899BC018CEE92E10E941E
:107D80008E9ACE0101960E94DE9A60EC75E0CE01DB
:107D900001960E944A9B6CEE72E1CE0101960E9410
:107DA000F899BC01CE010B960E94419BCE010B9627
:107DB0000E94F256CE010B960E94DE9ACE010196E9
:107DC0000E94DE9A41CF62ED77E0CE0101960E94DB
:107DD0004A9BBE016F5F7F4F84E093E10E94C79989
:107DE000182FCE0101960E94DE9A112369F062E4F9
:107DF00079E08CEE92E10E94699A6BED73E18CEE72
:107E000092E10E94629AC1CF69ED77E0CE010196BE
:107E10000E944A9BBE016F5F7F4F84E093E10E9406
:107E2000C799182FCE0101960E94DE9A112309F1FD
:107E30006FE179E08CEE92E10E94699A6CEE72E15A
:107E4000CE0101960E94419BCE0101960E94F256FE
:107E5000CE0101960E94DE9A0E94E20D1092EA0481
:107E60006FED77E08AE093E10E945E980E947C4A81
:107E7000EDCE63EE77E0CE0101960E944A9BBE01F3
:107E80006F5F7F4F84E093E10E94C799182FCE0166
:107E900001960E94DE9A112309F495C06BE679E001
:107EA000CE0101960E944A9BBE016F5F7F4F8AE020
:107EB00093E10E949199AC014F5F5F4F6AE073E1DB
:107EC000CE010B960E943858BE01655F7F4F86EE4B
:107ED00092E10E94A59ACE010B960E94DE9ACE01F5
:107EE00001960E94DE9A86EE92E10E94DB988B0159
:107EF00062E179E08CEE92E10E94699A8091E6114C
:107F0000882331F066E079E08CEE92E10E94699A74
:107F10000115110559F46CEE72E1CE0101960E9433
:107F2000419BCE0101960E94F25604C7CE010196F4
:107F30000E946F1ACE0101960E94F256CE01019660
:107F40000E94DE9A023011050CF47ECE67EC79E0D7
:107F5000CE010B960E94389BBE01655F7F4FCE011C
:107F600001960E94419BCE0101960E94F256CE01DD
:107F700001960E94DE9AF12CE12C8091E811082EE6
:107F8000000C990BE816F9068CF4B701CE010196A6
:107F90000E94072ACE0101960E94F256CE01019658
:107FA0000E94DE9AFFEFEF1AFF0AE7CFCE010B9691
:107FB0000E94DE9A0230110509F446CE8CE291E06F
:107FC0000E94CC9041CE6AEE77E0CE0101960E94ED
:107FD0004A9BBE016F5F7F4F84E093E10E94C79987
:107FE000182FCE0101960E94DE9A112309F482C354
:107FF0006AE073E1CE018F960E94419B6BE679E0C7
:10800000CE0101960E944A9BBE016F5F7F4FCE0159
:108010008F960E949199AC014F5F5F4FBE01615DE9
:108020007F4FCE0189960E943858CE0101960E945A
:10803000DE9ABE01615D7F4FCE0101960E94419B99
:10804000CE0101960E94A359CE0101960E94DE9AAC
:108050006EEE77E0CE0101960E944A9BBE016F5FF3
:108060007F4FCE0189960E949B998C01CE0101968B
:108070000E94DE9A6BEF7BE0CE0183960E944A9BC2
:108080006BEF7BE0CE014D960E944A9B10161106C5
:108090000CF099C1A8014F5F5F4F8DA59EA54817B1
:1080A000590790F4BE01675D7F4FCE0101960E9493
:1080B0003858BE016F5F7F4FCE0183960E94A59A0C
:1080C000CE0101960E94DE9A980150E040E0BE0188
:1080D000675D7F4FCE0101960E945B9BBE016F5F83
:1080E0007F4FCE014D960E94A59ACE0101960E9427
:1080F000DE9A89A19AA1892B09F418C2CE014D9666
:108100000E94DB986B0121E0C21AD108860138E198
:10811000C316D10414F007E110E017FF02C00FEFFF
:108120001FEFB801CE010B960E94959860EF77E0A3
:10813000CE0141960E944A9BBE01655F7F4FCE01F2
:1081400041960E94F899BC01CE0101960E94419B84
:10815000CE0101960E94A359CE0101960E94DE9A9B
:10816000CE0141960E94DE9ACE010B960E94DE9AC5
:10817000BE016D5D7F4FCE0189960E948E9A6EEE94
:1081800077E0CE0101960E944A9BBE016F5F7F4F50
:10819000CE0189960E949B997C01CE0101960E9496
:1081A000DE9A6BEF7BE0CE0183960E945E986BEFC8
:1081B0007BE0CE014D960E945E981E141F040CF0C9
:1081C00010C1A7014F5F5F4F8DA59EA548175907A6
:1081D00090F4BE01675D7F4FCE0101960E94385832
:1081E000BE016F5F7F4FCE0183960E94A59ACE019C
:1081F00001960E94DE9A970150E040E0BE01675D63
:108200007F4FCE0101960E945B9BBE016F5F7F4F47
:10821000CE014D960E94A59ACE0101960E94DE9A4B
:10822000A8014F5F5F4F8AE0849F9001859F300DCA
:108230001124A9014A515E4E5A01FE0131963F01B7
:10824000F12CE12C809F9001819F300D1124A90118
:108250004C505E4E2A012AE2322E89A19AA1892B26
:1082600009F4E8C0CE014D96E114F10409F0CEC046
:10827000D7FCCCC00E94E698A114B10439F044E0C8
:1082800050E0B501CE014D960E94A990B501CE01F6
:1082900041960E944A9B65EF77E0CE0147960E9487
:1082A0004A9BBE016F5E7F4FCE0147960E94F899B0
:1082B000BC01CE010B960E94419BCE010B960E9401
:1082C000A359CE010B960E94DE9ACE0147960E94DA
:1082D000DE9ACE0141960E94DE9A89A19AA1029768
:1082E00008F48DC061E070E0CE014D960E94B69911
:1082F000082E000C990B803391050CF44C96E32D5D
:10830000E81B8E2FF2018083FFEFEF1AFF0ABE01F8
:108310006D5D7F4FCE0189960E948E9A6EEE77E05A
:10832000CE010B960E944A9BBE01655F7F4FCE0136
:1083300089960E949B994C01CE010B960E94DE9A71
:108340006BEF7BE0CE0183960E945E986BEF7BE043
:10835000CE014D960E945E98181419040CF05CC072
:10836000A4014F5F5F4F8DA59EA54817590790F454
:10837000BE01675D7F4FCE010B960E943858BE014B
:10838000655F7F4FCE0183960E94A59ACE010B9622
:108390000E94DE9A940150E040E0BE01675D7F4F8D
:1083A000CE010B960E945B9BBE01655F7F4FCE01A5
:1083B0004D960E94A59ACE010B960E94DE9A52E03D
:1083C000650E711C4ACF6BEF7BE0CE0183960E9455
:1083D0005E98BE01675D7F4FCE014D960E948E9ADA
:1083E00088CE6BEF7BE0CE0183960E945E98BE0143
:1083F000675D7F4FCE014D960E948E9A11CFCE01C0
:108400004D960E94DB98F20160837ECF0E94DB983C
:10841000F3017183608378CF6BEF7BE0CE018396AD
:108420000E945E98BE01675D7F4FCE014D960E940F
:108430008E9AC5CFD7FE8BC06EEE77E0CE010B963D
:108440000E944A9BBE01655F7F4FCE0183960E94CA
:108450009B998C01CE010B960E94DE9A17FF66C095
:1084600009811A810931110514F008E110E0101694
:10847000110614F001E010E00093E811B801CE01FC
:1084800041960E94959863E078E0CE0147960E945D
:108490004A9BBE016F5E7F4FCE0147960E94F899BE
:1084A000BC01CE010B960E94419BCE010B960E940F
:1084B000A359CE010B960E94DE9ACE0147960E94E8
:1084C000DE9ACE0141960E94DE9AE114F10451F148
:1084D0008B819C8197FF02C090E080E09093EA112D
:1084E0008093E91121E0E216F104E1F08D819E8193
:1084F000081719070CF4C8011816190614F081E0C2
:1085000090E081508093ED1132E0E316F10451F0D8
:108510008F8198851816190614F081E090E081503B
:108520008093EE118CE291E00E945590CE014D9621
:108530000E94DE9ACE0183960E94DE9ACE01899631
:108540000E94DE9ACE018F960E94DE9A7FCB8091A8
:10855000E711082E000C990B081719070CF083C0BF
:10856000B701CE0141960E9495986DE078E0CE016A
:1085700047960E944A9BBE016F5E7F4FCE01479691
:108580000E94F899BC01CE010B960E94419BCE013E
:108590000B960E94A359CE010B960E94DE9ACE0143
:1085A00047960E94DE9ACE0141960E94DE9A8AE0AA
:1085B000809FF001819FF00D1124EA51FE4E81E071
:1085C000878783E090E0918B808B938B828BE11483
:1085D000F10409F4ABCF8B819C818038910514F0B4
:1085E0008FE790E080384FEF940714F480E89FEF16
:1085F000878751E0E516F10409F498CF8AE0809F5F
:10860000F001819FF00D1124EA51FE4E8D819E8173
:1086100097FF02C090E080E0918B808B82E0E816AB
:10862000F10409F483CF8AE0809FF001819FF00D6F
:108630001124EA51FE4E8F81988597FF02C090E089
:1086400080E0938B828B8091E811082E000C990BAF
:10865000081719071CF00F5F0093E8118CE291E0F6
:108660000E94CC9063CFBE016D5D7F4FCE014796D7
:108670000E94419B6091E711062E000C770BCE0102
:108680000B960E94959865E178E0CE0141960E9494
:108690004A9BBE01695E7F4FCE0141960E94F899C8
:1086A00066E278E00E94E299BE01655F7F4F0E941A
:1086B000F899BC01CE0147960E948E9ACE01419650
:1086C0000E94DE9ACE010B960E94DE9ABE01695E80
:1086D0007F4FCE010B960E94419BCE010B960E94CC
:1086E000F256CE010B960E94DE9ACE0147960E946A
:1086F000DE9A1CCF6AE278E0CE0101960E944A9B86
:10870000BE016F5F7F4F84E093E10E94C799182FED
:10871000CE0101960E94DE9A1123C9F16BE679E041
:10872000CE0101960E944A9BBE016F5F7F4F8AE097
:1087300093E10E949199AC014F5F5F4F6AE073E152
:10874000CE010B960E943858BE01655F7F4F86EEC2
:1087500092E10E94A59ACE010B960E94DE9ACE016C
:1087600001960E94DE9A86EE92E10E94DB986115E6
:10877000710531F481E0809385040E94E51664CA96
:108780006130710509F060CA10928504F6CF6FE27E
:1087900078E0CE0101960E944A9BBE016F5F7F4F39
:1087A00084E093E10E94C799182FCE0101960E94A0
:1087B000DE9A112309F43AC143E050E06AE073E124
:1087C000CE0101960E943858BE016F5F7F4F86EE42
:1087D00092E10E94A59ACE0101960E94DE9A66EE71
:1087E00072E1CE0101960E94419BCE0101960E944A
:1087F000A359CE0101960E94DE9A66EE72E1CE0187
:1088000001960E94419BCE0101960E94499ABC01AB
:1088100081EE93E10E948E9ACE0101960E94DE9A2B
:1088200066EE72E1CE0101960E94419BCE01019657
:108830000E94499ABC018BED93E10E948E9ACE0171
:1088400001960E94DE9A4091E5135091E61341157E
:10885000510549F08BE691E1009729F0BC0181EECA
:1088600093E10E94A9904091DF135091E0134115CC
:10887000510549F089EC91E1009729F0BC018BED9D
:1088800093E10E94A99090E080E00E947F9062E9CD
:1088900077E0CE0101960E944A9B66EE72E1CE011E
:1088A00001960E94F899BC01CE0141960E94419B1D
:1088B000CE0101960E94DE9A8091C5119091C61159
:1088C000892B39F4BE016F5E7F4F8DEF9DE00E94D2
:1088D000959D68EB7BE080E090E00E9439A5809157
:1088E000C5119091C611029709F087C066EE72E13A
:1088F000CE0147960E94419B63E378E0CE0101964A
:108900000E944A9BCE0101960E94CBACCE010196FB
:108910000E94DE9A64EF71E080E090E00E9439A549
:1089200066E378E0CE0101960E944A9BCE01019653
:108930000E94CBACCE0101960E94DE9A6CED75E0F0
:1089400080E090E00E9439A56FE378E0CE010196C7
:108950000E944A9BCE0101960E94CBACCE010196AB
:108960000E94DE9A64EF71E080E090E00E9439A5F9
:108970006DE478E0CE0101960E944A9BCE010196FB
:108980000E94CBACCE0101960E94DE9A64EF71E0AA
:1089900080E090E00E9439A562E977E0CE0101967F
:1089A0000E944A9BBE01695E7F4FCE0101960E94E4
:1089B000F899BC01CE010B960E94419BCE01019615
:1089C0000E94DE9ACE010B960E94E698BE01655F7A
:1089D0007F4FCE0101960E94419BCE0101960E94DD
:1089E000CBACCE0101960E94DE9ACE010B960E947E
:1089F000DE9ACE0147960E94DE9A68EB7BE080E02B
:108A000090E00E9439A56BE671E1CE0101960E94CB
:108A10004A9BCE0101960E94A359CE0101960E9465
:108A2000DE9A1092EA04CE0141968ECD6BE578E095
:108A3000CE0101960E944A9BBE016F5F7F4F84E08A
:108A400093E10E94C799182FCE0101960E94DE9AE9
:108A5000112309F487C044E050E06AE073E1CE01DD
:108A600001960E943858BE016F5F7F4F86EE92E1FB
:108A70000E94A59ACE0101960E94DE9A6AE977E0EB
:108A8000CE0101960E944A9B66EE72E1CE010196EC
:108A90000E94F899BC01CE010B960E94419BCE0129
:108AA00001960E94DE9A8091C5119091C611892B82
:108AB00069F4BE01655F7F4F8DEF9DE00E94959D3B
:108AC00068E873E180E090E00E9439A58091C511CB
:108AD0009091C611029759F560E678E0CE010196B3
:108AE0000E944A9B8091EA129091EB12892B21F50A
:108AF00069E678E0CE0101960E945E98BE01655F4E
:108B00007F4FCE0141960E94419BCE0141960E942B
:108B1000CBACCE0141960E94DE9A60ED77E080E01A
:108B200090E00E9439A5CE0101960E94DE9A109233
:108B3000EA04CE010B9608CDBE016F5F7F4FCE01D8
:108B400041960E94419BCE0141960E94CBACCE0142
:108B500041960E94DE9A60ED77E080E090E00E940E
:108B600039A5CCCF62E778E0CE0101960E944A9BFE
:108B7000BE016F5F7F4F84E093E10E94C799182F79
:108B8000CE0101960E94DE9A112309F462C06AE0C8
:108B900073E186EE92E10E948E9A81E08093EA046E
:108BA0006AE073E1CE0101960E94419BCE010196DD
:108BB0000E94A359CE0101960E94DE9A8091C511B0
:108BC0009091C611029709F166EE72E18DEF9DE07A
:108BD0000E94959D68EB7BE080E090E00E9439A5C3
:108BE000CE0101960E94BC70BE016F5F7F4F8AE08C
:108BF00093E10E94A59ACE0101960E94DE9A60ED53
:108C000077E080E090E00E9439A58091C5119091B5
:108C1000C611029771F466EE72E1CE0101960E94D0
:108C2000419BCE0101960E94CBACCE0101960E94E1
:108C3000DE9A80910E1390910F13892B09F404C8CA
:108C400060EC75E0CE0101960E944A9B6AE073E1F8
:108C5000A4C866E778E0CE0101960E944A9BBE0157
:108C60006F5F7F4F84E093E10E94C799182FCE0178
:108C700001960E94DE9A112309F462C08091C51109
:108C80009091C611019711F00C94243ECE010196EB
:108C90000E94CC2F8D819E81009709F44BC0E98101
:108CA000FA812081222309F445C0079708F442C0C5
:108CB0006DEF78E0CE010B960E94389B48EC50E0B7
:108CC0006FEF7FEFCE010B960E94CF59CE010B962E
:108CD0000E94DE9ABE016F5F7F4FCE010B960E940D
:108CE000419B40ED57E06FEF7FEFCE010B960E9466
:108CF0006857CE010B960E94DE9A6CE778E0CE01B1
:108D00000B960E944A9B6AE073E1CE010B960E948B
:108D1000F899BC01CE0141960E94419BCE0141963B
:108D20000E94F256CE0141960E94DE9ACE010B9629
:108D30000E94DE9ACE0101960E94DE9A0C94243E97
:108D40006AE878E0CE0101960E944A9BBE016F5FFF
:108D50007F4F84E093E10E94C799182FCE010196BE
:108D60000E94DE9A112361F125E030E044E050E0FA
:108D70006AE073E1CE0101960E945B9BBE016F5FCA
:108D80007F4F86EE92E10E94A59ACE0101960E9445
:108D9000DE9A6AE073E1CE0101960E94419BCE010A
:108DA00001960E94A359CE0101960E94DE9A86EE9A
:108DB00092E10E94DB98CB010E9464250C94243E32
:108DC0006FE878E0CE0101960E944A9BBE016F5F7A
:108DD0007F4F84E093E10E94C799182FCE0101963E
:108DE0000E94DE9A112361F127E030E046E050E076
:108DF0006AE073E1CE0101960E945B9BBE016F5F4A
:108E00007F4F86EE92E10E94A59ACE0101960E94C4
:108E1000DE9A86EE92E10E94DB98672B69F410924D
:108E2000310D6AE073E1CE0101960E94419BCE01B3
:108E300001960E94A3597ECF81E08093310DF1CF3E
:108E400066E978E0CE0101960E944A9BBE016F5F01
:108E50007F4F84E093E10E94C799182FCE010196BD
:108E60000E94DE9A112309F4F7C18091610C909160
:108E7000620C1816190614F00C94263E8091830497
:108E800090918404909382048093810488E592E019
:108E9000909384048093830484ED9FE00E94C38BAD
:108EA000198A1A8A1B8A1C8A66246394712C2E01E3
:108EB00091E1490E511CFE017596FEABEDAB809120
:108EC000610C9091620C861597050CF4BBC1009162
:108ED000830410918404093DFFE01F070CF0B2C128
:108EE00072016801C418D508C6018E0D9F1D0E942D
:108EF000D1B8F70181937F012DA93EA9E217F307AD
:108F000099F789889A88AB88BC88A5019401C50126
:108F1000B4010E9497BC81119DC0C8010496909332
:108F20008404809383048DE3E82E8CE0F82E0953AB
:108F30001C40C8018E0D9F1D0E94D1B8F70181937E
:108F40007F0121E63CE02E173F0799F723E0B501AA
:108F5000A401CE0101960E94E69ABE016F5F7F4F89
:108F6000CE010B960E94419B65E979E0CE010B96FC
:108F70000E94E299BC018CEE92E10E948E9ACE0191
:108F80000B960E94DE9ACE0101960E94DE9A6DE356
:108F90007CE0CE0101960E944A9BBE016F5F7F4F2D
:108FA00086EE92E10E94A59ACE0101960E94DE9A79
:108FB0006AE978E0CE0101960E944A9BBE016F5F8C
:108FC0007F4F86EE92E10E94C799182FCE0101963D
:108FD0000E94DE9A112309F49EC06AE978E0CE016E
:108FE00001960E944A9BA090EA12B090EB12A11445
:108FF000B10409F48CC08D809E808114910409F421
:1090000086C0E090DB11F090DC11E818F9080091BF
:10901000E6121091E71229803A80E114F104E1F59B
:1090200069817A81C8010E949BBF8C01009709F475
:109030006EC06091D7117091D8114091DB115091A1
:10904000DC110E9453BF8091DB119091DC11080F5D
:10905000191FE6CF8091810490918204909384043B
:1090600080938304812FE6960FB6F894DEBF0FBE7F
:10907000CDBFDF91CF911F910F91FF90EF90DF90C7
:10908000CF90BF90AF909F908F907F906F905F90A8
:109090004F903F902F9008956501C801F7FE62C080
:1090A000680169817A81C8010E949BBF4C010097C9
:1090B00051F15C01A01AB10AA501B801C6010E94D4
:1090C00053BFCA0CDB1C6091D7117091D81140912D
:1090D000DB115091DC11C6010E9453BF8091DB115E
:1090E0009091DC11C80ED91E0D811E81080D191D2D
:1090F0008091EA129091EB128E0D9F1D9093EB12CE
:109100008093EA12CECFB801C6010E9477BFCE018C
:1091100001960E94DE9A66EE72E18CEE92E10E9468
:10912000629A6CEE72E1CE0101960E94419BCE01E3
:1091300001960E94F256CE0101960E94DE9A80911D
:109140008304909184048496909384048093830490
:1091500064E170E080E090E00E9439A5FFEF6F1AB3
:109160007F0AADCEB1010E949BBF009729F0880D08
:10917000991DCE0CDF1CF6CFAC14BD0441F28091DA
:10918000E8129091E9128C159D0588F4B6016F5F85
:109190007F4FC8010E944CBE009709F4B8CF90934E
:1091A000E7128093E612D092E912C092E812409141
:1091B000EA125091EB124150510957FDA8CFBE0160
:1091C0006F5F7F4F86EE92E10E9443998C0197FD7D
:1091D0009ECF2D813E81280F391F8091E6129091FC
:1091E000E712820F931F4091EA125091EB12421B3B
:1091F000530BBC018E0D9F1D0E945CBF8091EA1233
:109200009091EB128E0D9F1D9093EB128093EA12BA
:109210002091E6123091E712820F931FFC01108219
:109220008091E6129091E7126091D7117091D81158
:109230004091DB115091DC11800F911F0E9453BFB0
:10924000A801B9CF80918104909182049093840405
:10925000809383040C94263E6EE978E0CE0101965B
:109260000E944A9BBE016F5F7F4F84E093E10E94A2
:10927000C799182FCE0101960E94DE9A1123D9F1C9
:1092800026E030E045E050E06AE073E1CE0101966F
:109290000E945B9BBE016F5F7F4F86EE92E10E9452
:1092A000A59ACE0101960E94DE9A86EE92E10E9476
:1092B000DB98672B29F410923C0C88E592E0C6CF2E
:1092C00081E080933C0C1092620C1092610C109221
:1092D000380C1092390C10923A0C10923B0C0E94F0
:1092E000F80F6093340C7093350C8093360C909388
:1092F000370C0C94263E64EA78E0CE0101960E9479
:109300004A9BBE016F5F7F4F84E093E10E94C79943
:10931000182FCE0101960E94DE9A112309F478C01D
:1093200080910E1390910F13079710F40C94263E22
:1093300046E050E06AE073E1CE0101960E943858A1
:10934000BE016F5F7F4F86EE92E10E94A59ACE012B
:1093500001960E94DE9A86EE92E10E94D098609378
:10936000E6047093E7048093E8049093E9046DEEBB
:1093700078E08CEE92E10E94699A4091E604509167
:10938000E7046091E8047091E90421E0CE010196C0
:109390000E94E69ABE016F5F7F4FCE010B960E943E
:1093A000419B6EEB76E0CE010B960E94E299BC01E8
:1093B0008CEE92E10E94629ACE010B960E94DE9A98
:1093C000CE0101960E94DE9A6CEE72E1CE0101960A
:1093D0000E94419BCE0101960E94F256CE01019659
:1093E0000E94DE9A0E94F80F28EE33E040E050E041
:1093F0000E9419B9CA01B9010E94AFB760932C0D40
:1094000070932D0D80932E0D90932F0D0C94263E6E
:109410006BEA78E0CE0101960E944A9BBE016F5F25
:109420007F4F84E093E10E94C799182FCE010196E7
:109430000E94DE9A112309F456C080910E13909178
:109440000F13079710F40C94263E46E050E06AE0B4
:1094500073E1CE0101960E943858BE016F5F7F4FC5
:1094600086EE92E10E94A59ACE0101960E94DE9AB4
:1094700086EE92E10E94D0986093EB047093EC0426
:109480008093ED049093EE046DED78E08CEE92E124
:109490000E94699A4091EB045091EC046091ED04B4
:1094A0007091EE0421E0CE0101960E94E69ABE0181
:1094B0006F5F7F4FCE010B960E94419B6EEB76E073
:1094C000CE010B960E94E299BC018CEE92E10E94C3
:1094D000629ACE010B960E94DE9ACE0101960E94FE
:1094E000DE9A0C948B3F0E94B31B182F81110C94B1
:1094F000263EB8CD11E0B6CDBF92CF92DF92EF926B
:10950000FF920F931F93CF93DF93CDB7DEB7A4974E
:109510000FB6F894DEBF0FBECDBF8091140C882328
:1095200091F01092140CA4960FB6F894DEBF0FBE03
:10953000CDBFDF91CF911F910F91FF90EF90DF9002
:10954000CF90BF90089580910E1390910F130497C0
:1095500008F043C06AE778E0CE0101960E944A9B7A
:10956000BE016F5F7F4F84E093E10E94C799082F8F
:10957000CE0101960E94DE9A002379F161E070E04D
:109580008AE093E10E94B69986340CF034C48033AB
:109590000CF4845E6AE270E0681B710987FD7395C4
:1095A000CE0101960E949598BE016F5F7F4F8AE0C1
:1095B00093E10E94A59ACE0101960E94DE9A6AE08C
:1095C00073E188EF92E10E948E9A8AE093E10E9413
:1095D000DB98CB010E941A77A6CF80910E13909151
:1095E0000F130297029730F561EA7BE0CE010196F6
:1095F0000E944A9BBE016F5F7F4F84E093E10E940F
:10960000C799082FCE0101960E94DE9A002391F09F
:1096100061E070E08AE093E10E94B69986340CF034
:10962000EAC362EB78E088EF92E10E945E9888EFEF
:1096300092E1CDCF6BED77E0CE0101960E944A9B7F
:10964000BE016F5F7F4F84E093E10E94C799082FAE
:10965000CE0101960E94DE9A002309F4DDC366EB79
:1096600078E0CE0101960E944A9BCE0101960E94AD
:10967000F256CE0101960E94DE9A62EC78E0CE01AD
:1096800007960E944A9B6BED73E1CE0107960E94FC
:10969000F899BC01CE0101960E94419BCE01019632
:1096A0000E94F256CE0101960E94DE9ACE010796E4
:1096B0000E94DE9A68ED78E0CE0107960E944A9BF0
:1096C00067EE73E1CE0107960E94F899BC01CE01C6
:1096D00001960E94419BCE0101960E94F256CE0156
:1096E00001960E94DE9ACE0107960E94DE9A609152
:1096F000C5047091C6048091C7049091C8040E946B
:10970000B1B720E030E048EC52E40E9429BAAB0146
:10971000BC0122E0CE0107960E94E69A66EE78E050
:10972000CE010D960E944A9BBE01695F7F4FCE011C
:109730000D960E94F89963EF75E00E94E299BC01D2
:10974000CE0101960E94419BCE0101960E94F256E5
:10975000CE0101960E94DE9ACE010D960E94DE9AFD
:10976000CE0107960E94DE9A4091C1045091C20436
:109770006091C3047091C40424E0CE0107960E9456
:10978000E69A6BEF78E0CE010D960E944A9BBE01EF
:10979000695F7F4FCE010D960E94F899BC01CE0102
:1097A00001960E94419BCE0101960E94F256CE0185
:1097B00001960E94DE9ACE010D960E94DE9ACE019D
:1097C00007960E94DE9A4091B5045091B6046091CC
:1097D000B7047091B80422E0CE0107960E94E69A81
:1097E0004091AD045091AE046091AF047091B0040B
:1097F00023E0CE010D960E94E69A4091B904509163
:10980000BA046091BB047091BC0422E0CE0143967F
:109810000E94E69A4091B1045091B2046091B30461
:109820007091B40423E0CE0149960E94E69A68E163
:1098300079E0CE014F960E944A9BBE01675E7F4F42
:10984000CE014F960E94F8996DE279E00E94E2996C
:10985000BE016D5E7F4F0E94F89960E379E00E943F
:10986000E299BE01635F7F4F0E94F8996DE279E053
:109870000E94E299BE01695F7F4F0E94F89966E3FA
:1098800079E00E94E299BC01CE0101960E94419BC1
:10989000CE0101960E94F256CE0101960E94DE9AF8
:1098A000CE014F960E94DE9ACE0149960E94DE9A22
:1098B000CE0143960E94DE9ACE010D960E94DE9A5A
:1098C000CE0107960E94DE9A63E377E0CE014996C7
:1098D0000E94389BF0907E110F2D0F2C000C110B65
:1098E0000115110509F07EC120917F113091801181
:1098F000409181115091821160E070E080EA90E423
:109900000E9429BAAB01BC0122E0CE0101960E945F
:10991000E69A68E176E0CE0107960E944A9BBE0176
:109920006F5F7F4FCE0107960E94F8996CE17BE054
:109930000E94E299BC01CE0149960E94629ACE0132
:1099400007960E94DE9ACE0101960E94DE9AC80117
:109950000297029738F58F2D9AE08902B001112401
:10996000CE0101960E9495986BE379E0CE010796AF
:109970000E944A9BBE016F5F7F4FCE0107960E94F7
:10998000F89965E17BE00E94E299BC01CE0149961D
:109990000E94629ACE0107960E94DE9ACE0101963D
:1099A0000E94DE9A63E177E00430110519F034F08B
:1099B0006BE077E0CE0149960E940B9ABE01675E8C
:1099C0007F4FCE0101960E94419BCE0101960E94DD
:1099D000F256CE0101960E94DE9A67E479E0CE014C
:1099E00049960E945E9880917B1160917C117091E4
:1099F0007D1183300CF09BC3CE0101960E94959897
:109A000062E479E0CE0107960E944A9BBE016F5F37
:109A10007F4FCE0107960E94F8996BE37AE00E948F
:109A2000E299BC01CE0149960E94629ACE01079646
:109A30000E94DE9ACE0101960E94DE9ABE01675E08
:109A40007F4FCE0101960E94419BCE0101960E945C
:109A5000F256CE0101960E94DE9A409183115091F8
:109A60008411609185117091861122E0CE010796D4
:109A70000E94E69A67E579E0CE010D960E944A9B26
:109A8000BE01695F7F4FCE010D960E94F8996DE689
:109A900079E00E94E299BC01CE0101960E94419BAF
:109AA000CE0101960E94F256CE0101960E94DE9AE6
:109AB000CE010D960E94DE9ACE0107960E94DE9A94
:109AC0004091991150919A1160919B1170919C1144
:109AD00022E0CE0107960E94E69A64E779E0CE0183
:109AE0000D960E944A9BBE01695F7F4FCE010D9685
:109AF0000E94F89965E076E00E94E299BC01CE01EF
:109B000001960E94419BCE0101960E94F256CE0121
:109B100001960E94DE9ACE010D960E94DE9ACE0139
:109B200007960E94DE9A83E9E82E84E0F82E01E091
:109B300010E099E1B92EE2E0EE0EF11C8091930461
:109B400090919404801791070CF457C0F701C080DE
:109B5000D180B601CE0107960E949598B801CE013A
:109B60000D960E94959867E879E0CE0143960E9491
:109B70004A9BBE01635F7F4FCE0143960E94F899D6
:109B80006FE879E00E94E299BE01695F7F4F0E9411
:109B9000F89962E979E00E94E299BC9CB001BD9C11
:109BA000700D1124685F7D4F0E94E299BC01CE01C7
:109BB00001960E94419BCE0101960E94F256CE0171
:109BC00001960E94DE9ACE0143960E94DE9ACE0153
:109BD0000D960E94DE9ACE0107960E94DE9A0F5FD4
:109BE0001F4FA9CF0130110509F0B1CE65E277E032
:109BF000CE0149960E940B9AAACE8091C5119091F0
:109C0000C611892B71F468E979E0CE0101960E94B2
:109C10004A9BCE0101960E94F256CE0101960E9407
:109C2000DE9A8091C5119091C611019771F467EA8F
:109C300079E0CE0101960E944A9BCE0101960E94D6
:109C4000F256CE0101960E94DE9A8091C511909144
:109C5000C611029771F461EB79E0CE0101960E9482
:109C60004A9BCE0101960E94F256CE0101960E94B7
:109C7000DE9A6091D2047091D304CE0107960E94BF
:109C8000959863EC79E0CE010D960E944A9BBE0147
:109C9000695F7F4FCE010D960E94F899BC01CE01FD
:109CA00001960E94419BCE0101960E94F256CE0180
:109CB00001960E94DE9ACE010D960E94DE9ACE0198
:109CC00007960E94DE9A4091E6045091E704609165
:109CD000E8047091E90422E0CE0107960E94E69A1A
:109CE00060EE79E0CE010D960E944A9BBE01695F4D
:109CF0007F4FCE010D960E94F8996EEB76E00E94A0
:109D0000E299BC01CE0101960E94419BCE010196D1
:109D10000E94F256CE0101960E94DE9ACE010D9667
:109D20000E94DE9ACE0107960E94DE9A4091EB04D3
:109D30005091EC046091ED047091EE0422E0CE01AC
:109D400007960E94E69A60EF79E0CE010D960E9498
:109D50004A9BBE01695F7F4FCE010D960E94F89924
:109D60006EEB76E00E94E299BC01CE0101960E9462
:109D7000419BCE0101960E94F256CE0101960E94AF
:109D8000DE9ACE010D960E94DE9ACE0107960E94C1
:109D9000DE9A6AEF76E0CE0101960E94389BCE01F2
:109DA00001960E940F57CE0101960E94DE9A6091A3
:109DB0002E0C70912F0CCE0101960E949598CE0129
:109DC00001960E940F57CE0101960E94DE9A6BED1C
:109DD00076E0CE0101960E94389BCE0101960E944A
:109DE000F256CE0101960E94DE9A1092EA04CE014C
:109DF00049960E94DE9A0E94F80F6093280D709396
:109E0000290D80932A0D90932B0D6BEF7BE08AE058
:109E100093E10E945E9887CB80910E1390910F136F
:109E20008330910508F080C18130910509F061C04F
:109E300070E060E08AE093E10E94B699182F812FCC
:109E4000110F990B0E942DBF892BB1F00E94D516DE
:109E50000E94265761E67AE0CE0101960E944A9B55
:109E60004AE050E070E060E0CE0101960E94CF59D8
:109E7000CE0101960E94DE9A6AE073E1CE01079658
:109E80000E94419B70E060E0CE0107960E94B69967
:109E9000823409F4F5C00CF0A7C0803309F426C160
:109EA0000CF081C0833209F40FC18A3209F415C164
:109EB000BE01695F7F4F88EF92E10E948E9A70E049
:109EC00060E088EF92E10E94B699082E000C990B91
:109ED000C0970A9738F488EF92E10E94DB98CB0193
:109EE0000E941A7764E670E080E090E00E9439A555
:109EF0006CC0029709F0A3CF6AE778E0CE01019623
:109F00000E944A9BBE016F5F7F4F84E093E10E94F5
:109F1000C799082FCE0101960E94DE9A002309F40A
:109F20008ECF61E070E08AE093E10E94B699682FDD
:109F3000CE0101960E94169BBE016F5F7F4F88EF96
:109F400092E10E94A59ACE0101960E94DE9A70E0ED
:109F500060E08AE093E10E94B699182F8091310D5C
:109F6000882309F46CCF60E07AE0CE0101960E946C
:109F70004A9B6AE073E1CE0101960E94F89961E67E
:109F80007AE00E94E299BC0184ED9FE00E94959DD9
:109F9000CE0101960E94DE9A68EF72E184ED9FE0A7
:109FA0000E94A39D4CCF813309F4AFC0813409F0E6
:109FB0007FCF6DE07AE08AE093E10E945E98809125
:109FC0002A0C90912B0C0E941A77CE0107960E94C2
:109FD000DE9A0E94F80F6093280D7093290D8093EC
:109FE0002A0D90932B0D07CF813619F30CF041C049
:109FF000833409F45DC0843409F05ACF8091FC1297
:10A000009091FD12892B09F361E070E0CE01079673
:10A010000E94B699182F8091310D882361F066E077
:10A020007AE084ED9FE00E94939D68EF72E184EDF9
:10A030009FE00E94A39D10330CF4145E6AE270E06E
:10A04000611B710917FD7395CE0101960E949598C9
:10A05000BE016F5F7F4F88EF92E10E94A59ACE010B
:10A0600001960E94DE9A88EF92E10E94DB98CB0174
:10A07000AACF8336E9F024F0843609F4BFCF18CF95
:10A080008091FC129091FD12029758F460E17AE001
:10A090008AE093E10E945E981092300D8CEF9FEF62
:10A0A00092CF62EB78E088EF92E10E945E98DBCF7E
:10A0B00063E17AE08AE093E10E945E9881E0809318
:10A0C000300D8DEF9FEF7FCF66E17AE08AE093E17C
:10A0D0000E945E988EEF9FEF76CF69E17AE08AE08A
:10A0E00093E10E945E988FEF9FEF6DCF62E077E083
:10A0F00088EF92E10E945E9862E077E08AE093E167
:10A100000E945E9890E080E05ECF6AE17AE088EF9E
:10A1100092E10E945E986AE17AE08AE093E10E940F
:10A120005E9881E090E04FCF0E94763D64CECE01F4
:10A1300001960E9495986CE17AE0CE0107960E9404
:10A140004A9BBE016F5F7F4FCE0107960E94F89930
:10A1500068CCCF92DF92EF92FF920F931F93CF9331
:10A16000DF93CDB7DEB7E0970FB6F894DEBF0FBE32
:10A17000CDBF8E01015E1F4F8130910509F0B7C040
:10A1800065E27AE0CE0101960E944A9B68E27AE09D
:10A19000CE0107960E944A9B6BE27AE0CE010D96B3
:10A1A0000E944A9B6DEC76E0C8010E94389B44E611
:10A1B00050E06FEF7FEFC8010E94885AC8010E94EB
:10A1C000DE9A62EC76E08AE093E10E94699A6091FF
:10A1D000D2047091D304CE0185960E9495986AE0CE
:10A1E00073E1C8010E94419BBE016B5D7F4FC801B6
:10A1F0000E94F899BC01CE018B960E94419B40EDD4
:10A2000057E06FEF7FEFCE018B960E946857CE012B
:10A210008B960E94DE9AC8010E94DE9ACE01859636
:10A220000E94DE9A63EB76E0C8010E94389B44E608
:10A2300050E06FEF7FEFC8010E94885AC8010E946A
:10A24000DE9A6CED79E0C8010E944A9B23E030E081
:10A25000A801BE016F5F7F4FCE0185960E9452AA72
:10A26000BE016B5D7F4F8AE093E10E94A59ACE010B
:10A2700085960E94DE9AC8010E94DE9A80910E1394
:10A2800090910F13892B09F4E3C270E060E08AE03B
:10A2900093E10E94B699082E000C990BC0970A977B
:10A2A00008F0D6C28AE093E10E94DB986B016EE26F
:10A2B0007AE0C8010E944A9B86E08C9DB0018D9D8A
:10A2C000700D112481E090E08C0F9D1F680F791FA5
:10A2D000C8010E94F899BC018AE093E10E948E9A1D
:10A2E000C8010E94DE9A0E94763D182FE2C08A3F84
:10A2F0002FEF920709F023C163E37AE0CE010196C4
:10A300000E944A9B6DE37AE0CE0107960E944A9B29
:10A3100065E47AE0CE010D960E944A9B6DE47AE0F6
:10A32000CE0143960E944A9B64EA76E0C8010E94EF
:10A33000389B44E650E06FEF7FEFC8010E94885AD7
:10A34000C8010E94DE9A6EE976E08AE093E10E94FD
:10A35000699A80917B11EE24E394F12CEC0EFD1EA2
:10A3600096E08902E00CF11C11246AE073E1C80157
:10A370000E94419BB701C8010E94F899BC01CE011F
:10A3800085960E94419B40ED57E06FEF7FEFCE0135
:10A3900085960E946857CE0185960E94DE9AC80174
:10A3A0000E94DE9A6EE876E0C8010E94389B44E67F
:10A3B00050E06FEF7FEFC8010E94885AC8010E94E9
:10A3C000DE9A63E57AE0C8010E944A9B24E030E00F
:10A3D000A801BE016F5F7F4FCE0185960E9452AAF1
:10A3E000BE016B5D7F4F8AE093E10E94A59ACE018A
:10A3F00085960E94DE9AC8010E94DE9A80910E1313
:10A4000090910F13892B09F498C070E060E08AE006
:10A4100093E10E94B699082E000C990BC0970A97F9
:10A4200008F08BC08AE093E10E94DB9862307105EE
:10A43000810591050CF46EC062E876E0C8010E94C7
:10A44000389B44E650E06FEF7FEFC8010E946857E9
:10A45000C8010E94DE9A44EF51E063E070E0CE0153
:10A4600085960E947FA969E57AE0C8010E944A9B0F
:10A470006AE073E1C8010E94F89960E67AE00E9400
:10A48000E299BE016B5D7F4F0E94F899BC018AE0A2
:10A4900093E10E948E9AC8010E94DE9ACE018596B1
:10A4A0000E94DE9A0E94763D182FCE0143960E94AC
:10A4B000DE9ACE010D960E94DE9ACE0107960E948A
:10A4C000DE9ACE0101960E94DE9A6CEF75E01111C2
:10A4D00002C06DEE75E0CE0101960E94389B48ECFB
:10A4E00050E06FEF7FEFCE0101960E946857CE01DA
:10A4F00001960E94DE9AE0960FB6F894DEBF0FBE7A
:10A50000CDBFDF91CF911F910F91FF90EF90DF9022
:10A51000CF90089569E57AE0C8010E944A9B6AE0FD
:10A5200073E1C8010E94F899BC018AE093E10E949E
:10A530008E9AC8010E94DE9AB5CF10E0B6CF0F9672
:10A5400009F0ECC0CE0101967C016BEF7BE0C70106
:10A550000E944A9B96E0E90EF11C0E151F05A9F713
:10A5600063E67AE0CE0101960E945E9880917E11AA
:10A57000811130C020917F11309180114091811163
:10A580005091821160E070E080EA90E40E9429BA64
:10A59000AB01BC0122E0CE0185960E94E69A69E6F5
:10A5A0007AE0C8010E944A9BBE016B5D7F4FC801E3
:10A5B0000E94F89965E17BE00E94E299BC01CE011E
:10A5C00001960E94629AC8010E94DE9ACE01859689
:10A5D0000E94DE9A67E776E0CE0107960E94699AAC
:10A5E0006BE676E0CE010D960E94699A6FE576E003
:10A5F000CE0143960E94699A63E576E0CE014996C2
:10A600000E94699A6DE476E0C8010E94699A6EE33F
:10A6100076E0C8010E94389B44E650E06FEF7FEF80
:10A62000C8010E94885AC8010E94DE9A6BEF7BE045
:10A630008AE093E10E945E9880917E1161E070E073
:10A640006C0F7D1F26E08202600D711D1124C80170
:10A650000E94419B40ED57E06FEF7FEFC8010E94E1
:10A660006857C8010E94DE9A6FE276E0C8010E9436
:10A67000389B44E650E06FEF7FEFC8010E94885A94
:10A68000C8010E94DE9A6AE073E1C8010E94419B02
:10A6900025E030E0A801BE016F5F7F4FCE018596B7
:10A6A0000E9452AABE016B5D7F4F8AE093E10E9437
:10A6B000A59ACE0185960E94DE9AC8010E94DE9A74
:10A6C00080910E1390910F13892B31F170E060E0AF
:10A6D0008AE093E10E94B699082E000C990BC0976E
:10A6E0000A97D0F461E176E0C8010E944A9B6AE0D3
:10A6F00073E1C8010E94F899BC018AE093E10E94CD
:10A700008E9AC8010E94DE9A0E94763D182FCE01D3
:10A7100049960E94DE9AC9CE10E0F9CF6CE67AE045
:10A72000CE0101960E944A9B6CEA79E0CE01079621
:10A730000E944A9B6FE67AE0CE010D960E944A9BEA
:10A740006FE176E0C8010E94389B44E650E06FEF6D
:10A750007FEFC8010E94885AC8010E94DE9A69E111
:10A7600076E08AE093E10E94699A8091C511909108
:10A77000C61126E0289F7001299FF00C112481E06A
:10A7800090E08C0F9D1FE80EF91E6AE073E1C8018E
:10A790000E94419BB701C8010E94F899BC01CE01FB
:10A7A00085960E94419B40ED57E06FEF7FEFCE0111
:10A7B00085960E946857CE0185960E94DE9AC80150
:10A7C0000E94DE9A69E076E0C8010E94389B44E668
:10A7D00050E06FEF7FEFC8010E94885AC8010E94C5
:10A7E000DE9A6AE073E1C8010E94419B23E030E0F9
:10A7F000A801BE016F5F7F4FCE0185960E9452AACD
:10A80000BE016B5D7F4F8AE093E10E94A59ACE0165
:10A8100085960E94DE9AC8010E94DE9A80910E13EE
:10A8200090910F13892BA1F070E060E08AE093E132
:10A830000E94B699082E000C990BC0970A9740F415
:10A840008AE093E10E94DB98CB010E9464254DCD04
:10A8500010E02FCECF92DF92EF92FF92CF93C09174
:10A860007E11C4304CF4C1300CF04BC0CC2359F1F4
:10A8700060E070E0CB013FC0C430D1F70E943618D1
:10A8800020E030E040EA50E40E9410B820E030ECD4
:10A890004FE754E40E9429BA20E030E040EA50E457
:10A8A0000E9429BA20E030E040E851E40E9410B84C
:10A8B00020E030E040E850E40E944BB920E030E076
:10A8C0004AE754E416C00E94361820E030E040EA1F
:10A8D00050E40E9410B820E030EC4FE754E40E94AE
:10A8E00029BA20917F1130918011409181115091AE
:10A8F00082110E9429BACF91FF90EF90DF90CF9004
:10A9000008950E9436182AE137E64CE950E40E9487
:10A9100010B820917F113091801140918111509198
:10A9200082110E944AB96B017C01EC2FEE0FFF0BE4
:10A93000E55AFA4F60817181072E000C880B990B44
:10A940000E94B1B79B01AC01C701B601D2CF809183
:10A950008504882349F08091E504882329F060E08C
:10A9600083EF93E10C949E1308958F929F92AF9280
:10A97000BF92CF92DF92EF92FF920F931F93CF93EC
:10A98000DF938C01862F0B30110509F092C0909156
:10A990005313992309F0F89462E10E9417A8EC017F
:10A9A00080915313882309F07894209701F180E077
:10A9B00090ECA9E7B4EC8093461390934713A093CF
:10A9C0004813B093491380934A1390934B13A09369
:10A9D0004C13B0934D13CE3F8FEFD80709F49DC0B1
:10A9E000CF3FDC0709F4EBC1CCEFDFEF24C1C0910E
:10A9F0004E13E0904F136E2D70E090E080E00E94C7
:10AA0000B1B72DEC3CEC4CEC5DE30E9410B84B016F
:10AA10005C016C2F70E090E080E00E94B1B79B0178
:10AA2000AC01C501B4010E944BB960934613709309
:10AA300047138093481390934913D0915013F0908B
:10AA400051136D2F6F7770E090E080E00E94B1B7F6
:10AA50004B015C016F2D70E090E080E00E94B1B787
:10AA60002DEC3CEC4CEC5DE30E9410B89B01AC017A
:10AA7000C501B4010E944BB9D7FD19C060934A13B8
:10AA800070934B1380934C1390934D13CE0DCD0FB9
:10AA9000CF0D81E090E020915213C21302C090E0EC
:10AAA00080E0892B09F487C0CFEFDFEF88C1905891
:10AAB000E5CFCFEFDFEF0631110509F0BCC0909173
:10AAC0005313992309F0F89461E00E9417A8EC0150
:10AAD00080915313882309F07894209709F180E03E
:10AAE00090ECA9E7B4EC8093461390934713A0939E
:10AAF0004813B093491380934A1390934B13A09338
:10AB00004C13B0934D13CF3FDC0709F458C1209785
:10AB100009F451C0229609F067CFCEEFDFEF8BC06A
:10AB2000C0914F13D0914E1360914E1370914F13FB
:10AB300076276727762790E080E00E94AFB72DEC5C
:10AB40003CEC4CEC5DE30E9410B8609346137093AC
:10AB500047138093481390934913E0905113F0905A
:10AB600050136F2D6F77762F6E2D90E080E00E944E
:10AB7000AFB72DEC3CEC4CEC5DE30E9410B8F7FC59
:10AB800018C060934A1370934B1380934C139093A7
:10AB90004D138C2F8D0F8E0D8F0DC1E0D0E0909155
:10ABA0005213891302C0D0E0C0E0D195C195D109FC
:10ABB000AACF9058E6CFC0904613D0904713E090AC
:10ABC0004813F090491320E030E048EC52E4C7010C
:10ABD000B6010E9432BBD0E0C0E0181614F4CBEFEF
:10ABE000DFEF20E030E0A901C701B6010E94AAB75B
:10ABF00087FF02C0CAEFDFEFC0904A13D0904B131B
:10AC0000E0904C13F0904D1320E030E048EC52EC13
:10AC1000C701B6010E94AAB787FF02C0C9EFDFEFE4
:10AC200020E030E040EF52E4C701B6010E9432BBA1
:10AC300018160CF4BFC00C30110509F0C0C08CE52B
:10AC40000E94DB8D90E080E00E94D68D0E94FCA2E5
:10AC500065E08CE50E9414A310925B0D80935A0D61
:10AC6000C82FD0E0209709F4A8C0C530D1050CF456
:10AC7000B6C005E11CE00E941491F80180870F5FC7
:10AC80001F4FC80185519C408C179D07A4F3C091AC
:10AC90001D0C00911E0C602F70E090E080E00E947F
:10ACA000B1B72DEC3CEC4CEC5DE30E9410B86B01AD
:10ACB0007C016C2F70E090E080E00E94B1B79B01B6
:10ACC000AC01C701B6010E944BB96B017C01C09277
:10ACD000150CD092160CE092170CF092180CD09133
:10ACE0001F0C1091200C6D2F6F7770E090E080E0CA
:10ACF0000E94B1B74B015C01612F70E090E080E0F1
:10AD00000E94B1B72DEC3CEC4CEC5DE30E9410B816
:10AD10009B01AC01C501B4010E944BB9D7FD5DC0D8
:10AD20006093190C70931A0C80931B0C90931C0C5D
:10AD3000C00FCD0FC10F8091210CC813B5CE20E0FC
:10AD400030E048EC52E4C701B6010E9432BBD0E0CB
:10AD5000C0E0181614F4CBEFDFEF20E030E040EA5B
:10AD600050E4C701B6010E94AAB787FF02C0CAEF2C
:10AD7000DFEFC090190CD0901A0CE0901B0CF090F3
:10AD80001C0C20E030E040EF51ECC701B6010E94FE
:10AD9000AAB787FF02C0C9EFDFEF20E030E040EF45
:10ADA00052E4C701B6010E9432BB181644F4C8EF42
:10ADB000DFEF05C0C8EFDFEF3ECFCEEFDFEFCE0114
:10ADC000DF91CF911F910F91FF90EF90DF90CF9087
:10ADD000BF90AF909F908F9008959058A1CFCDEFE6
:10ADE000DFEFEDCFCF93DF93FC0124813581232B5F
:10ADF00099F0EC01BC018DEF9DE00E94A39D6EE1F6
:10AE000070E080E090E00E9439A5BE0184ED9FE0F3
:10AE1000DF91CF910C94A39DDF91CF910895CF93B3
:10AE2000DF93FC0124813581232B69F0EC01BC0107
:10AE300084ED9FE00E94959DBE018DEF9DE0DF9126
:10AE4000CF910C94959DDF91CF91089580918504C9
:10AE50008823F9F08091E5048823D9F081E00E94ED
:10AE6000E58D8BE39FE10197F1F760E080E00E94C0
:10AE7000F68D65E07DE083EF93E10E94B59D61E092
:10AE800080E00E94F68D65EF7CE083EF93E10C9407
:10AE9000B59D0895CF93DF93209185042223A9F0D7
:10AEA0002091E504222389F0EC016FED83EF93E11B
:10AEB0000E941A9C8C819D81892B39F0BE0183EF01
:10AEC00093E1DF91CF910C94959DDF91CF910895FF
:10AED000EF92FF920F931F93CF93DF9320918504FE
:10AEE000222309F461C02091E504222309F45CC007
:10AEF0008A01EB017C01209719F1C095D09561E0A2
:10AF00008C2F0E94F68DB70183EF93E10E94959DEF
:10AF100064EE7CE083EF93E10E94B59DF7018481AC
:10AF200061E08C0F0E94F68DB801110F880B990B10
:10AF3000DF91CF911F910F91FF90EF900C9439A565
:10AF40000E94F80FAB01BC018091E40C9091E50CDC
:10AF5000A091E60CB091E70C8C599F4FAF4FBF4FBB
:10AF600084179507A607B707F8F461E080E00E9410
:10AF7000F68DB70183EF93E10E94959D63ED7CE030
:10AF800083EF93E10E94B59D61E0F70184810E9407
:10AF9000F68D0E94F80F6093E40C7093E50C80939B
:10AFA000E60C9093E70CC0CFDF91CF911F910F91EA
:10AFB000FF90EF900895FF920F931F93CF93DF932D
:10AFC000EC01F62E08811981C8010E94D1B8F8164B
:10AFD00021F06F2DC8010E94D9B8CE01DF91CF9129
:10AFE0001F910F91FF900895CF93DF93EC019A0189
:10AFF000AB01E889F98982E08083211581EE380769
:10B000004105510581F160E079E08DE390E00E9417
:10B0100019B921503109410951095695479537957C
:10B020002795EC85FD851082EE85FF852083188E9F
:10B03000EC89FD8986E08083EA89FB8980818061D3
:10B040008083EA89FB89808188608083EA89FB8923
:10B05000808180688083EA89FB8980818F7D8083FD
:10B06000DF91CF910895E889F989108220E1D9CF45
:10B07000CF93DF93EC01FB01248135810E945B9B20
:10B08000CE01DF91CF910895CF93DF93EC0148304B
:10B0900085E058076105710509F448C008F099C0BA
:10B0A000493481E058076105710509F4B2C008F020
:10B0B00040C0443481E058076105710509F476C049
:10B0C00000F5413481E058076105710509F456C067
:10B0D00048F4403451406105710509F4E4C06BEF58
:10B0E0007BE0E3C0423481E058076105710509F453
:10B0F00009C1433451406105710589F764E17AE083
:10B10000D4C0463481E058076105710509F40CC1CB
:10B1100008F49FC0473481E058076105710509F4C0
:10B1200055C04834514061057105C9F667E77AE0BA
:10B13000BCC0423085E058076105710509F4E2C0E2
:10B1400000F5443781E058076105710509F4F2C044
:10B1500040F4423751406105710509F665E17BE035
:10B16000A4C0411585E058076105710509F49BC02D
:10B17000413055406105710509F0B1CF6AE17AE0CF
:10B1800094C0453085E058076105710509F461C038
:10B1900080F4433085E058076105710509F4AECFAE
:10B1A000443055406105710509F099CF61E17AE0BD
:10B1B0007CC0463085E058076105710509F4B4C0CC
:10B1C000473055406105710509F089CF65E77AE0A0
:10B1D0006CC04D3B82E458078FEF6807710509F496
:10B1E000AFC008F048C04F3E80E158078FEF6807B6
:10B1F000710561F3F8F4423385E058076105710584
:10B2000009F4ACCF48F4493055406105710509F0A7
:10B2100066CF69E77AE049C0443385E058076105A5
:10B22000710509F487C04D3F52406F4F710509F415
:10B2300095CF55CF4D3D82E258078FEF68077105D6
:10B2400009F478C048F4473E58416F4F710509F042
:10B2500046CF6EE07AE029C04F3C80E358078FEF7D
:10B260006807710509F4A2CF473C58436F4F710539
:10B2700009F45CCF34CF473988E658078FEF680769
:10B28000710509F47BCF48F54D3A82E558078FEFF9
:10B290006807710509F451C078F4453B5A446F4F73
:10B2A000710509F01CCF62E077E0CE010E944A9B55
:10B2B000CE01DF91CF910895453A8AE558078FEF87
:10B2C0006807710509F4A5CF4D3952466F4F7105D6
:10B2D00009F005CF6BEA77E0E8CF473588EA5807F1
:10B2E0008FEF6807710519F180F445388AE7580730
:10B2F0008FEF68077105C1F0473658496F4F7105E8
:10B3000009F0EDCE67E17AE0D0CF4F3480EB5807FB
:10B310008FEF6807710509F4F1CE4D33524C6F4F32
:10B32000710509F41BCFDBCE63E77AE0BECF6AE795
:10B3300078E0BBCF61EA7BE0B8CF60EC75E0B5CFD9
:10B3400061E27BE0B2CF0F931F93CF93DF9300D0E6
:10B3500000D0CDB7DEB72091310D2223A9F08C01AA
:10B3600060EC75E0CE0101960E944A9BB801CE01C7
:10B3700001960E94F899BC0184ED9FE00E94A39D74
:10B38000CE0101960E94DE9A26960FB6F894DEBF93
:10B390000FBECDBFDF91CF911F910F910895AF9256
:10B3A000BF92CF92DF92EF92FF920F931F93CF93B2
:10B3B000DF93CDB7DEB762970FB6F894DEBF0FBE4E
:10B3C000CDBF20918504222309F447C02091E504D4
:10B3D000222309F442C07A016B015C010E94F80F3C
:10B3E000AB01BC018091E00C9091E10CA091E20CCA
:10B3F000B091E30C8C599F4FAF4FBF4F8417950707
:10B40000A607B70750F560E08FEFC816D806B1F56C
:10B4100080E00E94F68D00E0B50183EF93E10E9489
:10B42000959D62EC7CE083EF93E10E94B59DF50170
:10B43000848160E0800F0E94F68D0E94F80F609377
:10B44000E00C7093E10C8093E20C9093E30CB70155
:10B45000FF0C880B990B0E9439A562960FB6F894E1
:10B46000DEBF0FBECDBFDF91CF911F910F91FF9037
:10B47000EF90DF90CF90BF90AF90089580E00E9452
:10B48000F68D0E94F80F28EE33E040E050E00E9475
:10B49000E7B8CA01B90120E831E541E050E00E9477
:10B4A000E7B8AB01BC01CE0101960E946898BE01CD
:10B4B0006F5F7F4FCE0107960E94419B65E979E05F
:10B4C000CE0107960E94E299BC01CE010D960E9422
:10B4D000419BCE0107960E94DE9ACE0101960E9402
:10B4E000DE9ABE01635F7F4F83EF93E10E94959DDB
:10B4F00009891A89C114D10431F00C0D1D1D60E0B9
:10B50000802F0E94F68DCE010D960E94DE9A84CF88
:10B51000BF92CF92DF92EF92FF920F931F93CF9340
:10B52000DF93CDB7DEB762970FB6F894DEBF0FBEDC
:10B53000CDBF6C018B017A0180918504882369F16C
:10B540008091E504882349F177FF37C00095109575
:10B5500060E0802F0E94F68DB60183EF93E10E9498
:10B56000959D61EB7CE083EF93E10E94B59DF60130
:10B57000848160E0800F0E94F68D0E94F80F609336
:10B58000E00C7093E10C8093E20C9093E30CB70114
:10B59000FF0C880B990B0E9439A562960FB6F894A0
:10B5A000DEBF0FBECDBFDF91CF911F910F91FF90F6
:10B5B000EF90DF90CF90BF90089560E080E00E9410
:10B5C000F68D0E94F80F28EE33E040E050E00E9434
:10B5D000E7B8CA01B90120E831E541E050E00E9436
:10B5E000E7B8AB01BC01CE0101960E946898BE018C
:10B5F0006F5F7F4FCE0107960E94419B65E979E01E
:10B60000CE0107960E94E299BC01CE010D960E94E0
:10B61000419BCE0107960E94DE9ACE0101960E94C0
:10B62000DE9ABE01635F7F4F83EF93E10E94959D99
:10B63000B98860E08B2D0E94F68D0115110531F45B
:10B640000B2DCE010D960E94DE9A86CF60E0802FF2
:10B650000E94F68DF6CFAF92BF92CF92DF92EF921B
:10B66000FF920F931F93CF93DF93CDB7DEB72C9745
:10B670000FB6F894DEBF0FBECDBF8091300D8111A3
:10B6800002C00E94265780919104909192040297E3
:10B6900051F080912C0C90912D0C009709F4B4C1BD
:10B6A000039709F4B1C162E875E186EE92E10E9468
:10B6B000699A66EE72E1CE0101960E94419B44E1D7
:10B6C00050E070E060E0CE0101960E94885ACE0101
:10B6D00001960E94DE9A63E775E186EE92E10E9490
:10B6E000699A66EE72E1CE0101960E94419B44E1A7
:10B6F00050E06FEF7FEFCE0101960E946857CE01B8
:10B7000001960E94DE9A87E00E9414A58C0186E0D3
:10B710000E9414A5BC0190E080E00E94AFB72AE02F
:10B7200037ED43EA5CE30E9410B823E333E948E8CD
:10B7300053E40E944AB96B017C0184E0A82EB12C2D
:10B7400020E030E048EC52E4C701B6010E9432BB71
:10B7500018160CF05FC081E0A81AB108E9F064E6A1
:10B7600070E080E090E00E9439A586E00E9414A578
:10B77000BC0190E080E00E94AFB72AE037ED43EAD9
:10B780005CE30E9410B823E333E948E853E40E94E5
:10B790004AB96B017C01D4CF68E675E186EE92E18F
:10B7A0000E94699A66EE72E1CE0101960E94419B69
:10B7B0004AE050E070E060E0CE0101960E94885AB5
:10B7C000CE0101960E94DE9A6BE77AE0CE010196E7
:10B7D0000E944A9B66EE72E1CE0101960E94F899A2
:10B7E000BC018CEE92E10E948E9ACE0101960E94DD
:10B7F000DE9A80912C0C90912D0C049721F41092DC
:10B800002D0C10922C0C81E090E090939204809388
:10B810009104D9C0B80190E080E00E94AFB72AE05F
:10B8200037ED43EA5CE30E9410B823E333E948E8CC
:10B8300053E40E944AB9AB01BC0121E0CE0101965C
:10B840000E94E69A6DE87AE0CE0107960E944A9B34
:10B85000BE016F5F7F4FCE0107960E94F899BC0131
:10B860008CEE92E10E948E9ACE0107960E94DE9A9B
:10B87000CE0101960E94DE9A6CEE72E1CE01019635
:10B880000E94419B42E350E06FEF7FEFCE010196B3
:10B890000E946857CE0101960E94DE9A6BEA77E01B
:10B8A000CE0101960E944A9BCE0101960E944A5702
:10B8B000CE0101960E94DE9A6AEA77E08CEE92E170
:10B8C0000E94589A21E0B701A601CE0101960E947C
:10B8D000E69A62EE76E0CE0107960E944A9BBE0190
:10B8E0006F5F7F4FCE0107960E94F899BC0182EFEF
:10B8F00092E10E948E9ACE0107960E94DE9ACE01B6
:10B9000001960E94DE9A61E67AE0CE0101960E94DD
:10B910004A9B62EF72E1CE0101960E94F899BC0148
:10B9200086EE92E10E948E9ACE0101960E94DE9AE6
:10B9300066EE72E1CE0101960E94419B4AE050E022
:10B9400070E060E0CE0101960E94CF59CE010196D1
:10B950000E94DE9A6BEA77E0CE0101960E944A9B34
:10B96000CE0101960E944A57CE0101960E94DE9AAE
:10B970006AEA77E082EF92E10E94589A62EF72E100
:10B98000CE0101960E94419B61E67AE0CE010196CC
:10B990000E94E2996CEE72E10E94F899BC018CEE73
:10B9A00092E10E948E9ACE0101960E94DE9A8091C9
:10B9B0002C0C90912D0C039731F484E090E090933F
:10B9C0002D0C80932C0C64E670E080E090E00E94E7
:10B9D00039A58091300D882331F060E273E080E07A
:10B9E00090E00E9439A52C960FB6F894DEBF0FBEEA
:10B9F000CDBFDF91CF911F910F91FF90EF90DF901E
:10BA0000CF90BF90AF9008958AE99EE00E94F69093
:10BA100064E670E080E090E00E9439A568EA75E194
:10BA200086EE92E10E94699A66EE72E1CE0101967D
:10BA30000E94419B44E150E070E060E0CE0101963D
:10BA40000E94885ACE0101960E94DE9A69E975E14A
:10BA500086EE92E10E94699A66EE72E1CE0101964D
:10BA60000E94419B44E150E06FEF7FEFCE010196D1
:10BA70000E946857CE0101960E94DE9A8CE40E94D3
:10BA8000809F6B017C0104E010E0A7019601C701D3
:10BA9000B6010E9497BC882309F449C001501109DE
:10BAA00061F068EC70E080E090E00E9439A58CE4E1
:10BAB0000E94809F6B017C01E8CF6EE875E186EE05
:10BAC00092E10E94699A66EE72E1CE0101960E94AF
:10BAD000419B4AE050E070E060E0CE0101960E9498
:10BAE000885ACE0101960E94DE9A6BE77AE0CE0179
:10BAF00001960E944A9B66EE72E1CE0101960E9479
:10BB0000F899BC018CEE92E10E948E9ACE010196CA
:10BB10000E94DE9A80912C0C90912D0C039721F4B9
:10BB200010922D0C10922C0C82E090E06ECE21E051
:10BB3000B701A601CE0107960E94E69A6DE87AE069
:10BB4000CE0101960E944A9BBE01695F7F4FCE01E4
:10BB500001960E94F899BC018CEE92E10E948E9AA7
:10BB6000CE0101960E94DE9ACE0107960E94DE9ACF
:10BB70006CEE72E1CE0101960E94419B42E350E0DF
:10BB80006FEF7FEFCE0101960E946857CE010196BC
:10BB90000E94DE9A6BEA77E0CE0101960E944A9BF2
:10BBA000CE0101960E944A57CE0101960E94DE9A6C
:10BBB0006AEA77E08CEE92E10E94589A86E60E944B
:10BBC000809F6B017C0104E010E0A7019601C70192
:10BBD000B6010E9497BC882381F00150110909F435
:10BBE00084C068EC70E080E090E00E9439A586E6B1
:10BBF0000E94809F6B017C01E8CF21E0B701A60184
:10BC0000CE0107960E94E69A62EE76E0CE0101969A
:10BC10000E944A9BBE01695F7F4FCE0101960E9440
:10BC2000F899BC0182EF92E10E948E9ACE010196B2
:10BC30000E94DE9ACE0107960E94DE9A61E67AE0C3
:10BC4000CE0101960E944A9B62EF72E1CE010196FD
:10BC50000E94F899BC0186EE92E10E948E9ACE0174
:10BC600001960E94DE9A66EE72E1CE0101960E9474
:10BC7000419B4AE050E06FEF7FEFCE0101960E94BA
:10BC8000CF59CE0101960E94DE9A6BEA77E0CE0191
:10BC900001960E944A9BCE0101960E944A57CE010E
:10BCA00001960E94DE9A6AEA77E082EF92E10E94B2
:10BCB000589A62EF72E1CE0101960E94419B61E6C3
:10BCC0007AE0CE0101960E94E2996CEE72E10E9448
:10BCD000F899BC018CEE92E10E948E9ACE010196F9
:10BCE0000E94DE9A83E090E06ACE6BEF7BE082EF09
:10BCF00092E10E945E98DDCF4F925F926F927F92A9
:10BD00008F929F92AF92BF92CF92DF92EF92FF926B
:10BD1000CF93DF93CDB7DEB72C970FB6F894DEBF85
:10BD20000FBECDBF0E9426570E94D9A52B013C0112
:10BD30000E9484A54B015C016091C5047091C6040A
:10BD40008091C7049091C8040E94B1B76B017C0137
:10BD50000E94D9A50E94B1B7A70196010E9429BAF5
:10BD600021E03EED42E45EE30E94FDBB9B01AC019D
:10BD700060E070E080E89FE30E944AB920E03AE288
:10BD80004DE257E40E9410B86B017C01C301B2017F
:10BD90000E94B1B720E030E048EC52E40E9429BA9A
:10BDA000AB01BC0122E0CE0101960E94E69ABE01E1
:10BDB0006F5F7F4F80EE92E10E94A59ACE010196BF
:10BDC0000E94DE9A63EF75E080EE92E10E94589A3D
:10BDD00060EE72E186EE92E10E948E9A6FEE75E05F
:10BDE000CE0101960E944A9B60EE72E1CE0101965F
:10BDF0000E94F899BC0180EE92E10E948E9ACE01D9
:10BE000001960E94DE9A62EE76E08CEE92E10E944C
:10BE10005E9821E0B501A401CE0101960E94E69A48
:10BE2000BE016F5F7F4F8CEE92E10E94629ACE015D
:10BE300001960E94DE9A66E97AE08CEE92E10E9419
:10BE4000589A21E0B701A601CE0101960E94E69A18
:10BE5000BE016F5F7F4FCE0107960E94419B68E550
:10BE60007BE0CE0107960E94E299BC018CEE92E144
:10BE70000E94629ACE0107960E94DE9ACE01019638
:10BE80000E94DE9A60EE72E1CE0101960E94419B13
:10BE900061E67AE0CE0101960E94E2996CEE72E1D1
:10BEA0000E94F899BC018CEE92E10E948E9ACE011C
:10BEB00001960E94DE9A21E0B501A401CE0101960F
:10BEC0000E94E69ABE016F5F7F4F82EF92E10E946F
:10BED000A59ACE0101960E94DE9A62EF72E1CE0130
:10BEE00001960E94419B4AE050E070E060E0CE0184
:10BEF00001960E94885ACE0101960E94DE9A65E062
:10BF000070E080E090E00E9439A56BEA77E0CE0116
:10BF100001960E944A9BCE0101960E944A57CE018B
:10BF200001960E94DE9A66EE72E1CE0101960E94B1
:10BF3000419B4AE050E06FEF7FEFCE0101960E94F7
:10BF40006857CE0101960E94DE9A20E0B701A60153
:10BF5000CE0101960E94E69ABE016F5F7F4FCE012F
:10BF600007960E94419B68E57BE0CE0107960E9400
:10BF7000E299BC0182EF92E10E948E9ACE0107966F
:10BF80000E94DE9ACE0101960E94DE9A62EF72E173
:10BF9000CE0101960E94419B4AE050E064EF7FEFA2
:10BFA000CE0101960E946857CE0101960E94DE9A4A
:10BFB00065E070E080E090E00E9439A58091300D4E
:10BFC000882331F068E572E080E090E00E9439A5B6
:10BFD0002C960FB6F894DEBF0FBECDBFDF91CF9188
:10BFE000FF90EF90DF90CF90BF90AF909F908F9099
:10BFF0007F906F905F904F9008954F925F926F92F5
:10C000007F928F929F92AF92BF92CF92DF92EF92E8
:10C01000FF920F931F93CF93DF93CDB7DEB7CA5430
:10C02000D1090FB6F894DEBF0FBECDBF8C016BEF08
:10C030007BE0CE01C7960E944A9B6BEF7BE0CE016E
:10C04000CD960E944A9BBE016F5F7F4F87E293E1CE
:10C050000E94D90CCD88DE88EF88F88C20E030E093
:10C0600040E251E4C701B6010E9410B82B013C0127
:10C07000898D9A8DAB8DBC8D2B968CAF9DAFAEAF5D
:10C08000BFAF2B9720E030E040E251E4BC01CD018E
:10C090000E9410B84B015C0120E030E040E251E426
:10C0A0006D8D7E8D8F8D98A10E9410B827966CAFF4
:10C0B0007DAF8EAF9FAF2797C701B60190582B96E3
:10C0C0002CAD3DAD4EAD5FAD2B970E94CAB92BEDA7
:10C0D0003FE049EC5FE30E944BB92091C1043091ED
:10C0E000C2044091C3045091C4040E944BB96B0137
:10C0F0007C0120E030E0A9010E94AAB787FDCFC2F1
:10C10000C092DC0CD092DD0CE092DE0CF092DF0CE1
:10C11000C090DC0CD090DD0CE090DE0CF090DF0CD9
:10C120002BED3FE049EC50E4C701B6010E9432BB61
:10C13000181684F42BED3FE049EC50E4C701B6013A
:10C140000E944AB96093DC0C7093DD0C8093DE0C86
:10C150009093DF0C20E030E044E353E46091DC0C8A
:10C160007091DD0C8091DE0C9091DF0C0E9410B874
:10C170002BED3FE049E450E40E9429BA6093D80CCB
:10C180007093D90C8093DA0C9093DB0C0E94D5BA93
:10C19000CE018B960E9495986CE97AE0CE01859647
:10C1A0000E944A9BBE01655D7F4FCE0185960E942D
:10C1B000F89966EA7AE00E94E299BC0182EF92E186
:10C1C0000E948E9ACE0185960E94DE9ACE018B96B1
:10C1D0000E94DE9AC090D80CD090D90CE090DA0C76
:10C1E000F090DB0C20E030E044EB52E4C701B601F4
:10C1F0000E94AAB718160CF463C220E030E040E0B9
:10C200005FE3C701B6010E944BB90E94D5BACE01C7
:10C210008B960E9495986DEA7AE0CE0185960E94F1
:10C220004A9BBE01655D7F4FCE0185960E94F899BD
:10C23000BC01CE01C7960E948E9ACE0185960E94BF
:10C24000DE9ACE018B960E94DE9A61EC79E0CE01F7
:10C25000CD960E945E98BE01695C7F4FCE018596A7
:10C260000E94419B4AE050E070E060E0CE0185967C
:10C270000E94885ACE0185960E94DE9A0E94F80F8D
:10C28000AB01BC018091E00C9091E10CA091E20C1B
:10C29000B091E30C8C599F4FAF4FBF4F8417950758
:10C2A000A607B70708F091C26BEF7BE0CE01859639
:10C2B0000E944A9BCE0185960E944A57CE018596E0
:10C2C0000E94DE9ABE01635C7F4F83EF93E10E9480
:10C2D000959D61E67AE0CE0185960E944A9BBE015B
:10C2E000635C7F4FCE0185960E94F899BC01CE0118
:10C2F000C7960E94629ACE0185960E94DE9A0E949D
:10C30000F80FC090320DD090330DE090340DF090C6
:10C31000350D6C197D098E099F090E94AFB720E089
:10C3200030E04AE754E40E9429BAAB01BC0123E0A3
:10C33000CE018B960E94E69A6EEB7AE0CE0185964E
:10C340000E944A9BBE01655D7F4FCE0185960E948B
:10C35000F89965E979E00E94E299BC0180EE92E1EA
:10C360000E948E9ACE0185960E94DE9ACE018B960F
:10C370000E94DE9A60EE72E1CE0185960E94419B9A
:10C3800062EF72E1CE0185960E94F899BE01695C68
:10C390007F4F0E94F899BC01CE01C7960E948E9AE9
:10C3A000CE0185960E94DE9A66EA7CE08CEE92E1F0
:10C3B0000E94699A21E0B301A201CE0185960E94F4
:10C3C000E69ABE016B5D7F4F8CEE92E10E94629A0D
:10C3D000CE0185960E94DE9A21E027964CAD5DAD98
:10C3E0006EAD7FAD2797CE01C1960E94E69A21E0FF
:10C3F000B501A401CE018B960E94E69A61E67AE02F
:10C40000CE0185960E944A9BBE01655D7F4FCE019D
:10C4100085960E94F89961E67AE00E94E299BE0151
:10C420006F5C7F4F0E94F89965EB7AE00E94E29979
:10C43000BC018CEE92E10E94629ACE0185960E9428
:10C44000DE9ACE018B960E94DE9ACE01C1960E94A2
:10C45000DE9AA3019201C301B2010E9410B86B01E0
:10C460007C01A5019401C501B4010E9410B89B0193
:10C47000AC01C701B6010E944BB96B017C01279644
:10C480002CAD3DAD4EAD5FAD2797CA01B9010E94FD
:10C4900010B89B01AC01C701B6010E944BB90E94C4
:10C4A00053BC6093D40C7093D50C8093D60C9093AE
:10C4B000D70C69EB7AE08CEE92E10E94589A409199
:10C4C000D40C5091D50C6091D60C7091D70C21E012
:10C4D000CE0185960E94E69ABE016B5D7F4FCE012C
:10C4E0008B960E94419B65EF7AE0CE018B960E946D
:10C4F000E299BC0182EF92E10E948E9ACE018B9666
:10C500000E94DE9ACE0185960E94DE9A62EF72E169
:10C510008CEE92E10E94629AC090D40CD090D50C1F
:10C52000E090D60CF090D70C20E030E04AE754E4DD
:10C53000C701B6010E9432BB87FD29C020E030E070
:10C540004AE754E4C701B6010E9429BAAB01BC0115
:10C5500023E0CE0185960E94E69ABE016B5D7F4F77
:10C56000CE018B960E94419B66EF7AE0CE018B96BE
:10C570000E94E299BC0182EF92E10E948E9ACE0164
:10C580008B960E94DE9ACE0185960E94DE9A20E06C
:10C5900030E64AE656E46091D40C7091D50C809157
:10C5A000D60C9091D70C0E94AAB7BE01695C7F4F50
:10C5B00087FF2AC1CE0185960E94419B6DEB7AE0F0
:10C5C000CE0185960E94E2996CEE72E10E94F89984
:10C5D000BC018CEE92E10E948E9ACE0185960E945B
:10C5E000DE9A03301105A1F46CEE72E1CE0185965E
:10C5F0000E94419BCE0185960E94F256CE018596FF
:10C600000E94DE9A6BEF7BE08CEE92E10E945E98D6
:10C6100060EC7AE0CE0185960E944A9B62EF72E15F
:10C62000CE0185960E94F899BC01CE018B960E949E
:10C63000419B4AE050E06FEF7FEFCE018B960E9466
:10C640006857CE018B960E94DE9ACE0185960E9495
:10C65000DE9A6AE070E080E090E00E9439A5CE01A9
:10C66000CD960E94DE9ACE01C7960E94DE9AC65BE6
:10C67000DF4F0FB6F894DEBF0FBECDBFDF91CF9175
:10C680001F910F91FF90EF90DF90CF90BF90AF90F0
:10C690009F908F907F906F905F904F9008952BEDBB
:10C6A0003FE049EC50E4C701B6010E944BB96093EA
:10C6B000DC0C7093DD0C8093DE0C9093DF0C28CDA6
:10C6C00020E030E044E353E4C701B6010E94AAB77A
:10C6D0001816CCF0A701960160E070E884E393E4BB
:10C6E0000E944AB96093D80C7093D90C8093DA0CED
:10C6F0009093DB0C0E94D5BACE018B960E94959840
:10C7000060EB7AE08ACD20E030E047E853E4C701EF
:10C71000B6010E94AAB71816CCF120E030E044E33D
:10C7200053E4C701B6010E944AB920E030E040E07E
:10C730005FE30E944BB96093D80C7093D90C80933F
:10C74000DA0C9093DB0C0E94D5BACE018B960E9436
:10C75000959860EB7AE0CE0185960E944A9BBE01D7
:10C76000655D7F4FCE0185960E94F899BC01CE0190
:10C77000C7960E948E9ACE0185960E94DE9ACE01BF
:10C780008B960E94DE9A63EB7AE061CDA701960159
:10C7900060E070E084EB93E40E944AB920E030E06E
:10C7A00040E05FE30E944BB96093D80C7093D90CC2
:10C7B0008093DA0C9093DB0C0E94D5BACE018B9655
:10C7C0000E9495986DEA7AE0C6CF0E94F80F0E9409
:10C7D000AFB76B017C016091E00C7091E10C80912E
:10C7E000E20C9091E30C0E94B1B720E030E048ECFD
:10C7F00051E40E944BB99B01AC01C701B6010E94F4
:10C80000AAB787FD51CD65CD8CEE92E10E948E9A3C
:10C8100020CF2F923F924F925F926F927F928F9292
:10C820009F92AF92BF92CF92DF92EF92FF920F93BF
:10C830001F93CF93DF93CDB7DEB7C854D1090FB69E
:10C84000F894DEBF0FBECDBF2B013C012DA73EA744
:10C850004FA758AB28EE421623E05206610471043C
:10C8600034F030E9432E55245394612C712CCDA41F
:10C87000DEA4EFA4F8A820E1C21627E2D206E10464
:10C88000F10454F020E1C22E27E2D22EE12CF12C4B
:10C89000CDA6DEA6EFA6F8AA8091300D882341F040
:10C8A000C12CD12C7601C394CDA6DEA6EFA6F8AAA2
:10C8B0000E94F80F25966CAF7DAF8EAF9FAF259786
:10C8C0000E94F80F6DAB7EAB8FAB98AF25966CAD29
:10C8D0007DAD8EAD9FAD259728EE33E040E050E072
:10C8E0000E94E7B829962CAF3DAF4EAF5FAF2997B6
:10C8F00021E02DA319A61AA61BA61CA68E01035F74
:10C900001F4FCC24DD247601C418D508E608F708AB
:10C91000C9AADAAAEBAAFCAA6DA97EA98FA998AD2B
:10C920002596CCACDDACEEACFFAC25976C197D093F
:10C930008E099F09CDA4DEA4EFA4F8A86C157D058F
:10C940008E059F050CF0B6C30E94B1B720E030E021
:10C950004AE754E40E9429BAAB01BC0123E0C801B4
:10C960000E94E69AB80186EE92E10E94A59AC8015B
:10C970000E94DE9AA70196012A3031054105510532
:10C980008CF429964CAD5DAD6EAD7FAD2997C80195
:10C990000E946898B80186EE92E10E94A59AC801AB
:10C9A0000E94DE9A8091300D6EEB7AE0882309F4C4
:10C9B0006EC286EE92E10E945E98CE0101960E94C0
:10C9C000ABA46BEF7BE08CEE92E10E945E98AE012F
:10C9D0004F5F5F4F1A01812C912C5401D101CD90F2
:10C9E000DD90ED90FD901D01A7019601C701B601F4
:10C9F0000E9410B89B01AC01C501B4010E944BB963
:10CA00004B015C0123E0B701A601C8010E94E69A30
:10CA1000B801CE0143960E94419B61E67AE0CE01C7
:10CA200043960E94E299BC018CEE92E10E94629AC8
:10CA3000CE0143960E94DE9AC8010E94DE9A20161B
:10CA4000310661F6C501B4010E9453BC4B015C0183
:10CA5000BDE24B16B1E05B066104710434F00E9444
:10CA6000265760E080E00E94F68D23E0B501A40126
:10CA7000CE0143960E94E69A6AEF7BE0C8010E94CD
:10CA80004A9B66EE72E1C8010E94F89969EC7AE06F
:10CA90000E94E299BE016D5E7F4F0E94F8996DEC95
:10CAA0007AE00E94E299BC018CEE92E10E94629AC7
:10CAB000C8010E94DE9ACE0143960E94DE9A2AE9BE
:10CAC00039E949E55FE3C501B4010E9432BB18169C
:10CAD0000CF0F2C123E333E343E95FE3C501B401A2
:10CAE0000E94AAB7880F880BCDA0C822CDA2809142
:10CAF0002E0C90912F0C8130910509F4F2C1029710
:10CB000021F0DDA0DD2009F4ECC189849A84AB8496
:10CB1000BC84C980DA80EB80FC80CDA2DEA2EFA2CB
:10CB2000F8A6CD80DE80EF80F88420E030E0A90117
:10CB3000C501B4010E94AAB7882309F4BFC12DA181
:10CB40003EA14FA158A5CA01B9010E9410B869AF12
:10CB50007AAF8BAF9CAFA7019601C701B6010E94C7
:10CB600010B89B01AC0169AD7AAD8BAD9CAD0E9454
:10CB70004BB90E9453BCA50194010E94CAB920EE92
:10CB80003EE245E652E40E9410B869AF7AAF8BAF3F
:10CB90009CAF20E030E0A901C701B6010E94AAB70E
:10CBA000882309F490C12DA13EA14FA158A5CA0127
:10CBB000B9010E9410B821966CAF7DAF8EAF9FAFC8
:10CBC0002197A5019401C501B4010E9410B89B01F1
:10CBD000AC0121966CAD7DAD8EAD9FAD21970E94CD
:10CBE0004BB90E9453BCA70196010E94CAB920EE1E
:10CBF0003EE245E652E40E9410B821966CAF7DAF4C
:10CC00008EAF9FAF219720E030E0A9016DA17EA1FA
:10CC10008FA198A50E94AAB7882309F459C1A5013C
:10CC20009401C501B4010E9410B84B015C01A70139
:10CC30009601C701B6010E9410B89B01AC01C50165
:10CC4000B4010E944BB90E9453BC2DA13EA14FA13B
:10CC500058A50E94CAB96B017C0166EE72E1C80159
:10CC60000E94419B67ED71E1C8010E94F899BC01E7
:10CC70008CEE92E10E948E9AC8010E94DE9A6CEEC0
:10CC800072E1C8010E94419BC8010E940F57C80170
:10CC90000E94DE9A21E049AD5AAD6BAD7CADCE016C
:10CCA0004F960E94E69A21E021964CAD5DAD6EADA7
:10CCB0007FAD2197CE0149960E94E69A20EE3EE292
:10CCC00045E652E4C701B6010E9410B8AB01BC01B1
:10CCD00021E0C8010E94E69AB801CE0143960E9465
:10CCE000419B61E67AE0CE0143960E94E299BE0143
:10CCF000675E7F4F0E94F89961E67AE00E94E299B0
:10CD0000BE01615E7F4F0E94F899BC018CEE92E1FA
:10CD10000E948E9ACE0143960E94DE9AC8010E941C
:10CD2000DE9ACE0149960E94DE9ACE014F960E946D
:10CD3000DE9A6AE978E0C8010E944A9B6CEE72E1D3
:10CD4000C8010E94F899BC0180EE92E10E948E9A7F
:10CD5000C8010E94DE9A60EE72E1C8010E94419B08
:10CD6000C8010E946E19C8010E94DE9A6CEE72E141
:10CD700080EE92E10E948E9A6CEE72E1C8010E94F0
:10CD8000419BC8010E94F256C8010E94DE9A2DE222
:10CD9000421621E052066104710474F469A57AA573
:10CDA0008BA59CA525E030E040E050E00E94E7B86C
:10CDB000672B682B692BA9F56DE575E186EE92E18D
:10CDC0000E94699A60ED7AE0C8010E944A9B45E0A2
:10CDD00050E067EF7FEFC8010E94885AC8010E94A7
:10CDE000DE9A6BEF7BE0C8010E944A9BC8010E945B
:10CDF0004A57C8010E94DE9A6CEE72E1C8010E9497
:10CE0000419B45E050E070E060E0C8010E94685737
:10CE1000C8010E94DE9A6BEF7BE08CEE92E10E94EB
:10CE20005E98B201C30177FE04C069A97AA98BA9F3
:10CE30009CA90E9439A531E03DA30E94F80F6B0127
:10CE40007C012DA93EA94FA958ADC21AD30AE40A04
:10CE5000F50AC9A6DAA6EBA6FCA6C414D504E60416
:10CE6000F70444F4C301B2016C197D098E099F09CE
:10CE70000E9439A50E94F80F6DAB7EAB8FAB98AFC7
:10CE80006BEF7BE08CEE92E10E945E9845CDC8018D
:10CE90000E944A9B66EE72E1C8010E94F89965E91A
:10CEA00079E00E94E299BC0186EE92E10E948E9A9E
:10CEB000C8010E94DE9A81CD1DA219CE6BED7FE0E4
:10CEC00089EC9FE35CCE6BED7FE089EC9FE38FCE36
:10CED0008BEDC82E8FE0D82E89ECE82E8FE3F82E4C
:10CEE000BCCE67ED7AE0C8010E944A9B6CEE72E10D
:10CEF000C8010E94F899BC018CEE92E10E948E9AC2
:10CF0000C8010E94DE9A6CEE72E1C8010E94419B4A
:10CF1000C8010E94F256C8010E94DE9A6CEE72E1CE
:10CF2000C8010E94419BC8010E946E19C8010E945D
:10CF3000DE9A23E0B501A401CE0143960E94E69A51
:10CF40006AEC7AE0C8010E944A9BBE016D5E7F4F89
:10CF5000C8010E94F8996DEC7AE00E94E299BC0148
:10CF60008CEE92E10E948E9AC8010E94DE9ACE0158
:10CF700043960E94DE9A6CEE72E1C8010E94419BCA
:10CF8000C8010E946E19C8010E94DE9A66EE72E125
:10CF9000C8010E94419B6CEE72E1C8010E94F899A1
:10CFA000BC018CEE92E10E948E9AC8010E94DE9A2A
:10CFB00064EE7AE086EE92E10E94589A49855A859D
:10CFC0006B857C8522E0CE014F960E94E69A4D81CA
:10CFD0005E816F81788522E0CE0149960E94E69AB3
:10CFE00049815A816B817C8122E0C8010E94E69AC6
:10CFF000B801CE0143960E94419B61E67AE0CE01E2
:10D0000043960E94E299BE01675E7F4F0E94F899A5
:10D0100061E67AE00E94E299BE01615E7F4F0E9464
:10D02000F899BC0180EE92E10E948E9ACE0143965F
:10D030000E94DE9AC8010E94DE9ACE0149960E94A3
:10D04000DE9ACE014F960E94DE9A4DE2441641E0F0
:10D0500054066104710474F469A57AA58BA59CA596
:10D0600025E030E040E050E00E94E7B8672B682BF5
:10D07000692BF1F466EE72E1C8010E94419B45E024
:10D0800050E06FEF7FEFC8010E94885AC8010E94EC
:10D09000DE9A60EE72E1C8010E94419B45E050E0DB
:10D0A00070E060E0C8010E946857C8010E94DE9AE3
:10D0B0001DA2C3CE8091300D66EE72E1882309F483
:10D0C0005FC0CE010D960E94419B4AE050E067E0B0
:10D0D00070E0CE010D960E94CF59CE010D960E94B0
:10D0E000DE9ACDA0CC2001F165E575E1CE010D966B
:10D0F0000E94389B45E050E070E060E0CE010D9664
:10D100000E94885ACE010D960E94DE9A6BEF7BE05A
:10D11000CE010D960E944A9BCE010D960E944A5761
:10D12000CE010D960E94DE9A60EE72E1CE010D9660
:10D130000E94419B4AE050E06FEF7FEFCE010D96D9
:10D140000E946857CE010D960E94DE9AC85BDF4FA1
:10D150000FB6F894DEBF0FBECDBFDF91CF911F9108
:10D160000F91FF90EF90DF90CF90BF90AF909F9086
:10D170008F907F906F905F904F903F902F90089589
:10D18000CE010D960E94419B4AE050E06FEF7FEF89
:10D19000CE010D960E94885AA0CF4F925F926F9257
:10D1A0007F929F92AF92BF92CF92DF92EF92FF92C7
:10D1B0000F931F93CF93DF93CDB7DEB7A9970FB629
:10D1C000F894DEBF0FBECDBF982E882351F080911A
:10D1D000310D882331F06BEF7BE084ED9FE00E94FE
:10D1E000089C0E94B09760E08DE20E94FFA260E17F
:10D1F0008DE20E94FFA268E08DE20E94FFA24090B3
:10D200005613509057136090581370905913498ECD
:10D210005A8E6B8E7C8EC0905A13D0905B13E09028
:10D220005C13F0905D13CD8EDE8EEF8EF8A28091B0
:10D230005E1390915F13A0916013B09161138EA360
:10D240009FA3A8A7B9A789A39AA3ABA3BCA399201E
:10D25000C9F18091310D8823A9F167E475E1CE0110
:10D2600001960E94389BCE0101960E94A359CE01DF
:10D2700001960E94DE9A8E01075E1F4F5E0195E2C5
:10D28000A90EB11CD8016D917D918D919D918D015B
:10D2900046E00E94559C61E67AE084ED9FE00E94A2
:10D2A000939DA016B10671F76BEF7BE0CE0101965E
:10D2B0000E944A9BCE0101960E94A359CE0101967D
:10D2C0000E94DE9A23E938E144E85FE3C301B2013A
:10D2D0000E9410B82B013C014D865E866F86788ACD
:10D2E00022E430E645E85FE3C701B6010E9410B8CA
:10D2F0006B017C01C98ADA8AEB8AFC8A25E83BEE5D
:10D3000041E95FE36EA17FA188A599A50E9410B8AD
:10D310006D8B7E8B8F8B988F409256135092571344
:10D320006092581370925913C0925A13D0925B13A3
:10D33000E0925C13F0925D1360935E1370935F1341
:10D340008093601390936113992009F4A0C0809199
:10D35000310D882309F49BC06AE375E1CE01019683
:10D360000E94389BCE0101960E94A359CE010196DE
:10D370000E94DE9A8E01035F1F4F6E01B9E1CB0E52
:10D38000D11C7801F80161917191819191918F0186
:10D3900042E00E94559C61E67AE084ED9FE00E94A5
:10D3A000939DC016D10671F76BEF7BE0CE0101961D
:10D3B0000E944A9BCE0101960E94A359CE0101967C
:10D3C0000E94DE9A42E653E166E070E082E30E944A
:10D3D0002CA4A0906213B0906313C0906413D090FB
:10D3E000651300916613109167136DE275E184ED8A
:10D3F0009FE00E94B59D4AE050E0B50184ED9FE0BA
:10D400000E94469D61E67AE084ED9FE00E94939D34
:10D410004AE050E0B60184ED9FE00E94469D61E63F
:10D420007AE084ED9FE00E94939D4AE050E0B801CD
:10D4300084ED9FE00E94469D6BEF7BE084ED9FE0D2
:10D440000E94089CCE0101960E94ABA464E275E1A3
:10D4500084ED9FE00E94B59D8E010F5F1F4FD801A4
:10D460006D917D918D919D918D014AE00E94559C19
:10D4700061E67AE084ED9FE00E94939D0E151F0502
:10D4800071F76BEF7BE084ED9FE00E94089C61E008
:10D490008DE10E94FFA29920B1F08091310D882387
:10D4A00091F060E175E184ED9FE00E94B59DAE01D1
:10D4B0004B5D5F4F61E070E08DE10E942CA48DA177
:10D4C00090E00E94809D62E08EE10E94FFA263E0F6
:10D4D0008FE10E94FFA264E080E20E94FFA29920F7
:10D4E00009F450C08091310D882309F44BC064EFDA
:10D4F00074E184ED9FE00E94B59DAE014B5D5F4FEE
:10D5000061E070E08EE10E942CA4CDA0D12CAE0190
:10D510004B5D5F4F61E070E08FE10E942CA4EDA0B5
:10D52000F12CAE014B5D5F4F61E070E080E20E9444
:10D530002CA40DA110E04AE050E0B60184ED9FE07C
:10D540000E94469D61E67AE084ED9FE00E94939DF3
:10D550004AE050E0B70184ED9FE00E94469D61E6FD
:10D560007AE084ED9FE00E94939D4AE050E0B8018C
:10D5700084ED9FE00E94469D6BEF7BE084ED9FE091
:10D580000E94089C65E081E20E94FFA29920B1F010
:10D590008091310D882391F061EE74E184ED9FE07C
:10D5A0000E94B59DAE014B5D5F4F61E070E081E28E
:10D5B0000E942CA48DA190E00E94809D66E082E2F2
:10D5C0000E94FFA29920B1F08091310D882391F043
:10D5D00069EC74E184ED9FE00E94B59DAE014B5D66
:10D5E0005F4F61E070E082E20E942CA48DA190E088
:10D5F0000E94809D67E083E20E94FFA29920B1F023
:10D600008091310D882391F063EB74E184ED9FE00C
:10D610000E94B59DAE014B5D5F4F61E070E083E21B
:10D620000E942CA48DA190E00E94809D68E084E27D
:10D630000E94FFA29920B1F08091310D882391F0D2
:10D640006BE974E184ED9FE00E94B59DAE014B5DF6
:10D650005F4F61E070E084E20E942CA48DA190E015
:10D660000E94809D69E085E20E94FFA29920B1F0AE
:10D670008091310D882391F061E874E184ED9FE0A1
:10D680000E94B59DAE014B5D5F4F61E070E085E2A9
:10D690000E942CA48DA190E00E94809D6AE086E209
:10D6A0000E94FFA29920B1F08091310D882391F062
:10D6B0006BE674E184ED9FE00E94B59DAE014B5D89
:10D6C0005F4F61E070E086E20E942CA48DA190E0A3
:10D6D0000E94809D6BE088E20E94FFA29920B1F039
:10D6E0008091310D882391F062E574E184ED9FE033
:10D6F0000E94B59DAE014B5D5F4F61E070E088E236
:10D700000E942CA48DA190E00E94809D6CE089E293
:10D710000E94FFA2992009F479C08091310D8823DD
:10D7200009F474C06AE374E184ED9FE00E94B59D42
:10D73000AE014B5D5F4F61E070E089E20E942CA476
:10D740008DA190E00E94809D63E274E184ED9FE0F2
:10D750000E94B59D66E070E087E20E9465A490E0BB
:10D760000E94809D6CE074E184ED9FE00E94B59D75
:10D7700065E070E087E20E9465A490E00E94809DD1
:10D7800065EF73E184ED9FE00E94B59D64E070E079
:10D7900087E20E9465A490E00E94809D6CED73E199
:10D7A00084ED9FE00E94B59D62E070E087E20E94F8
:10D7B00065A490E00E94809D63EC73E184ED9FE09E
:10D7C0000E94B59D61E070E087E20E9465A490E050
:10D7D0000E94809D6AEA73E184ED9FE00E94B59DFE
:10D7E00070E060E087E20E9465A490E00E94809D66
:10D7F00069E973E184ED9FE00E94B59D63E070E00C
:10D8000087E20E9465A490E00E94809D41E067E06D
:10D8100070E087E20E9480A441E063E070E087E26C
:10D820000E9480A441E063E070E08AE20E9480A44C
:10D83000992091F08091310D882371F060E873E1B7
:10D8400084ED9FE00E94B59D63E070E08AE20E9453
:10D8500065A490E00E94809D40E063E070E08AE271
:10D860000E9480A4992091F08091310D882371F05D
:10D8700066E673E184ED9FE00E94B59D63E070E091
:10D880008AE20E9465A490E00E94809D41E062E0EF
:10D8900070E08AE20E9480A4992091F08091310D7D
:10D8A000882371F06AE473E184ED9FE00E94B59DE6
:10D8B00062E070E08AE20E9465A490E00E94809D90
:10D8C00040E062E070E08AE20E9480A4992091F03A
:10D8D0008091310D882371F06DE273E184ED9FE05A
:10D8E0000E94B59D62E070E08AE20E9465A490E02B
:10D8F0000E94809D41E061E070E08AE20E9480A485
:10D90000992091F08091310D882371F061E173E1EC
:10D9100084ED9FE00E94B59D61E070E08AE20E9484
:10D9200065A490E00E94809D40E061E070E08AE2A2
:10D930000E9480A4992091F08091310D882371F08C
:10D9400064EF72E184ED9FE00E94B59D61E070E0BC
:10D950008AE20E9465A490E00E94809D41E070E010
:10D9600060E08AE20E9480A4992091F08091310DBC
:10D97000882371F068ED72E184ED9FE00E94B59D0F
:10D9800070E060E08AE20E9465A490E00E94809DC1
:10D9900040E070E060E08AE20E9480A4992091F06B
:10D9A0008091310D882371F06BEB72E184ED9FE083
:10D9B0000E94B59D70E060E08AE20E9465A490E05C
:10D9C0000E94809D41E066E070E087E20E9480A4B2
:10D9D00041E065E070E087E20E9480A441E064E0FD
:10D9E00070E087E20E9480A440E062E070E087E29D
:10D9F0000E9480A440E061E070E087E20E9480A481
:10DA000040E070E060E087E20E9480A4992009F481
:10DA100075C08091310D882309F470C063EA72E10A
:10DA200084ED9FE00E94B59D66E070E08BE20E946D
:10DA300065A490E00E94809D65E872E184ED9FE01E
:10DA40000E94B59D65E070E08BE20E9465A490E0C5
:10DA50000E94809D67E672E184ED9FE00E94B59D83
:10DA600064E070E08BE20E9465A490E00E94809DDB
:10DA70006EE472E184ED9FE00E94B59D62E070E08B
:10DA80008BE20E9465A490E00E94809D65E372E1B4
:10DA900084ED9FE00E94B59D61E070E08BE20E9402
:10DAA00065A490E00E94809D6CE172E184ED9FE0AE
:10DAB0000E94B59D70E060E08BE20E9465A490E05A
:10DAC0000E94809D69E072E184ED9FE00E94B59D17
:10DAD00063E070E08BE20E9465A490E00E94809D6C
:10DAE00064EF71E184ED9FE00E94B59D64E070E019
:10DAF0008CE20E9465A490E00E94809D40E064E07A
:10DB000070E08CE20E9480A4AE014B5D5F4F61E04B
:10DB100070E08CE20E942CA46DA1607F66608CE2B4
:10DB20000E94FFA2992009F45EC08091310D8823E4
:10DB300009F459C060EE71E184ED9FE00E94B59D4B
:10DB4000AE014B5D5F4F61E070E08CE20E942CA45F
:10DB50006DA16F706650770B072E000C880B990B28
:10DB60000E94B1B79B01AC0160E070E080E090E4FE
:10DB70000E94FDBB20E030E048EC50E40E9410B869
:10DB80000E94379D69EC71E184ED9FE00E94B59D94
:10DB9000AE014B5D5F4F61E070E080E30E942CA41A
:10DBA0006DA14AE050E084ED9FE00E94F19B61EBA3
:10DBB00071E184ED9FE00E94B59D61E070E080E33B
:10DBC0000E9465A490E00E94809D68E971E184ED67
:10DBD0009FE00E94B59D61E070E08FE20E9465A425
:10DBE00090E00E94809D41E061E070E08FE20E9441
:10DBF00080A4992091F08091310D882371F060E824
:10DC000071E184ED9FE00E94B59D61E070E08EE2DD
:10DC10000E9465A490E00E94809D41E061E070E078
:10DC20008EE20E9480A440E067E070E081E30E9401
:10DC300080A4992009F455C08091310D882309F4FE
:10DC400050C06DE671E184ED9FE00E94B59D67E0F4
:10DC500070E081E30E9465A490E00E94809D6DEEDB
:10DC60007AE084ED9FE00E94939DAE014B5D5F4F93
:10DC700061E070E080E00E942CA48DA10E94A514B8
:10DC80006BEF7BE084ED9FE00E94089C0DE110E0CB
:10DC900065E377E084ED9FE00E94939D40E150E0D2
:10DCA000B80184ED9FE00E94469D61EF7AE084ED2B
:10DCB0009FE00E94939DAE014B5D5F4F61E070E07D
:10DCC000802F0E942CA48DA10E94A5146BEF7BE0F5
:10DCD00084ED9FE00E94089C0F5F1F4F0A331105DF
:10DCE000B9F6A9960FB6F894DEBF0FBECDBFDF918F
:10DCF000CF911F910F91FF90EF90DF90CF90BF9049
:10DD0000AF909F907F906F905F904F9008951F937A
:10DD1000CF93DF93CDB7DEB7A8970FB6F894DEBFE9
:10DD20000FBECDBF182F0E94B0978EE10E94DB8DF1
:10DD300062E081E790E10E94580C60E081E790E1A9
:10DD40000E94580C0E94FCA28EE10E94DB8D61E0D3
:10DD500081E790E10E94580C60E281E790E10E9427
:10DD6000580C0E94FCA280E290E090932B138093C9
:10DD70002A1380E090E8A9E8B4E48093E00490934B
:10DD8000E104A093E204B093E30480E090E0A5E70F
:10DD9000B4E48093DC049093DD04A093DE04B0939C
:10DDA000DF04BE016F5F7F4F87E293E10E948C0C1E
:10DDB000112309F484C06BE77CE084ED9FE00E94AE
:10DDC000B59D84ED9FE00E94ED9B6BE67CE084EDC9
:10DDD0009FE00E94B59DBE016F5F7F4F84ED9FE085
:10DDE0000E94089C6BE57CE084ED9FE00E94B59D5D
:10DDF0006D857E858F8598890E94219C6BE47CE0EF
:10DE000084ED9FE00E94B59D69897A898B899C8900
:10DE10000E94219C6BE37CE084ED9FE00E94B59D15
:10DE200020E030E040E251E4698D7A8D8B8D9C8D4D
:10DE30000E9410B842E00E94559C64EF7AE084EDA5
:10DE40009FE00E94089C6BE27CE084ED9FE00E94D2
:10DE5000B59D20E030E040E251E46D8D7E8D8F8DE8
:10DE600098A10E9410B842E00E94559C64EF7AE0AD
:10DE700084ED9FE00E94089C6BE17CE084ED9FE0D4
:10DE80000E94B59D20E030E040E251E469A17AA112
:10DE90008BA19CA10E9410B842E00E94559C64EFA7
:10DEA0007AE084ED9FE00E94089C65EF7BE084EDC2
:10DEB0009FE00E94B59D84ED9FE00E94ED9B64EF82
:10DEC00071E080E090E00E9439A5A8960FB6F89422
:10DED000DEBF0FBECDBFDF91CF911F910895DF92BE
:10DEE000EF92FF920F931F93CF93DF93CDB7DEB7DF
:10DEF00062970FB6F894DEBF0FBECDBF8C011092B3
:10DF0000210D6BEF7BE0CE010D960E944A9BFF2412
:10DF1000F39484ED9FE00E94208B2091210D181630
:10DF200019067CF521112DC084ED9FE00E94FE8A28
:10DF30008A3009F07EC089899A89892B09F481C0C9
:10DF4000F092210D68EF7AE0CE0101960E944A9B83
:10DF5000BE01635F7F4FCE0101960E94F899BC011C
:10DF6000CE0107960E94419BCE0107960E94A359BD
:10DF7000CE0107960E94DE9ACE0101960E94DE9A9B
:10DF800060C0F12CE12CDD24D394222309F460C07D
:10DF900089899A89019709F045C06EEB76E0CE0138
:10DFA00007960E944A9BBE01695F7F4FCE010D9686
:10DFB0000E94C799F12C811115C068EE77E0CE015F
:10DFC00001960E944A9BBE016F5F7F4FCE010D9666
:10DFD0000E94C799FF24F3948111F12CCE01019680
:10DFE0000E94DE9ACE0107960E94DE9AFF20A1F0E1
:10DFF00050E040E0BE01635F7F4FCE0101960E947A
:10E000003858BE016F5F7F4F88EF92E10E94A59A5A
:10E01000CE0101960E94DE9A64E170E080E090E01B
:10E020000E9439A5BE01635F7F4FC8010E942F9BEC
:10E0300090C08D3009F47FCF682FCE010D960E94DD
:10E04000359A6AE070E080E090E00E9439A561CFE7
:10E050008DEF9DE00E94208B1816190614F58DEFA8
:10E060009DE00E94FE8A8A30A9F08D3099F090914F
:10E07000210D91110FC0682FCE010D960E94359A87
:10E080008FEFE81AF80A65E070E080E090E00E9407
:10E0900039A5DECF89899A89892BA9F3D092210DE0
:10E0A000F2CF64E170E080E090E00E9439A5EF28B3
:10E0B000D1F189899A89892BB1F18091310D882319
:10E0C00061F160EC75E0CE0101960E944A9BBE01B1
:10E0D0006F5F7F4FCE010D960E94C799F82ECE013B
:10E0E00001960E94DE9AF11018C061E07BE084ED99
:10E0F0009FE00E94939DBE01635F7F4FCE0101961A
:10E100000E94419BBE016F5F7F4F84ED9FE00E94A4
:10E11000A39DCE0101960E94DE9A64E170E080E04A
:10E1200090E00E9439A589899A892091210D2111B9
:10E1300031CF009709F02ECF64E670E080E090E0E8
:10E140000E9439A50E94F80F6BEF7BE0C8010E9486
:10E150004A9BCE010D960E94DE9AC80162960FB6C8
:10E16000F894DEBF0FBECDBFDF91CF911F910F910D
:10E17000FF90EF90DF900895DF92EF92FF920F9360
:10E180001F93CF93DF93CDB7DEB72C970FB6F894DC
:10E19000DEBF0FBECDBF8C011092210D6BEF7BE077
:10E1A000CE0107960E944A9BF12CE12CDD24D394EA
:10E1B0008DEF9DE00E94208B1816190694F4809133
:10E1C000210D81110EC08DEF9DE00E94FE8A8A30E4
:10E1D000D1F58B859C85892B09F443C0D092210D04
:10E1E00040C062E370E080E090E00E9439A5EF2833
:10E1F00051F08DEF9DE00E94C38B64E670E080E0FB
:10E2000090E00E9439A58091210D811131C08B854C
:10E210009C85892B69F56BEF7BE0C8010E944A9BC6
:10E22000CE0107960E94DE9AC8012C960FB6F8948C
:10E23000DEBF0FBECDBFDF91CF911F910F91FF9039
:10E24000EF90DF9008958D3021F29091210D911182
:10E25000C0CF682FCE0107960E94359A8FEFE81A3B
:10E26000F80A6FE070E080E090E00E9439A5A0CF4E
:10E270008091310D882379F0BE01695F7F4FCE0117
:10E2800001960E94419BCE0101960E94F256CE015A
:10E2900001960E94DE9ABE01695F7F4FC8010E940D
:10E2A0002F9BBECF4F925F926F927F928F929F92E1
:10E2B000AF92BF92EF92FF920F931F93CF93DF9392
:10E2C000CDB7DEB762970FB6F894DEBF0FBECDBFF5
:10E2D0007C015B0181E19DE00E942791892BD9F4AB
:10E2E0006BEF7BE0C7010E944A9BC70162960FB6A5
:10E2F000F894DEBF0FBECDBFDF91CF911F910F917C
:10E30000FF90EF90BF90AF909F908F907F906F9015
:10E310005F904F9008954091150D5091160D6091AA
:10E32000170D7091180DCE0107960E9444588091E8
:10E33000310D882359F168E07BE0CE0101960E94FF
:10E340004A9BBE01695F7F4FCE0101960E94F899FA
:10E350006CE978E00E94E299BC0184ED9FE00E94A4
:10E36000959DCE0101960E94DE9A4091150D509127
:10E37000160D6091170D7091180D20E184ED9FE04E
:10E380000E94A19B84ED9FE00E94ED9B70E060E005
:10E39000CE0107960E94B699182F8A3211F010927A
:10E3A000140C0E94F80F6093280D7093290D809330
:10E3B0002A0D90932B0D6BEF7BE0CE010D960E9402
:10E3C0004A9B812F110F990BC0970A9708F068C0DC
:10E3D000CE0107960E94DB98633071058105910597
:10E3E0000CF084C001E010E082E0982E0A151B05B5
:10E3F00009F47CC06CE271E080E090E00E9439A5F5
:10E4000090927D1010928010412C512C320181E0AD
:10E410009DE00E942791892B91F48EE148165104CA
:10E420006104710449F16EE170E080E090E00E94C7
:10E4300039A58FEF481A580A680A780AE8CF8EE1A2
:10E440004816510461047104B9F04091050D5091D2
:10E45000060D6091070D7091080DCE0101960E9486
:10E460004458BE016F5F7F4FCE010D960E94A59A62
:10E47000CE0101960E94DE9A89899A89892B39F00A
:10E48000BE01635F7F4FCE0107960E94629A0F5FC5
:10E490001F4F6BEF7BE0CE010D960E945E98A6CFDA
:10E4A0006CE271E080E090E00E9439A582E0809308
:10E4B0007D1010928010812C912C540181E09DE000
:10E4C0000E942791892B61F58EE188169104A104A1
:10E4D000B10409F043C089899A89892B39F0BE01BA
:10E4E000635F7F4FCE0107960E94629A64E670E0F8
:10E4F00080E090E00E9439A582E080937D10109228
:10E500008010BE01695F7F4FC7010E942F9BCE0123
:10E510000D960E94DE9ACE0107960E94DE9AE5CE05
:10E520008EE188169104A104B104A9F24091050D71
:10E530005091060D6091070D7091080DCE01019666
:10E540000E944458BE016F5F7F4FCE010D960E941E
:10E55000A59ACE0101960E94DE9ABDCF6EE170E0D1
:10E5600080E090E00E9439A58FEF881A980AA80AE7
:10E57000B80AA4CFAF92BF92CF92DF92EF92FF92F0
:10E580000F931F93CF93DF93CDB7DEB72C970FB6C2
:10E59000F894DEBF0FBECDBF7C015B010E947DA061
:10E5A000182F811117C06BEF7BE0C7010E944A9BB7
:10E5B000C7012C960FB6F894DEBF0FBECDBFDF911A
:10E5C000CF911F910F91FF90EF90DF90CF90BF9070
:10E5D000AF9008958A3211F01092140C0E94F80F37
:10E5E0006093280D7093290D80932A0D90932B0D25
:10E5F000612FCE0107960E94169B812F012E000CE1
:10E60000990BC0970A9768F5CE0107960E94DB9890
:10E6100063307105810591050CF070C001E010E0D8
:10E620000A151B0509F46AC062E370E080E090E01F
:10E630000E9439A50E947DA0D12CC12C81113BC024
:10E640008FEFC81AD80A85E1C816D10409F456C05C
:10E650006EE170E080E090E00E9439A50E947DA00C
:10E66000EDCF612FCE0101960E94169BBE016F5F18
:10E670007F4FCE0107960E94A59ACE0101960E9477
:10E68000DE9A62E370E080E090E00E9439A50E948B
:10E690007DA010E000E0811121C00F5F1F4F0F31FE
:10E6A000110561F16EE170E080E090E00E9439A513
:10E6B0000E947DA0F0CF682FCE0101960E94169B8C
:10E6C000BE016F5F7F4FCE0107960E94629ACE0116
:10E6D00001960E94DE9A0F5F1F4FA2CF682FCE01D6
:10E6E00001960E94169BBE016F5F7F4FCE01079679
:10E6F0000E94629ACE0101960E94DE9ABE01695F75
:10E700007F4FC7010E942F9BCE0107960E94DE9A81
:10E710004FCF3F924F925F926F927F928F929F92D4
:10E72000AF92BF92CF92DF92EF92FF920F931F931F
:10E73000CF93DF93CDB7DEB7E4970FB6F894DEBF83
:10E740000FBECDBF8091140C8823D1F01092140C11
:10E75000E4960FB6F894DEBF0FBECDBFDF91CF9128
:10E760001F910F91FF90EF90DF90CF90BF90AF90EF
:10E770009F908F907F906F905F904F903F90089503
:10E7800081E08093140C6BEF7BE0CE0185960E94B4
:10E790004A9B6BEF7BE0CE018B960E944A9B10E078
:10E7A00000E082E0382E98EEC92E93E0D92EE12CBD
:10E7B000F12CF8013197E031F105B0F48827EC51E4
:10E7C000FC488F4F0C94D5BCC974607575757E7507
:10E7D00087759075A175AA75D975EA75F375FC757D
:10E7E0000576A076A976B2766BEF7BE0CE018596B2
:10E7F0000E945E988091C5119091C611892B31F4C9
:10E8000066E576E0CE0185960E945E988091C511FE
:10E810009091C611019731F460E576E0CE018596BE
:10E820000E945E988091C5119091C611029731F4B3
:10E830006AE576E0CE0185960E945E9889A59AA544
:10E84000892B31F06BED73E1CE0185960E94629ABF
:10E850006FE576E0CE0101960E944A9B67EE73E178
:10E86000CE0101960E94F899BC01CE018B960E94C0
:10E870008E9ACE0101960E94DE9A8091C5119091E8
:10E88000C611019709F046C0BE016B5D7F4FCE01F6
:10E8900001960E94419B48EC50E06FEF7FEFCE0164
:10E8A00001960E94885ACE0101960E94DE9ABE010E
:10E8B000655D7F4FCE0101960E94419B40ED57E080
:10E8C0006FEF7FEFCE0101960E946857CE0101964F
:10E8D0000E94DE9ACE0101960E94CC2F8D819E81EE
:10E8E0000097A1F0E981FA812081222379F007972E
:10E8F00068F06EED7EE0CE0185960E94699ABE01B9
:10E900006F5F7F4FCE018B960E948E9ACE0101964B
:10E910000E94DE9ABE016B5D7F4FCE0101960E9480
:10E92000419B48EC50E06FEF7FEFCE0101960E94D3
:10E93000CF59CE0101960E94DE9ABE01655D7F4FE0
:10E94000CE0101960E94419B48EC50E06FEF7FEFB3
:10E95000CE0101960E946857CE0101960E94DE9A70
:10E960000E947DA0982EB12CA12C911060C28FEF37
:10E97000A81AB80A95E6A916B10409F4FCC10E94C8
:10E980007DA0982E64E170E080E090E00E9439A5BF
:10E99000ECCF62ED7EE0CE0185960E94699A0E94DE
:10E9A000F80F4B015C010E94F80FA70196010E942D
:10E9B00019B9CA01B90120E831E541E050E00E94EF
:10E9C00019B920E13EE040E050E00E94E7B829ABF1
:10E9D0003AAB4BAB5CAB2CE330E040E050E00E9444
:10E9E000E7B829013A01AB01BC01CE0101960E94B2
:10E9F0006898B301A201CE0107960E94689849A9C0
:10EA00005AA96BA97CA9CE010D960E946898C501F0
:10EA1000B40120E03CE546E255E00E9419B9BA0194
:10EA2000A901CE0149960E946898BE01675E7F4F9A
:10EA3000CE0143960E94419B6DE07BE0CE01439660
:10EA40000E94E299BE01635F7F4F0E94F89960E1E6
:10EA50007BE00E94E299BE01695F7F4F0E94F899B6
:10EA600065EB76E00E94E299BE016F5F7F4F0E94E6
:10EA7000F8996EEB76E00E94E299BC01CE014F96C8
:10EA80000E94419BCE0143960E94DE9ACE01499698
:10EA90000E94DE9ACE010D960E94DE9ACE01079664
:10EAA0000E94DE9ACE0101960E94DE9ABE01615E4E
:10EAB0007F4FCE018B960E94A59ACE014F9628CF0C
:10EAC00080912C0C90912D0C63EC7EE0019711F05D
:10EAD00065EB7EE0CE0185960E94699A65EA7EE04C
:10EAE000CE018B960E94699A15CF65E97EE0CE0132
:10EAF00085960E94699A68E87EE0F2CF6BE77EE037
:10EB0000CE0185960E94699A60E77EE0E9CF64E6CF
:10EB10007EE0CE0185960E94699A63E57EE0E0CFB3
:10EB200080912C0C90912D0C68E47EE0039711F0FD
:10EB30006EE37EE0CE0185960E94699A63E37EE0F3
:10EB4000CFCF66E27EE0CE0185960E94699A67E1AA
:10EB50007EE0C6CF6CE07EE0CE0185960E94699A89
:10EB600060917C1170917D11CE0107960E9495985D
:10EB70006AE67AE0CE0101960E944A9BBE01695F77
:10EB80007F4FCE0101960E94F8996BE37AE00E94D4
:10EB9000E299BC01CE0185960E94629ACE0101964F
:10EBA0000E94DE9ACE0107960E94DE9A6FEF7DE00A
:10EBB00097CF80912C0C90912D0C6EEE7DE00297FA
:10EBC00011F06EED7DE0CE0185960E94699A61EDAF
:10EBD0007DE086CF65EC7DE0CE0185960E94699A46
:10EBE00065EB7DE07DCF6AEA7DE0CE0185960E94EF
:10EBF000699A60EA7DE074CF64E97DE0CE01859694
:10EC00000E94699A64E87DE06BCFB0907E1169E75D
:10EC10007DE0CE0185960E94699A83E08B1524F1F0
:10EC200092E0B9160CF073C0BB2031F181E0B81648
:10EC300009F464C060917E11062E000C770BCE01A2
:10EC400007960E9495986EE279E0CE0101960E94A7
:10EC50004A9BBE01695F7F4FCE0101960E94F899E1
:10EC6000BC018CEE92E13FC094E0B912E3CF67E1C2
:10EC70007BE08CEE92E146C080907F1190908011F5
:10EC8000A0908111B090821120E030E048E452E47D
:10EC9000C501B4010E94AAB787FF02C03324339490
:10ECA000A501940160E070E080EA90E40E9429BA36
:10ECB000AB01BC01232DCE0107960E94E69A6EEBB4
:10ECC0007AE0CE0101960E944A9BBE01695F7F4FA8
:10ECD000CE0101960E94F8996CE17BE00E94E299D6
:10ECE000BC01CE0185960E94629ACE0101960E94D7
:10ECF000DE9ACE0107960E94DE9A06C063E17BE0B1
:10ED0000CE0185960E94589A69E67DE0E9CE8B2D6A
:10ED10009AE08902B0011124CE0107960E949598CD
:10ED20006AE67AE0CE0101960E944A9BBE01695FC5
:10ED30007F4FCE0101960E94F89965E17BE0CECF2E
:10ED40006CE57DE0CE0185960E94699A6CE47DE0D9
:10ED5000C7CE60E47DE0CE0185960E94699A61E3AA
:10ED60007DE0BECE65E27DE0CE0185960E94699A87
:10ED700065E17DE0B5CE6BEF7BE08AE093E10E9438
:10ED80005E98CE0101960E946F6FBE016F5F7F4F4C
:10ED90008AE093E10E94A59ACE0101960E94DE9A34
:10EDA00080910E1390910F13892B89F461E070E02C
:10EDB000CE0101960E94BA72BE016F5F7F4F8AE05A
:10EDC00093E10E94A59ACE0101960E94DE9A80915D
:10EDD0000E1390910F13892B89F461E070E0CE013E
:10EDE00001960E945271BE016F5F7F4F8AE093E1EE
:10EDF0000E94A59ACE0101960E94DE9A80910E1380
:10EE000090910F13892B51F48091140C882331F0C9
:10EE10000F5F1F4F0131110509F0CBCCCE018B964E
:10EE20000E94DE9ACE0185960E94DE9A91CC1092C5
:10EE3000140CF4CF2F923F924F925F926F927F9279
:10EE40008F929F92AF92BF92CF92DF92EF92FF92FA
:10EE50000F931F93CF93DF93CDB7DEB7C554D1097E
:10EE60000FB6F894DEBF0FBECDBF8C01E0902A0C28
:10EE7000F0902B0C8091310D882349F063E671E10D
:10EE800084ED9FE00E94B59DC8010E94809DC8014D
:10EE90000596059710F40C94778A80912A0C90912E
:10EEA0002B0C80179107E1F00E9426570E94D5167F
:10EEB0000C3E2FEF120724F010932B0C00932A0C1A
:10EEC000B801CE0101960E949598BE016F5F7F4FF9
:10EED00088EF92E10E94A59ACE0101960E94DE9AE7
:10EEE0006BEF7BE08CEE92E10E945E9861E67AE047
:10EEF000CE0101960E944A9B4AE050E06FEF7FEFFF
:10EF0000CE0101960E94CF59CE0101960E94DE9A51
:10EF1000F8017E96E832F10510F00C94588A8827A3
:10EF2000EB56F8488F4F0C94D5BCD977588A68892E
:10EF3000588ABD89B58988897289588A6D89588AA5
:10EF4000588A588A588A588A7E78E9786F79F77A89
:10EF5000FE7AD27C857DAD7E84808181D681EB81F5
:10EF6000EE81588A2F823282DE839B85B785D586D3
:10EF700041870D8825882D8827890E94E516CB5B5F
:10EF8000DF4F0FB6F894DEBF0FBECDBFDF91CF913C
:10EF90001F910F91FF90EF90DF90CF90BF90AF90B7
:10EFA0009F908F907F906F905F904F903F902F90A9
:10EFB00008956FE17BE0CE0101960E944A9B64E0D8
:10EFC00073E1CE0101960E94F899BC0186EE92E1B0
:10EFD0000E948E9ACE0101960E94DE9A66EE72E140
:10EFE000CE0101960E94419BCE0101960E94F256ED
:10EFF000CE0101960E94DE9A63E27BE0CE0101968B
:10F000000E944A9B64E073E1CE0101960E94F89948
:10F01000BC01CE0180960E94419B48EC50E070E01C
:10F0200060E0CE0180960E94885ACE0180960E94B0
:10F03000DE9ACE0101960E94DE9A41E050E064E043
:10F0400073E1CE0101960E943858BE016F5F7F4F79
:10F0500080EE92E10E94A59ACE0101960E94DE9A6E
:10F0600080EE92E10E94DB98DC01CB010197A109BF
:10F07000B10962EE70E189309105A105B10590F406
:10F08000FC018827E95BF7488F4F0C94D5BC50787A
:10F09000667869786C786F787278757878787B782C
:10F0A00063E571E186EE92E10E94699A66EE72E193
:10F0B000CE0101960E94419B4CED55E06FEF7FEF32
:10F0C000CE0101960E9468570C94828966E471E132
:10F0D000E9CF66E371E1E6CF6CE271E1E3CF68E28C
:10F0E00071E1E0CF68E171E1DDCF6AE071E1DACF93
:10F0F0006CEF70E1D7CF6FEE70E1D4CF0E9426574E
:10F1000089E390E00E942A5420E030E04AE754E48A
:10F110000E9410B8AB01BC0121E0CE0101960E9413
:10F12000E69A68EA78E0CE0180960E944A9BBE018A
:10F130006F5F7F4FCE0180960E94F89969E27BE075
:10F140000E94E299BC018CEE92E10E948E9ACE015F
:10F1500080960E94DE9ACE0101960E94DE9A6DE2B0
:10F160007BE086EE92E10E945E9866EE72E1CE014F
:10F1700001960E94419B4AE050E068E070E0CE01B9
:10F1800001960E94885ACE0101960E94DE9A6CEE8A
:10F1900072E1CE0101960E94419B4AE050E06FEF80
:10F1A0007FEFCE0101960E946857CE0101960E9422
:10F1B000DE9A66EE72E18CEE92E10E94629A809194
:10F1C000300D882309F4C8C164E670E080E090E067
:10F1D0007DC4C0900402D09005020E94265789E3A6
:10F1E00090E00E942A5420E030E04AE754E40E9474
:10F1F00010B80E94D5BACE0101960E94959868EA8F
:10F2000078E0CE0180960E944A9BBE016F5F7F4FDF
:10F21000CE0180960E94F89969E27BE00E94E29913
:10F22000BC018CEE92E10E948E9ACE0180960E94E3
:10F23000DE9ACE0101960E94DE9A8091F0129091A2
:10F24000F11253E0F52E099710F042E0F42E809170
:10F250007B1140E050E0BA018330DCF4C6010E942B
:10F2600036184B015C0160917C1170917D11072E65
:10F27000000C880B990B0E94B1B7A50194010E9464
:10F2800010B820E030EC4FE754E40E9429BAAB01FB
:10F29000BC012F2DCE0101960E94E69A6BE57BE022
:10F2A000CE0180960E944A9BBE016F5F7F4FCE01C8
:10F2B00080960E94F89965E076E00E94E299BC0190
:10F2C0008CEE92E10E94629ACE0180960E94DE9AB4
:10F2D000CE0101960E94DE9A65E37BE042CF8091E9
:10F2E000300D882309F478C18AE99EE00E94F690E7
:10F2F00062E370E080E090E00E9439A561E08091D7
:10F300008E040E9441A060E080918C040E9441A084
:10F3100064E670E080E090E00E9439A56091880486
:10F320007091890480918A0490918B040E946416E4
:10F330000E948116AB01BC0123E0CE0180960E94A1
:10F34000E69ABE01605E7F4FCE0101960E94419B0E
:10F3500068E57BE0CE0101960E94E299BC0186EE51
:10F3600092E10E948E9ACE0101960E94DE9ACE0111
:10F3700080960E94DE9A69EB76E0CE0101960E94AB
:10F380004A9B66EE72E1CE0101960E94F899BC019B
:10F390008CEE92E10E948E9ACE0101960E94DE9A36
:10F3A0000E9481166B017C010E94E7A14B015C0168
:10F3B0008BE19EE40197F1F70E9481162B013C013D
:10F3C0000E94E7A19B01AC01281939094A095B0990
:10F3D00049015A0131ED831637E09306A104B104C7
:10F3E000CCF0A7019601C301B2010E944AB96B019A
:10F3F0007C0120E030E0A9010E9432BB181674F4B1
:10F4000026EA3BE944EC5BE3C701B6010E94AAB7D8
:10F4100087FF0EC040E050E0BA0126C026EA3BE973
:10F4200044EC5BEBC701B6010E9432BB181694F3A3
:10F43000C501B40128EE33E040E050E00E94E7B897
:10F44000CA01B9010E94B1B74B015C0120E030E074
:10F450004AE754E4C701B6010E9410B8A50194011F
:10F460000E9429BAAB01BC0122E0CE0180960E9425
:10F47000E69ABE01605E7F4FCE0101960E94419BDD
:10F480006CEB76E0CE0101960E94E299BC0180EE21
:10F4900092E10E948E9ACE0101960E94DE9ACE01E0
:10F4A00080960E94DE9A6EE37BE0CE0101960E9478
:10F4B0004A9B60EE72E1CE0101960E94F899BC0170
:10F4C0008CEE92E10E94629ACE0101960E94DE9A31
:10F4D00061E67AE0CE0101960E944A9B60EE72E1FD
:10F4E000CE0101960E94F899BC0186EE92E10E943D
:10F4F000629ACE0101960E94DE9A67EE7EE0CE010E
:10F5000001960E94389B4AE050E070E060E0CE0136
:10F5100001960E94885ACE0101960E94DE9A66EEFC
:10F5200072E1CE0101960E94419B45E050E06FEFF1
:10F530007FEFCE0101960E946857CE0101960E948E
:10F54000DE9A62E47BE08CEE92E10E94589A60E0E1
:10F5500080918E040E9441A08091F0129091F1124E
:10F56000009799F14197A8F40230110594F06CEEE0
:10F5700072E1CE0101960E94419B4AE050E06FEF9C
:10F580007FEFCE0101960E946857CE0101960E943E
:10F59000DE9A6CEE72E1CE0101960E94419BCE0193
:10F5A00001960E94F256CE0101960E94DE9A6CEE00
:10F5B00072E1CE0101960E94419BCE0101960E940C
:10F5C0006E19CE0101960E94DE9A64E670E080E03A
:10F5D00090E00E9439A5D3CC6091EB047091EC04CB
:10F5E0008091ED049091EE040E94222BB5CF809182
:10F5F0007B0490917C040E943D2DAECF40917D0410
:10F6000026964FAF269760E0842F0E9441A08091FC
:10F61000300D811109C08091E1113FE0C32ED12C42
:10F62000E12CF12C882329F023E0C22ED12CE12CEF
:10F63000F12C66EF7EE08CEE92E10E94699A6CEE0E
:10F6400072E1CE0101960E94419B4AE050E06FEFCB
:10F650007FEFCE0101960E94885ACE0101960E944A
:10F66000DE9A312C212C21961FAE219725961FAEB4
:10F6700025971CAE1DAE1EAE1FAE92E3692E712CF7
:10F68000812C912C540126968FAD26970E94C4A1FF
:10F69000092E000CAA0BBB0B880E991EAA1EBB1EBE
:10F6A00065E070E080E090E00E9439A551E0651AC5
:10F6B000710849F74090D4045090D5046090D60466
:10F6C0007090D704C501B4010E94B1B720E030E0CA
:10F6D00040EA50E40E9410B820E030E040E85AE3ED
:10F6E0000E9410B820E030E048E452E40E9429BAB9
:10F6F000A30192010E944AB920E030E040E751E4C2
:10F700000E9410B84B015C01A30192016AE979E9FA
:10F7100089E390E40E944AB99B01AC01C501B401A0
:10F720000E9429BA20E030E0A9010E944BB920E0F4
:10F7300030E040E251E40E9410B84B015C01232DFF
:10F74000322D21964FAD219725965FAD25970E94CA
:10F7500032BB181644F4382C292C2196AFAE2197D1
:10F760002596BFAE259720E030E0A901B401C50180
:10F770000E94AAB787FF04C0812C912CA12CB12C28
:10F7800022E0A401B501CE0180960E94E69ABE0156
:10F79000605E7F4FCE0101960E94419B65E57BE054
:10F7A000CE0101960E94E299BC0186EE92E10E9490
:10F7B0008E9ACE0101960E94DE9ACE0180960E941A
:10F7C000DE9A66EE72E1CE0101960E94419B4AE00C
:10F7D00050E070E060E0CE0101960E946857CE01D3
:10F7E00001960E94DE9A0E94F80FAB01BC01809145
:10F7F000E40C9091E50CA091E60CB091E70C8C59CB
:10F800009F4FAF4FBF4F84179507A607B70708F064
:10F81000AAC00E94A7546CE370E080E090E00E94D0
:10F8200039A58CAD9DADAEADBFAD0196A11DB11D8D
:10F830008CAF9DAFAEAFBFAFC816D906EA06FB06C8
:10F840000CF01BCF64E670E080E090E00E9439A5E8
:10F850000E94265764E670E080E090E00E9439A59F
:10F860006EEE7EE086EE92E10E94699A66EE72E1AB
:10F87000CE0101960E94419B44E150E070E060E0BF
:10F88000CE0101960E94885ACE0101960E94DE9A0E
:10F8900022E0432D522D21966FAD219725967FAD05
:10F8A0002597CE0180960E94E69ABE01605E7F4F4A
:10F8B000CE0101960E94419B65E57BE0CE01019659
:10F8C0000E94E299BC0186EE92E10E948E9ACE01DE
:10F8D00001960E94DE9ACE0180960E94DE9A66EE24
:10F8E00072E1CE0101960E94419B42E350E06FEF2E
:10F8F0007FEFCE0101960E946857CE0101960E94CB
:10F90000DE9A64E170E080E090E00E9439A50E94F8
:10F91000A7546EE170E080E090E00E9439A56EE1AE
:10F9200070E080E090E00E9439A56AE57BE0CE01BE
:10F9300001960E944A9B66EE72E1CE0101960E94FA
:10F94000F8996EE57BE00E94E2996CEE72E10E940C
:10F95000F899BC018CEE92E10E948E9ACE0101963C
:10F960000E94DE9AF9CD0E94F80F0E94AFB74B01BA
:10F970005C016091E40C7091E50C8091E60C909133
:10F98000E70C0E94B1B720E030E048EC51E40E945F
:10F990004BB99B01AC01C501B4010E94AAB787FD18
:10F9A00038CF39CF80917F049091800499270E94AD
:10F9B00036182DE038E643E55BE30E9410B86B0192
:10F9C0007C0120910705309108054091090550916F
:10F9D0000A050E94AAB718160CF47BC06091EF04C8
:10F9E0007091F0048091F1049091F20420E030E0F5
:10F9F00048EC52E40E9410B820E030E048EA51E4BC
:10FA00000E9410B82091D8043091D9044091DA04B2
:10FA10005091DB040E9429BA6B017C0163E07FE016
:10FA200086EE92E10E94699A66EE72E1CE0101963D
:10FA30000E94419B42E350E070E060E0CE010196FD
:10FA40000E94885ACE0101960E94DE9A22E0B701F8
:10FA5000A601CE0101960E94E69A68E67BE0CE01FF
:10FA600080960E944A9BBE016F5F7F4FCE018096B9
:10FA70000E94F89962E67BE00E94E299BC018CEE5C
:10FA800092E10E948E9ACE0180960E94DE9ACE016B
:10FA900001960E94DE9A6CEE72E1CE0101960E9400
:10FAA000419B42E350E06FEF7FEFCE0101960E9451
:10FAB0006857CE0101960E94DE9A8091300D88230E
:10FAC00009F44ACD60E273E080E090E00E9439A53D
:10FAD00043CD20911B0530911C0540911D0550918F
:10FAE0001E05C701B6010E9432BB87FF05C0C701D2
:10FAF000B6010E944D8F7ACF609103057091040585
:10FB0000809105059091060571CF0E94265767E305
:10FB10007FE08CEE92E10E94699A6CEE72E1CE0178
:10FB200001960E94419B4AE050E070E060E0CE0107
:10FB300001960E94885ACE0101960E94DE9A6EE2DA
:10FB40007FE086EE92E10E94699A66EE72E1CE0154
:10FB500001960E94419B44E150E06FEF7FEFCE01A0
:10FB600001960E946857CE0101960E94DE9A80910C
:10FB7000E80C9091E90C8230910509F041C00E9497
:10FB800021AB811104C01092E90C1092E80C809115
:10FB9000E80C9091E90C029709F448C062E27FE01A
:10FBA0008CEE92E10E94699A6CEE72E1CE010196B0
:10FBB0000E94419B4AE050E070E060E0CE01019677
:10FBC0000E94885ACE0101960E94DE9A6CEE72E184
:10FBD000CE0101960E94419B61E67AE0CE0101963A
:10FBE0000E94E29966EE72E10E94F899BC018CEEE7
:10FBF00092E10E948E9ACE0101960E94DE9A5DCF1C
:10FC0000892B61F60E9421AB882339F082E090E0D5
:10FC10009093E90C8093E80CBACF0E9421AB81113C
:10FC2000F5CF0E9421AB8111F1CFB1CF8AE090E0F6
:10FC30000E9411176B017C0120E030E0A9010E94B5
:10FC4000AAB7181634F08AE090E00E9411176B01F1
:10FC50007C018BE0A82EB12C20E030E042ED53E493
:10FC6000C701B6010E94AAB718168CF091E0A91A34
:10FC7000B10869F068EC70E080E090E00E9439A57E
:10FC800083E090E00E9411176B017C01E5CF20E03A
:10FC900030E0A901C701B6010E94AAB718166CF19D
:10FCA00064E17FE08CEE92E10E94699A6CEE72E171
:10FCB000CE0101960E94419B42E350E06FEF7FEF3F
:10FCC000CE0101960E946857CE0101960E94DE9AED
:10FCD0006BE07FE086EE92E10E94699A66EE72E147
:10FCE000CE0101960E94419B42E350E070E060E04B
:10FCF000CE0101960E94885ADCCE20E030E048EC2C
:10FD000052E4C701B6010E94AAB721E087FF20E0B4
:10FD1000B701A601CE0101960E94E69A67E67BE054
:10FD2000CE0180960E944A9BBE016F5F7F4FCE013D
:10FD300080960E94F8996CE67BE00E94E299BC01F3
:10FD40008CEE92E10E948E9ACE0180960E94DE9AFD
:10FD5000CE0101960E94DE9AA9CF0E94F80F2B01D6
:10FD60003C018AE99EE00E94F69064E670E080E043
:10FD700090E00E9439A540E855E260E070E08AE931
:10FD80009EE00E94F45764E670E080E090E00E94FC
:10FD900039A560E77FE086EE92E10E94699A66EEFF
:10FDA00072E1CE0101960E94419B42E350E06FEF69
:10FDB0007FEFCE0101960E94885ACE0101960E94E3
:10FDC000DE9A65E67FE086EE92E10E94699A66EE31
:10FDD00072E1CE0101960E94419B42E350E06FEF39
:10FDE0007FEFCE0101960E946857CE0101960E94D6
:10FDF000DE9A80912C0C90912D0C8D7F1CAEB12C35
:10FE0000A12CD12CC12CF12CE12C019709F47AC042
:10FE1000DE019096B9AFA8AFFE017E96FBAFEAAFC8
:10FE20000E94F80F6419750986099709683B7B40A1
:10FE30008105910508F066C08AE99EE00E94208B4A
:10FE4000892B09F44EC02CED35E040E050E02093C2
:10FE50009E0E30939F0E4093A00E5093A10E0E94D1
:10FE6000F88F97FD3EC082349105C9F7AE014F5F10
:10FE70005F4F1A014A010E94F88F97FF39C08981AC
:10FE80008D3479F590E080E0D1012D911D01820F34
:10FE9000911DEAADFBADEA17FB07B1F78E5B9F4FF3
:10FEA0002E8D30E0322F22274F8D240F311D8217E7
:10FEB0009307B9F4EC80F12CFE2CEE248D81E80E32
:10FEC000F11CCE80D12CDC2CCC248F81C80ED11C0F
:10FED000A884B12CBA2CAA248985A80EB11CF1E003
:10FEE000FCAF62E370E080E090E00E9439A598CF1B
:10FEF000D4018D934D01E8ADF9ADAE17BF0709F000
:10FF0000BACFBDCF0E94F80F641975098609970909
:10FF1000683B7B408105910518F43CAD3111BCC0B4
:10FF20000E94265766EE72E1CE0180960E94419BA8
:10FF300042E350E066E070E0CE0180960E94885A6D
:10FF4000CE0180960E94DE9A4CAD442309F4B3C0E2
:10FF500082E090E090932D0C80932C0CB501CE01A3
:10FF600080960E949598B601CE0186960E9495983B
:10FF7000B701CE01C2960E949598BE016E5C7F4F7C
:10FF8000CE018C960E94419B6CE978E0CE018C9664
:10FF90000E94E299BE016A5D7F4F0E94F8996CE968
:10FFA00078E00E94E299BE01605E7F4F0E94F8995E
:10FFB000BC018CEE92E10E948E9ACE018C960E943A
:10FFC000DE9ACE01C2960E94DE9ACE0186960E94EB
:10FFD000DE9ACE0180960E94DE9A6CEE72E1CE012E
:10FFE00080960E94419B4AE050E06FEF7FEFCE0188
:10FFF00080960E946857CE0180960E94DE9A6FE537
:020000021000EC
:100000007FE083EF93E10E94B59DB501CE0180961C
:100010000E949598B601CE0186960E949598B701E8
:10002000CE018C960E94959860E77BE0CE01C29647
:100030000E944A9BBE01645D7F4FCE01C2960E9422
:10004000F89961E67AE00E94E299BE016A5D7F4F0D
:100050000E94F89961E67AE00E94E299BE01605E32
:100060007F4F0E94F89960E87BE00E94E299BC0112
:100070008CEE92E10E948E9ACE01C2960E94DE9A88
:10008000CE018C960E94DE9ACE0186960E94DE9A60
:10009000CE0180960E94DE9A62E370E080E090E0FC
:1000A0000E9439A58AE99EE00E94F69062E370E022
:1000B00080E090E00BCD64E57FE08CEE92E10E9461
:1000C000699A6CEE72E1CE0180960E94419B4AE0F3
:1000D00050E070E060E0CE0180960E946857CE014B
:1000E00080960E94DE9A61E47FE08CEE92E10E94AD
:1000F000699A80912C0C90912D0C029769F61092C0
:100100002D0C10922C0CC8CFE0907904F0907A045A
:1001100066E87BE086EE92E10E945E980E94265798
:1001200066EE72E1CE0101960E94419B4AE050E0EA
:100130006FEF7FEFCE0101960E94885ACE010196A3
:100140000E94DE9AC7010E94471924966CAF7DAFCA
:100150008EAF9FAF24978090B1049090B204A0908E
:10016000B304B090B404A50194016091AD04709102
:10017000AE048091AF049091B0040E944AB92B0163
:100180003C0120E030E0A9010E94AAB7882309F4CD
:100190008EC0C090B904D090BA04E090BB04F09037
:1001A000BC0420E030E0A901C701B6010E94AAB753
:1001B00018160CF07CC08091B5049091B604A09103
:1001C000B704B091B8048CAF9DAFAEAFBFAF9C0188
:1001D000AD01C701B6010E94AAB7882309F467C020
:1001E000A70196016CAD7DAD8EAD9FAD0E9429BA81
:1001F0000E9481BB6CAF7DAF8EAF9FAFA501940114
:1002000024966CAD7DAD8EAD9FAD24970E944AB90A
:10021000A30192010E9429BA2CAD3DAD4EAD5FAD58
:100220000E9410B80E94A3BA9B01AC01C701B6019D
:100230000E9410B86B017C0166EE72E1CE0101965E
:100240000E94419B4AE050E070E060E0CE010196E0
:100250000E94885ACE0101960E94DE9A20E030E684
:100260004AEE56E4C701B6010E9432BB18161CF5CF
:100270006CE77FE08CEE92E10E94699A6CEE72E18D
:10028000CE0101960E94419B4AE050E06FEF7FEF64
:10029000CE0101960E946857CE0101960E94DE9A17
:1002A00064E670E080E090E00E9439A506CCC12CA5
:1002B000D12C7601C1CF21E0B701A601CE018096F5
:1002C0000E94E69A60E97BE0CE0101960E944A9B7B
:1002D000BE01605E7F4FCE0101960E94F89964E9ED
:1002E0007BE00E94E299BC018CEE92E10E948E9A22
:1002F000CE0101960E94DE9ACE0180960E94DE9A7F
:10030000BDCFE0900402F09005020E94265765E000
:1003100070E080E090E00E9439A580917B1140E080
:1003200050E0BA018330DCF4C7010E9436186B013B
:100330007C0160917C1170917D11072E000C880B5F
:10034000990B0E94B1B7A70196010E9410B820E056
:1003500030EC4FE754E40E9429BAAB01BC0123E022
:10036000CE0101960E94E69A6BE57BE0CE01809675
:100370000E944A9BBE016F5F7F4FCE0180960E9414
:10038000F89965E076E00E94E299BC018CEE92E17A
:100390000E948E9ACE0180960E94DE9ACE0101962E
:1003A0000E94DE9A68E97BE00C94B1788091000DA0
:1003B00091E089278093000D8091300D882331F0E2
:1003C0006CEE72E18DEF9DE00E94A39D68EC70E001
:1003D00080E090E07BCB1092300DBEC881E080932E
:1003E000300D8093EF118091E611882349F169E780
:1003F00078E088EF92E10E945E9886EE9FEF9093FE
:100400002B0C80932A0C2091E9113091EA118091F4
:10041000EB119091EC118217930724F01092EC11DC
:100420001092EB111092DD111092DE111092DF117B
:100430001092E0116CE271E080E090E00E9439A53A
:1004400068EF72E18EEF92E10E948E9A80912A0C01
:1004500090912B0C9093270D8093260D7DC80E94C0
:1004600089737AC887E39FE00E94F69040E052ECDF
:1004700061E070E087E39FE00E94F4578CED95E027
:10048000A0E0B0E080933B0F90933C0FA0933D0F12
:10049000B0933E0F64E670E080E090E00E9439A5E2
:1004A0008091E80C9091E90C019779F583E090E058
:1004B0000E94AB18811104C01092E90C1092E80C54
:1004C0008091E80C9091E90C0197C9F16BEB7FE00A
:1004D00086EE92E10E94699A66EE72E1CE01019683
:1004E0000E94419B44E150E06FEF7FEFCE01019607
:1004F0000E946857CE0101960E94DE9A6FEA7FE063
:100500008CEE92E10E94699A26C181E090E00E94FF
:10051000AB18882339F081E090E09093E90C809348
:10052000E80CCECF83E090E00E94AB188111F3CFAE
:1005300083E090E00E94AB188111EDCFC1CF63EA58
:100540007FE08CEE92E10E94699A6CEE72E1CE013E
:1005500001960E94419BCE0101960E94A359CE01B3
:1005600001960E94DE9A62E370E080E090E00E94D3
:1005700039A56CEE72E1CE0101960E94419B42E3E7
:1005800050E06FEF7FEFCE0101960E94885ACE01B6
:1005900001960E94DE9A67E97FE086EE92E10E9472
:1005A000699A66EE72E1CE0101960E94419B44E198
:1005B00050E06FEF7FEFCE0101960E946857CE01A9
:1005C00001960E94DE9A8BEB88A38AEA89A381E0D8
:1005D0008AA368011801412C512C3201C6016AE03E
:1005E00070E00E94C1BC892B49F443E050E0BE0199
:1005F000605E7F4F87E39FE00E94A98A65E070E01C
:1006000080E090E00E9439A5BFEFCB1ADB0A7801A9
:10061000812C912C540187E39FE00E94208B892B31
:1006200039F4E4E08E169104A104B1040CF049C041
:10063000F6E0EF16F1040CF044C087E39FE00E945F
:10064000208B892B71F087E39FE00E94FE8AE1E016
:10065000F0E0EC0FFD1FEE0DFF1D80832FEFE21A7F
:10066000F20A65E070E080E090E00E9439A536E093
:10067000E316F10401F5998188A198131CC09A81B1
:1006800089A1981318C09B818AA1981314C08D81E9
:1006900090E0B0E0A0E0BA2FA92F982F88272C81F6
:1006A000820F911DA11DB11D480E591E6A1E7B1E91
:1006B0004FEF241A340A5FEF851A950AA50AB50A86
:1006C000AACF94E02916310434F4A0E9CA16A1E0B7
:1006D000DA0609F083CFC301B2010E94B1B720E06E
:1006E00030E040E251E40E9429BA20E030E040E8E6
:1006F0005EE30E9410B86B017C0120E030E040EA2C
:1007000051E40E9432BB18160CF055C021E0B7012D
:10071000A601CE0101960E94E69A6BEE77E0CE012B
:1007200080960E944A9BBE016F5F7F4FCE018096EC
:100730000E94F89960EA7BE00E94E299BC018CEE8D
:1007400092E10E948E9ACE0180960E94DE9ACE019E
:1007500001960E94DE9A6CEE72E1CE0101960E9433
:10076000419B4AE050E070E060E0CE0101960E94BB
:10077000885ACE0101960E94DE9A6CEE72E1CE019B
:1007800001960E94419B61E67AE0CE0101960E94AB
:10079000E29966EE72E10E94F899BC018CEE92E15A
:1007A0000E948E9ACE0101960E94DE9A87E39FE016
:1007B0000E94F69082C96BE87FE0A2CE66E570E108
:1007C000CE0101960E94389B4AE050E06FEF7FEF28
:1007D000CE0101960E946857CE0101960E94DE9AD2
:1007E00060918604709187048091D2049091D30423
:1007F0000E94B55464E1862E912CA12CB12CD12CF1
:10080000C12CAFEFCA1ADA0AC501B4010E9439A59A
:1008100060918604709187048091D2049091D304F2
:100820000E94B5547C01B3E0CB16D10434F08EE1C4
:10083000C816D10444F4EF2851F094E1890E911CBC
:10084000A11CB11CDECFE114F10409F00CC18091B0
:10085000D2049091D3048B30910509F0DFC08091D0
:100860004A1390914B13A0914C13B0914D13809368
:10087000260C9093270CA093280CB093290C809100
:10088000461390914713A0914813B0914913809358
:10089000220C9093230CA093240CB093250C409130
:1008A000260C5091270C6091280C7091290C21E0A6
:1008B000CE0101960E94E69A62EE76E0CE01809625
:1008C0000E944A9BBE016F5F7F4FCE0180960E94BF
:1008D000F899BC018CEE92E10E948E9ACE0180962E
:1008E0000E94DE9ACE0101960E94DE9A4091220C6F
:1008F0005091230C6091240C7091250C21E0CE01C5
:1009000001960E94E69A61EA77E0CE0180960E9405
:100910004A9BBE016F5F7F4FCE0180960E94F8997F
:10092000BC018CEE92E10E94629ACE0180960E94F8
:10093000DE9ACE0101960E94DE9A65E67BE08CEE9F
:1009400092E10E94589A6BEF7BE0CE0101960E94E3
:100950004A9B44E150E070E060E0CE0101960E94C5
:10096000885ACE0101960E94DE9AC090260CD09043
:10097000270CE090280CF090290C20E030E0A90131
:10098000C701B6010E9432BB20E030E040E05FE3E7
:1009900087FD64C0C701B6010E944BB90E94D5BA59
:1009A000AB01BC01CE0101960E946898BE016F5F49
:1009B0007F4F86EE92E10E94A59ACE0101960E9499
:1009C000DE9A60E087E00E94F68D66EE72E183EFCA
:1009D00093E10E94959D6FED83EF93E10E941A9C35
:1009E00067EA77E083EF93E10E94939D6091220C88
:1009F0007091230C8091240C9091250C0E94D5BA03
:100A00004AE050E083EF93E10E94469D65E67BE07B
:100A100083EF93E10E94939D0C94E47886319105D5
:100A200009F41DCF0C9709F03ACF8091190C9091E1
:100A30001A0CA0911B0CB0911C0C8093260C909367
:100A4000270CA093280CB093290C8091150C909141
:100A5000160CA091170CB091180C19CFC701B60154
:100A60000E944AB99BCFEFEFEE16FE06D4F068E481
:100A700070E1CE0101960E94389B4AE050E070E0A0
:100A800060E0CE0101960E94885ACE0101960E9434
:100A9000DE9A65E270E18CEE92E10E94699A0C9414
:100AA000AC7AFEEFEF16FFEFFF0681F167E170E130
:100AB000CE0101960E94389B4AE050E070E060E071
:100AC000CE0101960E94885ACE0101960E94DE9ABC
:100AD00068E070E18CEE92E10E94699AB701CE0164
:100AE00001960E949598BE016F5F7F4F8CEE92E158
:100AF0000E94629ACE0101960E94DE9A62EF7FE028
:100B00008CEE92E10E940B9A0C94AC7A67EE7FE037
:100B1000CE0101960E94389B4AE050E070E060E010
:100B2000CE0101960E94885ACE0101960E94DE9A5B
:100B300067EC7FE0B0CF80919004882311F40C948F
:100B4000AC7A6BEF7BE0CE0101960E944A9B4AE0B3
:100B500050E061E070E0CE0101960E94885ACE011B
:100B600001960E94DE9A0E947C5E0C94AC7A809181
:100B7000300D811109C08091E1115EE1452E512CAB
:100B8000612C712C882329F043E0442E512C612CD8
:100B9000712C64E670E18CEE92E10E94699A6CEE31
:100BA00072E1CE0101960E94419B4AE050E06FEF56
:100BB0007FEFCE0101960E946857CE0101960E94F8
:100BC000DE9A812C912C54011CAE1DAE1EAE1FAEC0
:100BD00083E20E94DB8D87E090E00E94D68D0E9428
:100BE000FCA266E970E080E090E00E9439A583E213
:100BF0000E94DB8D80E290E00E94D68D0E94FCA2D4
:100C000066E970E080E090E00E9439A562E070E063
:100C100083E290E00E94E3A3C12CD12C7601809165
:100C20005A0D90915B0D891B990B181619065CF4EF
:100C30000E941491FE2CED2CDC2CCC24C80ED11C6F
:100C4000E11CF11CECCFC701B6010E94B1B72AE943
:100C500039E949E95FE30E9429BA0E94D5BAAB019C
:100C6000BC0184169506A606B70614F44A015C0179
:100C7000CE0180960E946898BE01605E7F4FCE01D3
:100C800001960E94419B63EA7BE0CE0101960E949F
:100C9000E299BC0186EE92E10E948E9ACE01019605
:100CA0000E94DE9ACE0180960E94DE9A66EE72E184
:100CB000CE0101960E94419B4EE150E070E060E061
:100CC000CE0101960E94CF59CE0101960E94DE9A74
:100CD0002CAD3DAD4EAD5FAD2F5F3F4F4F4F5F4FE2
:100CE0002CAF3DAF4EAF5FAF42165306640675069C
:100CF0000CF06ECFB501A401CE0180960E946898D9
:100D0000BE01605E7F4FCE0101960E94419B63EA67
:100D10007BE0CE0101960E94E299BC0186EE92E151
:100D20000E948E9ACE0101960E94DE9ACE01809694
:100D30000E94DE9A66EE72E1CE0101960E94419B0E
:100D40004AE050E070E060E0CE0101960E94885ACF
:100D5000CE0101960E94DE9AB501A401CE01019652
:100D60000E94689866E776E0CE0180960E944A9BD2
:100D7000BE016F5F7F4FCE0180960E94F89967EAAF
:100D80007BE00E94E2996CEE72E10E94F899BC014E
:100D90008CEE92E10E948E9ACE0180960E94DE9A9D
:100DA000CE0101960E94DE9A81C9E0900202F09085
:100DB000030281E08093E40464E670E080E090E068
:100DC0000E9439A50E942657C7010E9436180E942A
:100DD000D5BA20E034E0A901461B570BBA01CE0179
:100DE00001960E9495986CEA7BE0CE0180960E9465
:100DF0004A9BBE016F5F7F4FCE0180960E94F8999B
:100E0000BC018CEE92E10E948E9ACE0180960E94E7
:100E1000DE9ACE0101960E94DE9A60E087E00E9491
:100E2000F68D64E770E1CE0101960E94389B42E3A3
:100E300050E068E070E0CE0101960E94885ACE0131
:100E400001960E94DE9A6CEE72E1CE0101960E943C
:100E5000419B42E350E06FEF7FEFCE0101960E948D
:100E60006857CE0101960E94DE9A63EB7BE0CE01CB
:100E700001960E944A9B6CEE72E1CE0101960C94A1
:100E8000F47D80910002909101020E9436180E9428
:100E9000D5BA7093EB0C6093EA0C62E370E080E0EB
:100EA00090E00E9439A56091EA0C7091EB0CCE01A4
:100EB00001960E949598BE016F5F7F4F8CEE92E184
:100EC0000E94A59ACE0101960E94DE9A8091441359
:100ED00090914513892B09F45EC060E473E1CE0163
:100EE00080960E94419BBE01605E7F4FCE010196BD
:100EF0000E94419B44E150E070E060E0CE01019629
:100F00000E94885ACE0101960E94DE9A6DEB7BE02A
:100F1000CE0101960E944A9B6CEE72E1CE010196D1
:100F20000E94F899BC0186EE92E10E948E9ACE0151
:100F300001960E94DE9A66EE72E1CE0101960E9451
:100F4000419B44E150E06FEF7FEFCE0101960E949C
:100F50006857CE0101960E94DE9ABE01605E7F4F07
:100F6000CE0101960E94419B61E67AE0CE01019696
:100F70000E94E29966EE72E10E94F899BC018CEE43
:100F800092E10E948E9ACE0101960E94DE9ACE01D5
:100F900080960C945B7D68EC7BE086EE92E10E948B
:100FA0005E9866EE72E1CE0101960E94419B44E19B
:100FB00050E070E060E0CE0101960E94885ACE01B8
:100FC00001960E94DE9A6CEA7BE0CE0101960E94B7
:100FD0004A9B6CEE72E1CE0101960E94F899BC0129
:100FE00086EE92E10E948E9ACE0101960E94DE9AD0
:100FF00066EE72E1CE0101960E94419B44E150E011
:101000006FEF7FEFCE0101960E946857CE010196E7
:101010000E94DE9A6DEB7BE02ACF809190048823BA
:1010200011F40C94AC7A8091300D811104C0809140
:10103000E111882331F082E090E00E94FD5F0C9482
:10104000AC7A0E949EA70C94AC7A0E942B5B8DEF29
:101050009DE00E94C38B0C94AC7A6CE870E186EE44
:1010600092E10E94699A66EE72E1CE0101960E94B9
:10107000419B4AE050E070E060E0CE0101960E94A2
:10108000885ACE0101960E94DE9A30900602809125
:10109000F80C811105C00E94F80F81E08093F80CD4
:1010A0008091F00C811105C00E94F80F81E08093BF
:1010B000F00C1092130C1092120CE090120CF090A5
:1010C000130C58E2E516F1040CF07EC0832D0E944B
:1010D000C4A1F701EE0FFF1FE25AF24F9183808304
:1010E0000E94238E20E030E040EA50E40E9410B8D5
:1010F00020E030E040E85AE30E9410B86B017C0128
:101100004090A9045090AA046090AB047090AC0485
:10111000A30192016091A5047091A6048091A70497
:101120009091A8040E944AB99B01AC0160E070E074
:1011300080EC90E40E944AB94B015C0120E030E071
:10114000A9010E94AAB720E030E040E650E48111F6
:101150001CC0C701B6010E9410B86093EC0C7093DC
:10116000ED0C8093EE0C9093EF0C64E170E080E066
:1011700090E00E9439A58091120C9091130C019679
:101180009093130C8093120C98CFC701B6010E9464
:1011900010B8A30192010E944BB920E030E040E872
:1011A00050E40E944AB9A50194010E9429BA20E0A6
:1011B00030E040EC50E40E9410B820E030E040E81D
:1011C00050E40E944BB9C9CFC090EC0CD090ED0C0C
:1011D000E090EE0CF090EF0C20E030E0A901C701A8
:1011E000B6010E9432BB87FD22C022E0B701A601F2
:1011F000CE0180960E94E69A6CEC7BE0CE010196CF
:101200000E944A9BBE01605E7F4FCE0101960E9404
:10121000F899BC018CEE92E10E948E9ACE01019663
:101220000E94DE9ACE0180960E94DE9A06C06DE78B
:1012300070E18CEE92E10E94699A6CEE72E1CE014F
:1012400001960E94419B4AE050E00C945E788091A8
:101250009004882311F40C94AC7A8091300D8111A4
:101260002EC08091E11181112AC0C090EB04D09072
:10127000EC04E090ED04F090EE0420E030E04AE76A
:1012800054E4C701B6010E9410B80E94D5BA4B01C0
:101290005C0120E030E040EA50E4C701B6010E9462
:1012A00010B820E030E040EA50E40E944BB90E94C0
:1012B000D5BAA50194010E9409640C94AC7A21E08E
:1012C00030E040E050E06AE070E080E090E0F3CF92
:1012D000C7010E94A9500C94AC7AC7010E9438261D
:1012E0000C94AC7A8091310D882311F40C94AC7A73
:1012F0006AED70E1CE0101960E94389BCE01019605
:101300000E94F256CE0101960E94DE9A0C94AC7AAD
:1013100080915C0D90915D0D892B81F481E090E0CE
:1013200090935D0D80935C0D8EE492E00E942A9074
:1013300068EC70E080E090E00E9439A56DEC70E10F
:10134000CE0101960E94389B44E650E06FEF7FEF9C
:10135000CE0101960E946857CE0101960E94DE9A46
:10136000F0E0E0E019950C94AC7A0E94E4AB0E94A6
:1013700026570E94D5160C94AC7A8091E61191E024
:1013800089278093E611882309F48BC066EC70E10D
:101390008CEE92E10E94699A0E94F80F6093DD1131
:1013A0007093DE118093DF119093E0118091E91129
:1013B0009091EA11181619065CF42091EB11309106
:1013C000EC112817390724F01092EC111092EB1150
:1013D0009091ED118091E811981724F01092ED1181
:1013E0001092EE118091E6118093E1116CEE72E1A2
:1013F000CE0101960E94419B4AE050E068E070E017
:10140000CE0101960E94885ACE0101960E94DE9A72
:1014100061EB70E1CE0101960E94389B4AE050E0FA
:101420006FEF7FEFCE0101960E946857CE010196C3
:101430000E94DE9A63EA70E18CEE92E10E940B9AC0
:1014400060EC75E0CE0101960E944A9B6CEE72E161
:10145000CE0101960E94F899BC018CEE92E10E94A7
:101460008E9ACE0101960E94DE9A8091300D809373
:10147000EF118CE291E00E9455908091300D88230D
:1014800011F40C94AC7A69E778E088EF92E10E945D
:101490005E9886EE9FEF90932B0C80932A0C0C9411
:1014A000AC7A6EEB70E18CEE92E10E94699A9ACF71
:1014B000F0922B0CE0922A0C8DEF9DE00E94C38BE2
:1014C00065E970E18CEE92E10E94699A6BEF7BE036
:1014D000CE0101960E944A9B4AE050E070E060E035
:1014E000CE0101960E94885ACE0101969DCE0E3FF4
:1014F000FFEF1F0711F40C94BD776BEF7BE08CEED0
:1015000092E10E945E980C94887796E0899FD001C2
:101510001124A859BC4E90967C936E935F9791E0EE
:1015200091969C939197E091D513F091D613909159
:10153000D413992339F0309751F0811108C080916C
:1015400084131994309719F05C968C91FACF089512
:101550000895AF92BF92CF92DF92EF92FF920F93D6
:101560001F93CF93DF936C017B018B01040F151F39
:10157000EB015E01AE18BF08C017D10759F06991A1
:10158000D601ED91FC910190F081E02DC6011995F5
:10159000892B79F7C501DF91CF911F910F91FF90B2
:1015A000EF90DF90CF90BF90AF900895FC01A0899D
:1015B000B1898C91A689B78982FD0FC09C91818DDC
:1015C0008F5F8F73228D821749F0A18DAE0FBF2FD1
:1015D000B11D5D969C93818F08958C910895FC01B7
:1015E000538D448D252F30E0842F90E0821B930B88
:1015F000541710F0CF96089501970895FC01918D2E
:10160000828D981761F0A28DAE0FBF2FB11D5D9630
:101610008C91928D9F5F9F73928F90E008958FEFD2
:101620009FEF0895FC01918D828D981731F0828D86
:10163000E80FF11D858D90E008958FEF9FEF0895DD
:10164000FC01918D228D892F90E0805C9F4F821B41
:1016500091098F73992708958DEF9DE00E94208B4B
:1016600021E0892B09F420E0822F08958AE99EE089
:101670000E94208B21E0892B09F420E0822F08951D
:1016800087E39FE00E94208B21E0892B09F420E072
:10169000822F089584ED9FE00E94208B21E0892B0A
:1016A00009F420E0822F0895FC01A48DA80FB92F22
:1016B000B11DA35ABF4F2C91848D90E001968F737A
:1016C0009927848FA689B7892C93A089B1898C9199
:1016D000837080648C93938D848D981306C00288E8
:1016E000F389E02D80818F7D80830895EF92FF92B2
:1016F0000F931F93CF93DF93EC0181E0888F9B8D35
:101700008C8D98131AC0E889F989808185FF15C0EE
:101710009FB7F894EE89FF896083E889F989808111
:101720008370806480839FBF81E090E0DF91CF91E0
:101730001F910F91FF90EF900895F62E0B8D10E002
:101740000F5F1F4F0F731127E02E8C8D8E110CC071
:101750000FB607FCFACFE889F989808185FFF5CFBC
:10176000CE010E94548BF1CFEB8DEC0FFD2FF11DBC
:10177000E35AFF4FF0829FB7F8940B8FEA89FB89F9
:1017800080818062CFCFCF93DF93EC01888D882357
:10179000B9F0AA89BB89E889F9898C9185FD03C0D4
:1017A000808186FD0DC00FB607FCF7CF8C9185FFB9
:1017B000F2CF808185FFEDCFCE010E94548BE9CF1F
:1017C000DF91CF91089580E090E0892B29F00E946D
:1017D0004A8B81110E94000080E090E0892B29F063
:1017E0000E94408B81110E94000080E090E0892BD4
:1017F00029F00E94368B81110E94000080E090E069
:10180000892B29F00E942C8B81110C9400000895E3
:101810008150823108F05AC0E82FF0E08827EC5E52
:10182000F3478F4F0C94D5BC348C388C268C2C8C81
:10183000308C668C3B8C418C458C4B8C4F8C538C04
:10184000598C5D8C668C618C678C6B8C8091800070
:101850008F77809380000895809180008F7DF9CFED
:1018600080918000877FF5CF84B58F7784BD089500
:1018700084B58F7DFBCF8091B0008F778093B000CF
:1018800008958091B0008F7DF9CF809190008F777F
:10189000809390000895809190008F7DF9CF809182
:1018A0009000877FF5CF8091A0008F778093A00074
:1018B00008958091A0008F7DF9CF8091A000877F4F
:1018C000F5CF809120018F7780932001089580913A
:1018D00020018F7DF9CF80912001877FF5CF0F9375
:1018E0001F93CF93DF93C82FD62F86E0C89FF001B8
:1018F0001124E859FC4E11A2878D90A181309105E9
:10190000F1F058F082309105F1F1039709F440C0ED
:10191000DF91CF911F910F9108956623C9F361E084
:1019200070E08C2F0E94858A0E94F80F6093C0138C
:101930007093C1138093C2139093C313E9CF0E9495
:10194000F80F0091C0131091C1132091C213309170
:10195000C313AB01BC01401B510B620B730B809195
:10196000D2139091D313B0E0A0E084179507A60797
:10197000B70748F462E070E08C2FDF91CF911F91A0
:101980000F910C94858A63E070E0D111C1CFF4CF40
:1019900070E060E0F1CF8F929F92AF92BF92CF92B2
:1019A000DF92EF92FF920F931F93CF93DF93DB01B0
:1019B000ED91FC91EC01AC85BD8501E010E0EA17EA
:1019C000FB070CF045C0EF01CC0FDD1FDC011A96C0
:1019D0008D919C91DC01AC0FBD1FAD90BC908F012F
:1019E00000951095017011278CE99FEFE0FF02C070
:1019F00084E690E0E9016A017B014C01820E931EAE
:101A0000B401C5010E94611421E030E0892BB9F4D2
:101A10008C0E9D1EB401C5010E94611422E030E0CD
:101A2000892B69F4BE01680D791DC5010E946114FE
:101A300023E030E0892B19F40FEF1FEF09C0E60116
:101A40008881998101968217930784F4998388830A
:101A5000C801DF91CF911F910F91FF90EF90DF9020
:101A6000CF90BF90AF909F908F9008951982188269
:101A7000D7018D919C91119701968D939C93E8CFFE
:101A8000FB0101900020E9F73197AF01461B570B8E
:101A9000DC01ED91FC910280F381E02D1994CF934C
:101AA000DF93EC0188819981009711F00E94C3BDFA
:101AB000198218821D821C821B821A82DF91CF91AB
:101AC00008950F931F93CF93DF93EC018881998141
:101AD000009759F02A813B812617370730F081E0C3
:101AE000DF91CF911F910F9108958B016F5F7F4F11
:101AF0000E944CBE009759F0998388831B830A8308
:101B00002C813D81232B59F7FC011082E8CF80E026
:101B1000E7CFEF92FF920F931F93CF93DF9361155F
:101B2000710541F480E0DF91CF911F910F91FF90FB
:101B3000EF90089541155105B1F07B01EC010C8146
:101B40001D81040F151FB8010E94618D882351F378
:101B5000288139818C819D81B701820F931F0E945A
:101B600077BF1D830C8381E0DECFEF92FF920F934E
:101B70001F93CF93DF93EC017B018A01BA010E948E
:101B8000618D81110BC0CE010E944F8DCE01DF917E
:101B9000CF911F910F91FF90EF9008951D830C83BB
:101BA000B701888199810E9477BFF0CF682F81E7C4
:101BB00090E10C94580C91E09093DA0D8093FF1310
:101BC0001092DB0D1092FC0D0895CF93C82F682F53
:101BD000607F83EF93E10E94851380E1C89FB0018D
:101BE000112483EF93E1CF910C948513CF93DF936E
:101BF00000D000D01F921F92CDB7DEB798E0E3E689
:101C0000F5E0DE01119601900D929A95E1F7909121
